:020000040000FA
:10800000F00E0120E58200002583000009820000B7
:10801000298300002B8300002D8300000000000056
:1080200000000000000000000000000025820000A9
:1080300031830000000000008182000089AE000052
:108040003783000037830000378300003783000048
:108050003783000037830000378300003783000038
:10806000BDB4000037830000378300003783000071
:108070003783000037830000378300003783000018
:1080800037830000619F0000D19F0000378300000C
:108090003783000025A000003783000037830000ED
:1080A00037830000378300003783000037830000E8
:1080B00037830000378300003783000037830000D8
:1080C00091B00000A5B00000B9B00000CDB0000034
:1080D000E1B0000011B100003783000037830000D9
:1080E00037830000378300003783000037830000A8
:1080F0003783000037830000378300003783000098
:1081000041B1000071B100003783000037830000E7
:108110003783000037830000378300003783000077
:10812000998A0000158B0000378300003783000018
:108130003783000037830000378300003783000057
:108140003783000037830000378300003783000047
:108150003783000037830000378300003783000037
:108160003783000037830000A1B10000D1B10000C7
:108170003783000037830000378300003783000017
:108180003783000037830000378300003783000007
:1081900037830000378300003783000037830000F7
:1081A00059A00000378300003783000037830000A8
:1081B00037830000378300003783000037830000D7
:1081C00037830000378300003783000037830000C7
:1081D000378300003783000001B2000031B2000095
:1081E00037830000378300003783000037830000A7
:1081F00037830000DFF80CD000F010FC0048004787
:10820000A50D0200F00E012004207146084202D0A4
:10821000EFF3098001E0EFF308807146004A104750
:1082200045A100002C4B19680868B0E8F04F80F3B6
:108230000988BFF36F8F4FF0000080F311887047FB
:108240000000000008480068006880F308884FF0CC
:10825000000080F3148862B661B6BFF34F8FBFF39E
:108260006F8F00DF00BF00BF08ED00E0DFF80C00FB
:10827000016841F470010160704700BF88ED00E0C3
:10828000EFF30980BFF36F8F134B1A681EF0100FC6
:1082900008BF20ED108A20E9F04F106009B44FF0BC
:1082A000500080F31188BFF34F8FBFF36F8F2DF015
:1082B00003F84FF0000080F3118809BC19680868C2
:1082C000B0E8F04F1EF0100F08BFB0EC108A80F33A
:1082D0000988BFF36F8F70472C330020EFF30580C0
:1082E0007047000014484FF0590101604FF016012B
:1082F00001604FF0880101601048416841F48041FD
:1083000041600F48416841F002014160416841F01D
:10831000040141600B48804707484FF000010160AD
:1083200009480047FEE7FEE7FEE7FEE7FEE7FEE757
:10833000FEE7FEE7FEE7FEE7000100400002004026
:108340000070004021AF0000F58100002DE9F05FD2
:108350000546002092469B468846064681464024B4
:108360001BE0284641464746224600F0A1FA534604
:108370005A46C01A914110D311461846224600F0C1
:1083800016F82D1A67EB01084F46224601200021FE
:1083900000F00DF817EB00094E41201EA4F1010476
:1083A000DFDC484631462A464346BDE8F09F202A96
:1083B00004DB203A00FA02F1002070479140C2F13C
:1083C000200320FA03F319439040704740EA010369
:1083D0009B0703D009E008C9121F08C0042AFAD27B
:1083E00003E011F8013B00F8013B521EF9D270473F
:1083F000D2B201E000F8012B491EFBD270470022E7
:10840000F6E710B513460A4604461946FFF7F0FF93
:10841000204610BD421C10F8011B0029FBD1801A18
:108420007047034611F8012B00F8012B002AF9D1FF
:10843000184670472DE9FE4F804681EA0300C00FC1
:108440000C46009021F0004123F00045B8EB0200FB
:10845000A94105D24046214690461C460B4602469D
:1084600023F00040104347D0270DC7F30A00C3F3A1
:108470000A510290401A019040286BDAC3F31300AE
:1084800040F4801B0098924620B10023D2EB030AEF
:1084900063EB0B0B01985946C0F140025046FFF7C1
:1084A00086FF06460D4650465946019A00F010FADE
:1084B00010EB08006141002487EA115284EAE77357
:1084C0001A4340D0009A62B3019A012A4FEA075238
:1084D00015DC001B61EB02014FF0004202EA07527B
:1084E000CDE90042001C41F5801132462B4600F0D8
:1084F00047FA03B0BDE8F08F40462146F9E7001B7C
:1085000061EB0201001C41F5801300185B4120184B
:10851000A2F5001747EB030140EAD570B6196D418B
:1085200011E06D084FEA360645EAC0754FEA07527A
:10853000001B61EB0201001C41F5801149084FEA64
:1085400030000019514132462B4603B0BDE8F04FD0
:1085500000F007BA0098012240000023D0EB02028D
:1085600063EBE073009821464FEAE074B8EB00003B
:1085700061EB0401E9E783F000435BE781F0004130
:1085800058E72DE9FE4F81EA030404F0004421F08E
:10859000004100944FF0000B23F0004350EA010427
:1085A0005ED052EA03045BD0C3F30A54C1F30A5508
:1085B0002C44A4F2F3340194A0FB0254C1F3130140
:1085C00041F48011C3F3130343F4801301FB02440D
:1085D00000FB034E840A970A44EA815447EA835712
:1085E000A4FB076802958D0A05FB07854FEA932CCB
:1085F00004FB0C542705029D4FEA065847EA16373C
:10860000B5EB08056EEB070C870E920E47EA811753
:1086100042EA8312A7FB0201B6EB0B0164EB0004F4
:108620002B0D43EA0C335E1844EB1C50DA465146DE
:10863000E7FB0201C5F313044FEA0B3343EA14537B
:108640004FEA0432019C43EA0603A4F10C040294AD
:10865000009CCDE900B400F093F903B0BDE8F08FC1
:1086600000200146F9E72DE9F04D81EA030404F00A
:10867000004B21F0004514464FF0000A23F0004162
:1086800050EA050220D054EA01021DD0C5F30A5772
:108690000246C5F31303C1F31300C1F30A5640F4B5
:1086A000801543F48013A7EB0608101BD64608F28A
:1086B000FD3873EB050002D308F1010801E09218C0
:1086C0005B41B8F1000F03DA00200146BDE8F08DF0
:1086D00000204FF48011064684460EE0171B73EB12
:1086E000050705D3121B63EB050306434CEA010C97
:1086F00049084FEA300092185B4150EA0107EDD17A
:1087000052EA030012D082EA040083EA050108431A
:1087100005D0101BAB4106D20122002306E0002247
:108720004FF0004302E06FF0010253101AEB060015
:108730004CEB085110EB0A0041EB0B01BDE8F04D8A
:1087400000F00FB90EB5C10F80EAE0700844CA0707
:10875000002140F233438DE80E000A460B4600F03C
:108760000FF903B000BD0EB540F233410291002174
:10877000CDE900110A460B4600F002F903B000BD36
:1087800070B5C1F30A5201F000450024C1F3130192
:1087900040F2FF3341F480119A4201DA002070BDAB
:1087A00040F233439A42A2F2334203DC524200F0D9
:1087B0007FF800E090402C43F1D0404270BDC1F3FF
:1087C0000A5210B5C1F3130140F2FF3341F4801196
:1087D0009A4201DA002010BD40F233439A42A2F2DD
:1087E000334203DC524200F063F810BD904010BDEC
:1087F00000F0004230F000400AD0C10D01F5607178
:10880000C0F3160042EA0151C20840071143704705
:10881000002001467047000030B5041E71F10004CD
:1088200004DB4FF00044404264EB0101141E73F17D
:10883000000405DB1C464FF00043524263EB040387
:108840008B4208BF824230BD30B5041E71F1000476
:1088500004DB4FF00044404264EB0101141E73F14D
:10886000000405DB1C464FF00043524263EB040357
:10887000994208BF904230BD01F0004330B421F06E
:10888000004150EA010206D00A0DA2F56072C1F360
:108890001301002A02DC30BC00207047440F44EA78
:1088A000C104C100E01830BC00EBC25000F022B897
:1088B000202A04DB203A21FA02F00021704721FA35
:1088C00002F3D040C2F1200291400843194670479C
:1088D000202A06DBCB17203A41FA02F043EAE07384
:1088E00006E041FA02F3D040C2F120029140084371
:1088F000194670470029A8BF7047401C490008BFAF
:1089000020F00100704710B4B0FA80FC00FA0CF0BF
:1089100050EA010404BF10BC704749B1CCF12004F7
:1089200021FA04F411FA0CF118BF01212143084384
:10893000A3EB0C01CB1D4FEA00614FEA102042BFB0
:10894000002010BC704700EBC35010440029A4BFA6
:1089500010BC7047401C490008BF20F0010010BC4B
:10896000704710B5141E73F1000408DA401C41F181
:10897000000192185B411A4301D120F0010010BDA3
:108980002DE9F04D92469B4611B1B1FA81F202E019
:10899000B0FA80F220329046FFF709FD04460F46F8
:1089A00040EA0A0041EA0B0153465A46084313D0F5
:1089B000114653EA010019D0C8F140025046FFF7B2
:1089C00077FF05460E46504659464246FFF7EFFCF4
:1089D000084305D0012004E020463946BDE8F08D6B
:1089E0000020054346EAE0762C4337430A986305A6
:1089F000E40AA0EB08000022FD0A44EA47540A30CA
:108A000002D500200146E9E7010510196941DDE9B9
:108A1000084500196941BDE8F04DA2E7064C074D35
:108A200006E0E06840F0010394E80700984710343E
:108A3000AC42F6D3FFF7E2FBC8890300E8890300E4
:108A400070B58C1810F8015B15F0070301D110F810
:108A5000013B2A1106D110F8012B03E010F8016B3D
:108A600001F8016B5B1EF9D12B0705D40023521EC0
:108A70000DD401F8013BFAE710F8013BCB1A921C28
:108A800003E013F8015B01F8015B521EF9D5A14226
:108A9000D8D3002070BD000010B51C480469B4F59F
:108AA000004F1DD1406800F0100028B11748406801
:108AB00020F0100015494860144840681348406889
:108AC0001248406800F08000F8B141200F4908606A
:108AD0000846006820F0410008600E20086014E09D
:108AE00064B1601EC1B200200EF050F80748006962
:108AF000401EC1B2054800F00FF906E004480068C6
:108B0000012802D100200249086010BD00000A407F
:108B10006C010A4010B51B480469B4F5004F1DD123
:108B2000406800F0100028B11648406820F010009E
:108B3000144948601348406812484068114840682A
:108B400000F08000E8B141200E4908600846006846
:108B500020F0410008600E20086012E054B1601E51
:108B6000C1B201200EF012F8601EC1B2054800F03B
:108B7000D3F806E004480068012802D10020024929
:108B8000086010BD00100A406C110A4010B5024682
:108B9000012098239B5803F400430BB9002047E0C1
:108BA000536823F010035360332484239C50942390
:108BB0009B5803F480433BB900230B6094239B58DC
:108BC000C3F38A038B600BE001230B6094239B5853
:108BD000DB04DB088B6090239B588C681C438C6003
:108BE00094239B58C3F3403383F001034B609823D5
:108BF0009B5803F00F030B739C239B584B739C23D0
:108C00009B581C0A8C73D2F8A030CB73D2F8A030DA
:108C10001C0A0C74D2F8A4304B74D2F8A4301C0A8D
:108C20008C74D2F8A830CB74D2F8A8301C0A0C751A
:108C300010BD000070B502460023012434480568C9
:108C400005E05B1CAB4202D94FF0FF3070BD106AEB
:108C500000F400400028F4D1506820F00800506073
:108C6000086830B90026166308894005C60C5663AB
:108C700008E0088986B216638868C0F30C4040F4A7
:108C800080465663486820B1506B40F400565663E6
:108C900003E0506B20F400565663906B20F00F00F9
:108CA0000E7B304390634E7B887B46EA0026D6637A
:108CB000CE7B087C46EA002616644E7C887C46EA19
:108CC00000265664CE7C087D46EA00269664106A2B
:108CD00020F400401062106A00F4004008B1002443
:108CE00013E0106A40F400401062002305E0106AAF
:108CF00000F4004000B903E05B1C06488342F6D351
:108D000000BF0448834200D3002420469EE70000B1
:108D100000000020FFFF0F0070B504460E462046FD
:108D200001F052FE0546022800D100250C2105EB7A
:108D3000450204F1200000EB42104160701C05EB7D
:108D4000450204F1200101EB42110860294620464A
:108D500001F0A2FE70BD026822F00E0201F00E03C7
:108D60001A430260704741F0410202607047026896
:108D700042F0800202604161704710B5024610293E
:108D800005D2D2F8200101238B40184010BDD2F843
:108D90002401A1F1100301249C402040F6E70000CB
:108DA000084A1168026822F04102026002E001B93B
:108DB00005E0491E026802F00102002AF7D100BF57
:108DC00070470000000000202DE9F04105460E46E6
:108DD00014463146284600F0FFF80746012C03D11F
:108DE00004212846FFF7C3FF3846BDE8F0810000A4
:108DF0002DE9F04704460F4690461E464FF0010A03
:108E0000644800684FEA400939462046FFF7B5FF3D
:108E100010B94FF0000ABAE0204601F0D5FD054632
:108E2000022802D14FF0000AB1E0606820F0100083
:108E30006060B8F1000F01D0042000E0002040F095
:108E40007B0105EB450204F1200000EB421041607C
:108E5000781C05EB450204F1200101EB421108608A
:108E60000CE0B9F1000F07D12946204601F014FEAD
:108E70004FF0FF30BDE8F087A9F1010905EB45018E
:108E800004F1200000EB4110006800F400400028CD
:108E9000E7D105EB450104F1200000EB41104069EA
:108EA00000F4804060B90020306005EB450104F11A
:108EB000200000EB41104069C0F38A00B06014E06C
:108EC0000120306005EB450104F1200000EB41106A
:108ED000016905EB450204F1200000EB42104069F6
:108EE000C0F30C0041EA0040B06005EB450104F11D
:108EF000200000EB4110806900F00F00307305EB9B
:108F0000450104F1200000EB4110C069707305EBCE
:108F1000450104F1200000EB4110C069010AB17362
:108F200005EB450104F1200000EB4110006AF073ED
:108F300005EB450104F1200000EB4110006A010A35
:108F4000317405EB450104F1200000EB4110406A4B
:108F5000707405EB450104F1200000EB4110406AFC
:108F6000010AB17405EB450104F1200000EB41104A
:108F7000806AF07405EB450104F1200000EB41101C
:108F8000806A010A31752946204601F085FD504668
:108F900070E70000000000202DE9F04104460E4675
:108FA00015460127606900F00408206800F0800081
:108FB00040B1B8F1000F05D029462046FFF7E6FD85
:108FC000074606E0F1B22B4601222046FFF710FFCC
:108FD00007463846BDE8F0812DE9F04F8FB0814655
:108FE0000E4678480D90002400200C900B9082468D
:108FF0000025099008904FF47A70079000200690A1
:1090000000BF01200021CDE9040103904846FFF78D
:10901000AAFE01F053FF6C48814502D06B488145A0
:109020000CD16B48006800F00700049001210498FF
:1090300001FA00F0C117CDE904010EE06548814551
:109040000BD163480068C0F302100490012104981A
:1090500001FA00F0C117CDE904015F48DDE90423FE
:1090600000680021FFF772F9074688465B48864290
:1090700000D306465A48864202D940F2EE2B07E05A
:109080005848864202D94FF4487B01E040F26B3BDE
:10909000312554E0012000EB55000A900A9800FBAE
:1090A00006FC6246002338464146FFF74FF905EBC0
:1090B000D5714910A5EB4101029510EB010A00BFE3
:1090C000BAF1000F02D0BAF5806F00D936E00A99E4
:1090D0000AFB01F0C11702460B46CDE900013846F4
:1090E0004146FFF733F90E900E98341A002C00DA3F
:1090F00064420D98844200DD20E00D94A4B905EB94
:10910000D570411008AB09AA5846029505F01FFE1C
:1091100006900698ABEB0004002C00DA6442079836
:10912000844200DD0AE00794284605EBD07149101F
:109130000C91CDF82CA004B903E000BF6D1E062DE4
:10914000A8D200BF08AB09AA58460C9905F0FFFD4C
:1091500006900398042801D90420039008990398E5
:10916000814201D208980390DDE908100844401CB0
:109170000B994843C11702460B46CDE9000138461A
:109180004146FFF7E3F806460898401E0103099898
:10919000401E41EA00210B98401E00F03F000143B1
:1091A000039841EA8010C9F80C000B98401EC0F3E8
:1091B0008310C9F818004846FFF7F2FD30460FB09B
:1091C000BDE8F08F00CA9A3B00000A4000200A4028
:1091D0003402004000100A400000002040420F000E
:1091E00000350C0020A107002DE9FC4706460C467F
:1091F00015461F46DDF828804FF001094FF0000AA0
:1092000008E00AF101008246B0F1805F02D34FF01E
:1092100000090AE00120EAB2E1B23B46CDE9008054
:10922000304600F006F80028EBD000BF4846BDE805
:10923000FC872DE9F05F04460F4690461E46DDE9A7
:109240000A9A4FF0010B204601F0BEFB05460228AA
:1092500002D14FF0000B9DE0F32105EB450204F134
:10926000200000EB42104160B8F1000F15D1002141
:1092700005EB450204F1200000EB42100161C6F34A
:109280000A004FF4004141EA800105EB450204F178
:10929000200000EB4210416112E0B1B205EB450243
:1092A00004F1200000EB42100161C6F30C4040F4D1
:1092B000404105EB450204F1200000EB4210416102
:1092C0001FFA89F105EB450204F1200000EB421082
:1092D00081604FF6FF7000EA194105EB450204F189
:1092E000200000EB4210C1604FF4A05105EB450295
:1092F00004F1200000EB42108161BAF1000F10D0A0
:1093000005EB450104F1200000EB4110806940F0BD
:10931000800105EB450204F1200000EB4210816161
:109320000FE005EB450104F1200000EB41108069DE
:1093300020F0800105EB450204F1200000EB421013
:109340008161002105EB450204F1200000EB421091
:10935000C16105EB450204F1200000EB42100162FF
:1093600005EB450204F1200000EB4210416205EBE1
:10937000450204F1200000EB42108162781C05EBED
:10938000450204F1200101EB421108602946204604
:1093900001F082FB5846BDE8F09F2DE9F0410446FC
:1093A0000F4616464FF00108204601F00DFB05461A
:1093B000022802D14FF000089EE0F32105EB4502A0
:1093C00004F1200000EB421041603068C0B9002178
:1093D00005EB450204F1200000EB421001613089E9
:1093E000C0F30A004FF4005141EA800040F400410C
:1093F00005EB450204F1200000EB4210416114E04E
:10940000308981B205EB450204F1200000EB4210E7
:109410000161B068C0F30C4040F4604105EB4502C7
:1094200004F1200000EB42104161706880B105EB4F
:10943000450104F1200000EB4110406940F4005167
:1094400005EB450204F1200000EB421041610FE002
:1094500005EB450104F1200000EB4110406920F4C8
:10946000005105EB450204F1200000EB4210416180
:10947000717BB07B41EA002105EB450204F120003D
:1094800000EB4210C161F17B307C41EA002105EB29
:10949000450204F1200000EB42100162717CB07CB7
:1094A00041EA002105EB450204F1200000EB4210E7
:1094B0004162F17C307D41EA002105EB450204F177
:1094C000200000EB42108162307B40F4084040F005
:1094D000800105EB450204F1200000EB42108161A0
:1094E000781C05EB450204F1200101EB42110860F4
:1094F0002946204601F0D0FA4046BDE8F0812DE92A
:10950000F04104460F4615460126606900F0040844
:10951000206800F0800058B1B8F1000F08D029464B
:109520002046FFF787FB0646002E0DDA00260BE0EB
:109530002A4639462046FFF730FF08B9002603E0E7
:109540003946204600F004F83046BDE8F0810000BE
:109550002DE9F04104460E464FF001082548076802
:10956000204601F031FA0546022802D14FF00008EA
:109570003DE0606820F0080060600C2105EB4502CA
:1095800004F1200000EB42104160701C05EB450225
:1095900004F1200101EB4211086009E03FB92946BE
:1095A000204601F079FA4FF0FF30BDE8F0817F1ED0
:1095B00005EB450104F1200000EB4110006800F4C8
:1095C00000400028EAD1842105EB450204F1200087
:1095D00000EB42104160701C05EB450204F12001D4
:1095E00001EB421108602946204601F055FA404639
:1095F000DBE70000000000200448006840F48030F1
:109600004FF08041C1F84002704700004002004026
:1096100070B5294D2D68EDB2012D42D100F0407496
:1096200000F0406100F0405200F0404354B1224D40
:109630009C352D6825F0407505434FF08046C6F8EF
:10964000905238E051B11C4D9C352D6825F0406595
:1096500005434FF08046C6F890522CE052B1164DAB
:109660009C352D6825F0405505434FF08046C6F8DF
:10967000905220E053B1104D9C352D6825F04045A7
:1096800005434FF08046C6F8905214E00A4D9C35D1
:109690002D6825F4403505434FF08046C6F89052BA
:1096A00009E0054D9C352D6825F4403505434FF004
:1096B0008046C6F8905270BDF401004010B50022FB
:1096C000002100F01F04012303FA04F204490323DC
:1096D00003EA907301EB83010B6813430B6010BD29
:1096E000040200402DE9F34F87B00C46FFF784FFDA
:1096F000079880B95948006840F001004FF0804158
:10970000C1F80002012000F0CBFA00200690DFF83B
:109710005091022610E05148006840F004004FF0DC
:109720008041C1F80002102000F0BAFA4FF4002086
:109730000690DFF82C9104264A48844277D84A489C
:10974000844274D34FF0FF380020029003900190C0
:10975000009401254BE0B8F1000F00D149E0032D42
:1097600044D0042D02D10098840003E0022D01D1E1
:1097700000984400022636E0B8F1000F00D134E032
:10978000B9FBF6FB394883452CD34000834529D8E3
:109790004FF0020A21E0CBF35D0000FB0AF73248EC
:1097A000874218D33248874215D8B7EB940F02D9B5
:1097B000A7EB940001E0C7EB9400049004984045A7
:1097C00009D2DDF810800296CDF80CA00195B8F111
:1097D000000F00D105E00AF1010A40F201208245A4
:1097E000D9D900BF761C202EC6D900BF6D1C042D10
:1097F000B1D900BF0198401E069941EA8031029814
:10980000401E41EA40210398801E01431348403026
:109810000160042000F044FADDE901014843B9FB8E
:10982000F0F0039948434000059012E0FFE70798E5
:1098300028B944F21E2009494031086003E00D4870
:10984000064940310860042000F02AFA00F094F83C
:109850000590059809B0BDE8F08F000000020040B7
:10986000001BB7000065CD1D80F0FA0200093D0025
:10987000405973071E42080010B501F01FFB014854
:10988000006810BD0000002010B501F017FB1A4859
:10989000006800F0070010B91848046829E016486D
:1098A000006800F00700012803D11448006844084C
:1098B0001FE01148006800F00700022803D10F489C
:1098C0000068840815E00C48006800F007000328D1
:1098D00003D10A480068C4080BE00748006800F09C
:1098E0000700042803D105480068040901E0034883
:1098F0000468204610BD0000340200400000002033
:1099000010B501F0DBFA1A48006800F0700010B9D9
:109910001848046829E01648006800F07000102814
:1099200003D11448006844081FE01148006800F0A3
:109930007000202803D10F480068840815E00C4807
:10994000006800F07000302803D10A480068C4089D
:109950000BE00748006800F07000402803D105487C
:109960000068040901E003480468204610BD0000B7
:109970003402004000000020F8B5002018A6366828
:109980000096184E316801F4A02606B127E001F4D4
:109990000036B6F5003F09D101F40026B6F5002FD8
:1099A00001D1114A00E0104A104618E001F40026E7
:1099B000B6F5002F01D10C4A00E00B4AC1F3813704
:1099C0001DF80740C1F30806B31CC1F34426751CFB
:1099D00096085E4315FB04F7B6FBF7F6F000F8BDFA
:1099E0000102020440020040001BB7000D49096853
:1099F00041F004010B4A11600B49096841F08001F4
:109A00009206C2F80012094908681146D1F8F01010
:109A100021F00301C2F8F01030BF1146C1F8F00088
:109A20007047000010ED00E000020040F000004030
:109A300070B504462548006800F0100524488442AB
:109A400000D9044621485038006840F004004FF027
:109A50008041C1F80002102000F022F94FF0804050
:109A6000D0F8100240F007004FF08041C1F810021A
:109A70000846D0F8200220F00F00C1F82002134859
:109A80005038006800F0010028B121460020FFF79F
:109A900029FE044609E021464FF40020FFF722FE8C
:109AA00004460A48006800F010050021022000F07A
:109AB00011F845B905485038006820F004004FF00F
:109AC0008041C1F80002204670BD000050020040F5
:109AD00000B0710B70B504460D461C48006800F0DC
:109AE00010064FF08040D0F8000240F00400174903
:109AF00050390860102000F0D3F81448403800684E
:109B000020F00700C01D4FF08041C1F810020F483F
:109B10003038006820F00F002843C1F820020B48BD
:109B20004038006820F007002043084940390860A9
:109B300001F0C4F946B905485038006820F0040027
:109B40004FF08041C1F8000270BD0000500200409B
:109B5000F0B500230024C0F38725002D4CD0304DF4
:109B60002D68EDB2012D2AD1C0F38145022D06D119
:109B700000F01F051F2D02D1294C343433E0C0F30F
:109B80008145022D06D100F01F051D2D02D1244C68
:109B9000343428E0C0F38145022D02D1204C383402
:109BA00021E0C0F38145032D02D11D4C3C341AE065
:109BB000C0F381451A4E2C3606EB850413E0C0F342
:109BC0008145022D02D1164C38340CE0C0F381459A
:109BD000032D02D1124C3C3405E0C0F38145104EF8
:109BE0002C3606EB85042568C0F38726C0F344179E
:109BF000BE40B54315432560C0F3426575B1C0F35F
:109C00000175074E1C3606EB85031D68C0F34266DE
:109C1000C0F30457BE40B5430D431D60F0BD0000C6
:109C2000F401004010B504461C480068C0B2012889
:109C300019D1042C0BD100BF18489C30006820F0CB
:109C4000700040F010002107C1F890021BE0052CC5
:109C500019D1042411489C30006820F070002107BD
:109C6000C1F890020FE0042C01D0052C0BD10B4859
:109C70000C30006840F008004FF08041C1F800024D
:109C8000082000F00DF805489C30006820F007001F
:109C900020434FF08041C1F8900210BDF401004014
:109CA00010B501460C4B1B685A08012000230B4CD1
:109CB000236004E0531E1A1E01D1002004E0084B6B
:109CC0001B680B408B42F5D100BF1AB94FF0FF3330
:109CD000024C236010BD0000000000203400002072
:109CE0005002004030B500F1800454F82140084D86
:109CF0002C4000F1800545F821402C4654F82140C5
:109D000042EA03052C4300F1800545F8214030BDAF
:109D1000C0FFE0FF10B50F4B1A6800230E4C236004
:109D2000036D23F480730365036D41F00104234345
:109D3000036506E0531E1A1E03D1531E064C236012
:109D400005E0D0F8103103F00103002BF2D000BF82
:109D500010BD00000000002038000020034800680B
:109D600020F00100014908607047000000C0004079
:109D700010B5034600201D490860B3F5001F02D14D
:109D800000F03AF810BD22201949C8600846436027
:109D900001200861174800680A21B0FBF1F0840037
:109DA00000BF201EA4F1010406DD1148C030006888
:109DB00000F001000028F4D1002C04DC4FF0FF304B
:109DC0000A490860DEE70A48006800F0400050B128
:109DD0000748006840F04000054908604FF0FF3038
:109DE00002490860CEE70020CCE700003C000020DC
:109DF00000C000400000002000201B4A106022200C
:109E00001A4AD0604FF40010506019489060012049
:109E10001061184800680A22B0FBF2F0810000BF10
:109E2000081EA1F1010106DD1048C030006800F0F5
:109E300001000028F4D1002904DC4FF0FF300A4A69
:109E4000106070470948006800F0400050B10748B2
:109E5000006840F04000054A10604FF0FF30024AB1
:109E60001060EEE70020ECE73C00002000C000405E
:109E700003AA5500000000200348006840F00100DC
:109E8000014908607047000000C000400146002002
:109E9000114B1860114BD8601846416001201861C1
:109EA0000F4800680A23B0FBF3F0420000BF101E09
:109EB000A2F1010206DD0948C030006800F001008F
:109EC0000028F4D1002A04DC4FF0FF30024B186068
:109ED000704702488068FBE73C00002000C000405B
:109EE0000000002010B5024600201A4C20602120FE
:109EF000194CE060204642608160012020611748D3
:109F000000680A24B0FBF4F0430000BF181EA3F160
:109F1000010306DD1048C030006800F00100002891
:109F2000F4D1002B04DC4FF0FF300A4C206010BD50
:109F30000948006C00F0400050B10748006C40F048
:109F40004000054C20644FF0FF30024C2060EEE7EB
:109F50000020ECE73C00002000C000400000002092
:109F600008B54FF04020006E00F0010038B101202C
:109F70004FF04021086606201449087024E04FF095
:109F80004020006E00F0040038B104204FF0402162
:109F9000086602200D49087016E04FF04020006E60
:109FA00000F4805040B14FF480504FF040210866DB
:109FB00003200649087007E04FF04020006E009033
:109FC0004FF040210098086608BD00000C010020F9
:109FD00008B51148006800F0010030B101200E49B9
:109FE000086004200D49087014E00B48006800F474
:109FF000804038B14FF4804007490860012008498B
:10A00000086007E00448006800904FF04021009885
:10A01000C1F8A00008BD0000A04000400C010020D5
:10A020007800002008B50A48006800F0400030B110
:10A0300040200749086005200649087007E00448E9
:10A04000006800904FF040210098C1F8600108BD01
:10A05000604100400C01002008B50B48006800F486
:10A06000806038B14FF480600749086006200749D6
:10A07000087007E00448006800904FF04021009805
:10A08000C1F8E00108BD0000E04100400C010020E3
:10A0900010B5836901248C40A343140E8C402343E4
:10A0A0008361C3694FF001148C40A34322F07F44C5
:10A0B0008C402343C36110BD70B50346002011E0FE
:10A0C000012484400C4001258540AC4209D11C6824
:10A0D00046000325B540AC43450002FA05F52C4384
:10A0E0001C60401C1028EBD370BD70B503460020E7
:10A0F0000EE0012484400C404CB11C6B460003254B
:10A10000B540AC43450002FA05F52C431C63401CE6
:10A110001028EED370BD70B5034600200EE0012478
:10A1200084400C404CB19C6A46000325B540AC43CA
:10A13000450002FA05F52C439C62401C1028EED322
:10A1400070BD0000044604A001F0EEF9204628F09E
:10A1500079FC00BFFEE70000496E20486172642070
:10A160004661756C742048616E646C65720A00000B
:10A1700038B504460D46022C00DB38BD2946204682
:10A180000CF08CFC04EBC40101EB0411104B03EB4D
:10A19000811204EB44010F4B03EB8100642120F09A
:10A1A000CDFA002040F2FF730246052100902046C0
:10A1B0000CF0B0FD0020084B012206210090204643
:10A1C0000CF0A8FD054920460CF09AFD00BFD4E72D
:10A1D000103E0020904A00200201F018E1A6020083
:10A1E00030B504460D46022C01DB002030BD04EBE7
:10A1F00044000A4901EB800393E8070020F0A5FA28
:10A2000048B904EB4401054A02EB8100294620F0DD
:10A21000AFFA0120EAE70020E8E70000904A0020BA
:10A220000FB438B50446022C02DB38BC5DF814FBD1
:10A2300008980090204605A90EC90CF00FFD00BF3C
:10A24000F3E7000010B5034A012108460CF002FFB5
:10A2500010BD0000E5A3000030B503460C46002108
:10A26000062B01DB002030BD00210BE003EB430097
:10A2700000EB83200A4D05EB4000001D405C60545C
:10A28000481C81B2914202DAB1F5006FEEDB03EBBC
:10A29000430000EB8320024D05EB40004088E2E7DD
:10A2A000BC0100200146062901DB0020704701EBBC
:10A2B000410000EB8120024A02EB40004088F5E7B4
:10A2C000BC01002070B504460D46062C00DB70BDB5
:10A2D00004EB440101EB84210A4A12F811002946DB
:10A2E0000DF088FB04EB440101EB8421054A12F8D0
:10A2F000110005490DF072FD204600F053F800BF33
:10A30000E5E70000BC0100205DA40000014606292D
:10A3100001DB0020704701EB410000EB8120054A82
:10A3200002EB40004078022801D10120F2E7002032
:10A33000F0E70000BC01002010B50446062C00DB4D
:10A3400010BD34B1012C0AD0022C0ED0032C0ED13A
:10A350000CE04FF4806107480CF031FE07E04FF449
:10A36000007104480CF02BFE01E000E000BF00BFCC
:10A3700000BFE5E78040004070B504460D46164634
:10A38000062C00DB70BD04EB440101EB8421044A80
:10A3900012F81100324629460DF0B2FC00BFF1E779
:10A3A000BC010020062800DB7047002100EB4002C2
:10A3B00002EB80220A4B03EB4202517000EB400299
:10A3C00002EB802203EB4202518000EB400202EBE1
:10A3D000802203EB4202A2F8041800BFE4E7000069
:10A3E000BC01002010B50146002000BF30E000EBAA
:10A3F000400202EB8022184B03EB42025278012A02
:10A4000024D100EB400202EB802203EB4202B2F8BF
:10A410000428521C00EB400303EB80230E4C04EB9A
:10A420004303A3F8042800EB400202EB80222346FA
:10A4300003EB4202B2F804281E2A07DB022200EBDB
:10A44000400303EB802304EB43035A70421CD0B259
:10A450000628CCDB10BD0000BC01002070B5024610
:10A460000B4600210020082A00DB70BD00210CE013
:10A4700001EB410404EB8124424D15F81440944251
:10A4800001D1084603E04C1CE1B20629F0DB00BF15
:10A4900000EB400404EB80243A4D05EB440464785F
:10A4A00084BB002400EB400505EB8025354E06EB10
:10A4B00045056C8000EB400505EB802506EB450566
:10A4C000A5F8044800EB400404EB8024354605EB76
:10A4D0004404237100EB400404EB802405EB4404A6
:10A4E0006488641C00EB400505EB802506EB450500
:10A4F0006C80012400EB400505EB802506EB45054B
:10A500006C703DE0FFE700EB400404EB80241D4D40
:10A5100005EB44046478012C32D100EB400404EBD9
:10A52000802405EB44046488B4F5006F28DA00EB5E
:10A53000400404EB802405EB4404241D00EB40059B
:10A5400005EB80250F4E06EB45056D88635500EB46
:10A55000400404EB8024354605EB44046488641C05
:10A5600000EB400505EB802506EB45056C800024DB
:10A5700000EB400505EB802506EB4505A5F80448F2
:10A5800000BF72E7BC01002010B5002400BF1CE032
:10A5900004EB44001B4911F82000012813D104EBFF
:10A5A000440001EB8000406868B104EB44020B46B4
:10A5B00003EB8202916804EB440203EB82025068D1
:10A5C00000220CF0D3FC601CC4B20D2CE0DB0E4862
:10A5D000006820F440104FF04021C1F8F001084617
:10A5E000D0F8F00140F48010C1F8F0010846006F87
:10A5F00020F0030008670846006F40F0010008677C
:10A6000010BD000018010020F041004010B50024EA
:10A61000802115480CF0CBFC08B944F0010440211E
:10A6200011480CF0C4FC08B944F0020420210E4883
:10A630000CF0BDFC08B944F0040410210A480CF0E9
:10A64000B6FC08B944F00804082107480CF0AFFC38
:10A6500008B944F01004042103480CF0A8FC08B920
:10A6600044F02004204610BD0041004070B504466F
:10A6700000250D2C01DB012070BD04EB44020C4BC6
:10A6800003EB8202916804EB440203EB8202506800
:10A690000CF08DFC054604EB4400054901EB8000FD
:10A6A0004078A84201D10020E6E70120E4E700005D
:10A6B0001801002010B5044604EB4400154901EBD5
:10A6C00080008078012812D104EB44020B4603EB92
:10A6D0008202916804EB440203EB820250680CF0A2
:10A6E0005EFC012801D1002010BD0120FCE704EB35
:10A6F0004402084B03EB8202916804EB440203EB33
:10A70000820250680CF04BFC012800D1ECE70020DD
:10A71000EAE70000407B030010B5002400BF3FE0E3
:10A7200004EB4400204911F82000012836D104EB45
:10A73000440001EB8000406810B304EB44020B4678
:10A7400003EB8202916804EB440203EB820250683F
:10A7500001220CF00BFC04EB4400134901EB8000D8
:10A76000407801280DD104EB44020B4603EB820232
:10A77000916804EB440203EB820250680CF023FC66
:10A780000CE004EB4402084B03EB8202916804EBFB
:10A79000440203EB820250680CF011FC601CC4B24E
:10A7A0001D2CBDDB10BD0000407B030070B50446CE
:10A7B0000D461D2C00DB70BD04EB44001A4901EB73
:10A7C0008000406800B9F6E704EB4400164901EB4D
:10A7D00080008078012800D145B104EB4400124983
:10A7E00001EB8000807878B9012D0DD104EB440293
:10A7F0000D4B03EB8202916804EB440203EB8202EF
:10A8000050680CF0E0FB0CE004EB4402064B03EB59
:10A810008202916804EB440203EB820250680CF060
:10A82000CEFB00BFC7E70000407B030010B501204E
:10A830002CF0FAF90349086001200CF095FC08F0AF
:10A8400000FE10BDB40100202DE9F04104460D4684
:10A850001646002764210A4800682CF08BFC32461B
:10A860002946204608F0F3FD074600231A461946FC
:10A87000034800682CF062FA3846BDE8F081000019
:10A88000B40100202DE9F04104460D46164600278C
:10A8900064210A4800682CF06DFC324629462046A7
:10A8A00008F02FFE074600231A46194603480068A1
:10A8B0002CF044FA3846BDE8F0810000B4010020D5
:10A8C00013B501202CF0B0F903490860DDE900015F
:10A8D00008F052FF1CBD0000B801002070B504460E
:10A8E00000256421084800682CF044FC204608F04C
:10A8F0007DFF054600231A461946034800682CF0E0
:10A900001DFA284670BD0000B801002013B564216F
:10A91000084800682CF02EFCDDE9000109F056F82B
:10A9200000231A461946034800682CF007FA012054
:10A930001CBD0000B801002010B50DF05BFA10BD81
:10A9400030B501461C4CA14201D1002208E01B4C4D
:10A95000A14201D1012203E0194CA14200D10222FF
:10A9600002200C6804F00E030C6824F00E040C6046
:10A970000C6A04F4004444B9124C14F8124024B98F
:10A980000124104D05F81240002002280FD1802428
:10A99000645804F4004454B90A4C04EB420464784B
:10A9A0002CB90124074D05EB42056C7001200C68A1
:10A9B0001C430C6030BD000000000A4000100A403B
:10A9C00000200A402C00002070B50646002407E055
:10A9D0003046FFF7B5FF0546022800D003E0641CAF
:10A9E000B4F1805FF4D300BF284670BD00F01F02B1
:10A9F000012191404209920002F1E022C2F80011C7
:10AA0000704700F01F02012191404209920002F1BB
:10AA1000E022C2F80011704700F01F0201219140AE
:10AA20004209920002F1E022C2F8001170470000D2
:10AA300010B5002807DA0A07140E054A00F00F03C4
:10AA40001B1FD45403E00A07130E024A135410BD0F
:10AA500018ED00E000E400E000BF00BF00BFBFF35E
:10AA60004F8F00BF00BF00BF0948006800F4E060DE
:10AA700008490843001D0649086000BF00BF00BF29
:10AA8000BFF34F8F00BF00BF00BF00BF00BFFDE797
:10AA90000CED00E00000FA0530B50A46022A1CD28F
:10AAA0000E4CA04201D1002108E00D4CA04201D182
:10AAB000012103E00B4CA04200D10221046804F004
:10AAC0000E03046824F00E0404600024064D05EB18
:10AAD0004105AC5404681C43046030BD00000A40CA
:10AAE00000100A4000200A402C000020016941F4B7
:10AAF000807101617047816821F0090181607047B0
:10AB00002DE9F84F04460F46934698460A9E0025C5
:10AB100000200090206E20F001002066B8F1200F88
:10AB200000D1A846FEF7A8FE8246002F70D1002073
:10AB3000A06047EA082040EA0B0040F001002060D6
:10AB4000564531D39B48844209D19B48006820F088
:10AB5000300040F02000A104C1F8180224E097481A
:10AB6000844209D19448006820F0C00040F0800081
:10AB70006104C1F8180217E0914884420AD18E4856
:10AB8000006820F4406040F400604FF08041C1F85C
:10AB9000180209E08848006820F4405040F4005052
:10ABA0004FF08041C1F81802824884421CD182488B
:10ABB000006800F0300008B9824D76E07E480068F9
:10ABC00000F03000102803D1FEF7D6FE05466CE0F9
:10ABD0007948006800F03000202803D1FEF790FE8D
:10ABE000054662E0774D60E0744884421DD17248AA
:10ABF000006800F0C00008B9724D56E06E48006869
:10AC000000F0C000402804D1FEF7B6FE05464CE037
:10AC100084E06948006800F0C000802803D1FEF796
:10AC200033FE054641E0674D3FE0654884421ED152
:10AC30006148006800F4406008B9624D35E05E4844
:10AC4000006800F44060B0F5806F03D1FEF794FE19
:10AC500005462AE05848006800F44060B0F5006FEF
:10AC600003D1FEF74DFE05461FE0564D1DE052484C
:10AC7000006800F4405008B9524D16E04E48006894
:10AC800000F44050B0F5805F03D1FEF775FE054635
:10AC90000BE04948006800F44050B0F5005F03D174
:10ACA000FEF7F2FD054600E0464D564503D3002071
:10ACB000606000957BE0AE4203D3002060600095A9
:10ACC00075E03EB9606840F2FF1108436060280AF1
:10ACD00000906CE005EB85004000B0FBF6F0401DF5
:10ACE0000A21B0FBF1F0A0F10109B9F1FF0F09D978
:10ACF0004FF0FF09606840F2FF1108436060280AC6
:10AD0000009054E060686FF3080040EA090060605A
:10AD100009F10100B5FBF0F0009048E00020A060D0
:10AD200047EA082040EA0B0040F0010020600020C4
:10AD30006060204884420CD11F48006820F0300039
:10AD400040F02000A104C1F81802FEF7D9FD0090E0
:10AD50002DE01A4884420CD11748006820F0C0004A
:10AD600040F080006104C1F81802FEF78DFD0090EC
:10AD70001DE0134884420DD10F48006820F4406064
:10AD800040F400604FF08041C1F81802FEF7B8FDB2
:10AD900000900CE00848006820F4405040F4005057
:10ADA0004FF08041C1F81802FEF76EFD0090009848
:10ADB000BDE8F88F00100640180200400020064051
:10ADC00000300640001BB7000020014908607047B2
:10ADD0000001004000BF592007490860162089057E
:10ADE000C1F800018820C1F80001C006D0F80001B8
:10ADF0000028F0D0704700000001004000BF59203B
:10AE00000749086016208905C1F800018820C1F8AB
:10AE10000001C006D0F800010028F0D07047000003
:10AE20000001004000BF592007490860162089052D
:10AE3000C1F800018820C1F80001C006D0F8000167
:10AE40000028F0D0704700000001004010B5044613
:10AE5000204600F001F810BD00BF0A49896901F4DD
:10AE600000010029F9D10A2809D10D21054A1160F4
:10AE700000BF0449896901F400010029F9D10149A1
:10AE8000086070470000074010B500BF502080F3F5
:10AE90001188BFF34F8FBFF36F8F00BF2CF0D2FA32
:10AEA00018B14FF080500449086000BF002080F3C3
:10AEB000118800BF10BD000004ED00E070B5FEF782
:10AEC0005BFD114908601148006800F00705022D7C
:10AED00002D10846046802E00D4850F825400B48AE
:10AEE0001030006800F00F00461CB4FBF6F0094972
:10AEF000086008460068084908444900B0FBF1F0C2
:10AF00000649086070BD00000800002010020040E3
:10AF10000C0000200000002020A1070004000020F9
:10AF20002048006840F470001E4908601E48C06C4C
:10AF300020F00F0040F008001B49C8641B4800685F
:10AF400040F480204FF08041C1F898020846D0F8C4
:10AF5000080240F00200C1F808021548D0F80401C8
:10AF600000F0F7301249C1F804010846D0F8080192
:10AF700000F0F730C1F808018804D0F8080220F08A
:10AF800002000A499039086000BF4FF04020D0F815
:10AF9000400120F0F0004FF04021C1F8400100BF17
:10AFA0007047000088ED00E000C0004098020040BB
:10AFB00000100440012181607047000070B588B026
:10AFC000044620221A496846FDF700FA19488442CF
:10AFD00004D119480068C0F3022513E017488442E1
:10AFE00004D115480068C0F302350BE014488442D0
:10AFF00004D111480068C0F3024503E00E48006820
:10B00000C0F30255022D0DD10A48844202D00B48EC
:10B01000844203D1FEF738FC064605E0FEF770FCDB
:10B02000064601E05DF82560304608B070BD0000BE
:10B03000A87A03000000054014020040000105400A
:10B04000001005402DE9F047064689461746304670
:10B05000FFF7B4FF804600240025B7EB580F01D955
:10B06000022406E0B8FBF7F4250E15B1681CB4FB0A
:10B07000F0F449EA050030607460681C6043B8FB76
:10B08000F0F0BDE8F087016841F080410160704751
:10B0900010B50BF0A7FF0248FFF78CFF10BD0000B2
:10B0A0000000054010B50BF0ABFF0248FFF782FF30
:10B0B00010BD00000001054010B50BF0AFFF0248C5
:10B0C000FFF778FF10BD00000010054010B50BF031
:10B0D000B3FF0248FFF76EFF10BD000000110540EE
:10B0E00010B50A48C46904F4807010B904F48050A3
:10B0F00058B104E005490968C8B20CF00BFC0348DC
:10B10000806900F480400028F4D010BD00000740A2
:10B1100010B50A48C46904F4807010B904F4805072
:10B1200058B104E005490968C8B20CF001FC0348B5
:10B13000806900F480400028F4D010BD0010074062
:10B1400010B50A48C46904F4807010B904F4805042
:10B1500058B104E005490968C8B20CF0F7FB034890
:10B16000806900F480400028F4D010BD0020074022
:10B1700010B50A48C46904F4807010B904F4805012
:10B1800058B104E005490968C8B20CF0EDFB03486A
:10B19000806900F480400028F4D010BD00300740E2
:10B1A00010B50A48C46904F4807010B904F48050E2
:10B1B00058B104E005490968C8B20CF0E3FB034844
:10B1C000806900F480400028F4D010BD00400740A2
:10B1D00010B50A48C46904F4807010B904F48050B2
:10B1E00058B104E005490968C8B20CF0D9FB03481E
:10B1F000806900F480400028F4D010BD0050074062
:10B2000010B50A48C46904F4807010B904F4805081
:10B2100058B104E005490968C8B20CF0CFFB0348F7
:10B22000806900F480400028F4D010BD0060074021
:10B2300010B50A48C46904F4807010B904F4805051
:10B2400058B104E005490968C8B20CF0C5FB0348D1
:10B25000806900F480400028F4D010BD00700740E1
:10B2600042680A43426070472DE9FF4104460D469B
:10B270000026B046584B0FCB8DE80F0000275748EB
:10B2800084420AD156480068C0F301664FF08040FE
:10B29000D0F82002C0F303286DE05248844209D15F
:10B2A0004F480068C0F38166A004D0F82002C0F3C4
:10B2B000033860E04C4884420AD1494808300068AD
:10B2C000C0F301666004D0F8300200F00F0852E0CD
:10B2D000464884420BD1424808300068C0F381667A
:10B2E0004FF08040D0F83002C0F3031843E04048EC
:10B2F00084420AD13A4808300068C0F3017620043D
:10B30000D0F83002C0F3032835E03A48844209D12E
:10B31000334808300068860FA004D0F83002C0F32C
:10B32000033828E03448844211D12D482038006881
:10B33000C0B201280BD12A4808300068C0F301567A
:10B340004FF08040D0F83002C0F3034813E02B48A0
:10B35000844210D1224820380068C0B201280AD1A6
:10B360001F4808300068C0F381564FF08040D0F885
:10B370003002C0F30358002020630320E060A0687F
:10B380001F490840A060012E03D1FEF7F5FA4DF8E1
:10B390002600FDB15DF8261008F10100B1FBF0F0C8
:10B3A00000EB5500B0FBF5F0871EB7F5803F0ED3DC
:10B3B0005DF8261008F10100B1FBF0F000EBC500CC
:10B3C000B0FBF5F00221C1EB1010606202E047F023
:10B3D00040506062BDE8FF81C87A0300000007406A
:10B3E00014020040001007400020074000300740D2
:10B3F00000400740005007400060074000700740D1
:10B400000FFFF0FF70B503460025002013E0002475
:10B4100005E0641CB4F1804F01D3012504E09E696E
:10B4200006F40006002EF4D100BF012D00D104E087
:10B430000E5C1E60401C9042E9D100BF70BD000050
:10B440002DE9F04105460E460024002700BF2DE0FF
:10B4500004EB4400184901EB80008088284404EB89
:10B460004401154A02EB8101888004EB4400114637
:10B4700001EB8000808804EB440102EB81014988E4
:10B48000884211DB002004EB440102EB810188803B
:10B490003A467B1CDFB206EB021004EB4402064B7B
:10B4A00003EB820291688847601CC4B2062CCFD39C
:10B4B0003846BDE8F0810000E837002011480068F8
:10B4C000C0F3C00038B10F48006820F0240040F0FD
:10B4D00008000C4908600B480068C0F3401080B1B8
:10B4E0000848006820F00C0040F020000549086082
:10B4F00045F6A52088600448007810B9012002496B
:10B5000008707047000004400C01002030B5054C65
:10B51000616040F0800444EA420444EA0314014DAF
:10B520002C6030BD000004400FB4054B10B503A9DA
:10B53000044A029800F018F810BC5DF814FB0000F3
:10B54000ED8601004000002002E008C8121F08C17B
:10B55000002AFAD170477047002001E001C1121F94
:10B56000002AFBD1704700002DE9FF4F8DB09B46AC
:10B570000F460446002606E025280BD05A460F99B0
:10B580009047641C761C20780028F5D111B0304615
:10B59000BDE8F08F0025A8460122984900E0054348
:10B5A00014F8013F203B02FA03F00842F7D120785B
:10B5B0002E2817D114F8010F45F004052A280ED0C3
:10B5C0006FF02F022078A0F1300109290AD808EB8A
:10B5D000880102EB410100EB0108641CF2E757F817
:10B5E000048B641C20786C280DD004DC4C2812D00D
:10B5F0006A2811D104E074280DD07A280CD10AE011
:10B6000045F4001507E0617845F48015814202D1C8
:10B61000641C05F58015641C2278692A45D008DC75
:10B62000002AB3D0582A69D0632A10D0642A08D1DE
:10B630003BE0702A67D0732A13D0752A5CD0782A31
:10B640005CD010465A460F999047761CD3E017F805
:10B65000040B8DF8000000208DF80100E946012060
:10B6600003E057F8049B4FF0FF3069074FF00005E7
:10B6700001D40AE06D1C45450DDA8542FADB19F864
:10B6800005100029F6D106E06D1C8542FCDB19F897
:10B6900005100029F8D12E4404E019F8010B5A4690
:10B6A0000F9990476D1EF8D2A5E00A200021CDE940
:10B6B0000801C5F3025002280DD001CFC117031EA7
:10B6C00071F100030DDA4FF0000CD0EB0C006CEBC5
:10B6D00001012D2308E0FF1D27F00707F7E802010D
:10B6E000EDE72B0504D52B238DF8283001233BE013
:10B6F000EB0739D02023F7E70A2000E010200021D3
:10B70000CDE9080107E01020002145F00405CDE94E
:10B7100008014FF00808C5F3025002280FD001CFEE
:10B7200000214FF0000A2B071FD5702A0DD0DDE94C
:10B7300008C38CF0100C5CEA030C0CD015E0FF1D64
:10B7400027F00707F7E80201EBE740228DF82820F1
:10B750004FF0010A0BE050EA010306D030238DF8C8
:10B7600028308DF8292002239A46582A04D024A292
:10B770000DF120090B9209E026A2F9E7DDE9082383
:10B78000FCF7E4FD0B9B9B5C09F8013D50EA0102CC
:10B79000F4D1ADEB090020300890680701D44FF0D8
:10B7A00001080899884502DDA8EB010000E00020AF
:10B7B0008046002506E00AA85A46405D0F9990474A
:10B7C0006D1C761C5545F6DB04E030205A460F9977
:10B7D0009047761CB8F10001A8F10108F5DC05E0FE
:10B7E00019F8010B5A460F999047761C0899481E84
:10B7F00008900029F4DC641CC5E60000092801005B
:10B8000030313233343536373839616263646566D6
:10B810000000000030313233343536373839414298
:10B8200043444546000000002DE9F04105460E4620
:10B830000024002700BF2DE004EB4400184901EB71
:10B8400080008088284404EB4401154A02EB810102
:10B85000888004EB4400114601EB8000808804EBF3
:10B86000440102EB81014988884211DB002004EB8E
:10B87000440102EB810188803A467B1CDFB206EB73
:10B88000021004EB4402064B03EB820291688847E6
:10B89000601CC4B20A2CCFD33846BDE8F08100004A
:10B8A000F038002010B5034619785A78002039295D
:10B8B00003DDA1F13704E1B202E0A1F13004E1B20D
:10B8C00001F00F01392A03DDA2F13704E2B202E0F0
:10B8D000A2F13004E2B202F00F0202EB0114E0B276
:10B8E00010BD30B5044600252046FFF7DBFF0502FA
:10B8F000A01CFFF7D7FF0543284630BD014601F0E5
:10B900000F000A1102EB820200EB4200C0B2704746
:10B91000014601F00F000A1102EB820200EB420027
:10B92000C0B2704710B50B48406888B10BF0B8FA48
:10B9300000200849486047F20101481E0BF07EFADA
:10B94000802204494FF4E0400BF0DCFA0BF066FA79
:10B9500010BD00004064002010B50BF0A1FA802259
:10B960001C494FF4E0400BF0ABFA04221A494FF4A3
:10B97000F0400BF0A5FA0020184A12680A23B2FB27
:10B98000F3F251000022164B1A600422154BDA60C4
:10B9900082005A6000229A6001221A6107E0114A6F
:10B9A000126902F0010212B90E4A926807E00A1EFB
:10B9B000A1F10101F3D1521E094B1A6000BF0A48E0
:10B9C00002600548006800F065F8074908600BF060
:10B9D00025FA10BD406400202C3200200000002019
:10B9E0003C00002000C000403032002010B504466A
:10B9F0000BF056FA802214494FF4E0400BF060FA45
:10BA0000114844604FF496400F49C8604FF4E1304C
:10BA100008614FF41640486188614FF4E130C86115
:10BA20004FF41640086200200863486347F20101A2
:10BA3000481E0BF003FA802203494FF4E0400BF05C
:10BA400061FA0BF0EBF910BD40640020014620299B
:10BA500001DB00207047024850F82100FAE700009F
:10BA60004064002010B500220023020900F00F03FB
:10BA7000092A02DC02F1300401E002F137040C7003
:10BA8000092B02DC03F1300401E003F137044C70B0
:10BA900010BD000001460248084448400146704776
:10BAA0004D3C2B1A10B50246002003E012F8014B62
:10BAB000231898B20B1EA1F10104A1B2F6D1C34321
:10BAC00098B2431C98B210BD10B5044601202070F6
:10BAD00060700820A07009486060D32029F032FC13
:10BAE0002081D12029F02EFC6081D42029F02AFC6D
:10BAF000A081D22029F026FCE08110BD00010300C6
:10BB000010B504460120207060700820A0700C4819
:10BB1000606000202081002161811AF02FFA10B9A5
:10BB20000121A18101E00021A18101201AF026FA62
:10BB300010B90121E18101E00021E18110BD000087
:10BB40000002030070B52DED068B04460025012090
:10BB5000207060700820A0704FF441306060C820F1
:10BB600029F0F0FB0646FCF7FEFD41EC190B9FEDBA
:10BB7000220B53EC102BFCF704FD41EC180BFCF7E7
:10BB80001EFE2081CA2029F0DDFB0646C92029F0CF
:10BB9000D9FB06EB00452846FCF7D4FD41EC190B18
:10BBA0009FED150B53EC102BFCF7EBFC41EC180B45
:10BBB000FCF705FE6081F62029F0C4FB0646FCF781
:10BBC000D2FD41EC1A0B9FED0C0B53EC102BFCF744
:10BBD000D8FC41EC190B9FED0A0B53EC102BFCF732
:10BBE000CAFC41EC180BFCF7EAFDA08115F018FA2D
:10BBF000E081BDEC068B70BD9A9999999999B93FEE
:10BC00009A9999999911714070B5044600250120BF
:10BC1000207060700820A0700E486060E12029F05C
:10BC200091FBC5B2642D00DD6425D02029F08AFB8C
:10BC300020816581D02029F085FB00EBC00101EB5C
:10BC400000104FF6FF7101EA8001A1810021E1811E
:10BC500070BD00000005030010B5044601202070EF
:10BC600060700820A0700848606002201AF086F911
:10BC7000012801D1208101E0002020810021618183
:10BC8000A181E18110BD00000007030001210170C6
:10BC900000214170082181704FF4A8714160012199
:10BCA0000181002242818281C281704710B5044621
:10BCB00001202070002060700820A07040F2511018
:10BCC00060600D20207202216172492029F03AFB48
:10BCD00060813F201CF0BCF8A0813F201CF0B8F828
:10BCE0004FF6FF7101EA4011E18110BD10B5044625
:10BCF00001202070002060700820A0704FF4C070F8
:10BD00006060D32029F01EFB2081D42029F01AFB8B
:10BD10006081D12029F016FBA081D22029F012FBEE
:10BD2000E08110BD70B52DED048B04460026002582
:10BD300001202070002060700820A07040F2811067
:10BD400060601949088DFCF70EFD41EC190B9FED61
:10BD5000170B53EC102BFCF714FC41EC180BFCF701
:10BD60002EFD20811049D1F82A00FCF7EBFC41ECB4
:10BD7000190B9FED0E0B53EC102BFCF702FC41EC62
:10BD8000180BFCF7FDFC06B266810748418EA181C5
:10BD9000E12029F0D7FAC5B2642D00DD6425E581E4
:10BDA000BDEC048B70BD00000CD200209A999999CB
:10BDB0009999B93F38B5044600200090002501202C
:10BDC0002070002060700820A0704FF4C170606087
:10BDD0001748D0F82A00002801DD012507E01448A3
:10BDE000D0F82A00002801DA022500E00025002012
:10BDF0001AF0C4F89DF8001060F3000100910120D2
:10BE00001AF0BCF89DF8001060F341010091022087
:10BE10001AF0B4F89DF8001060F3820100919DF8CB
:10BE200000002072257200216181A181E18138BD6D
:10BE30000CD2002010B50446012020700020607054
:10BE40000820A07040F283106060DA2029F07AFAAE
:10BE50002081DC2029F076FA6081DE2029F072FA58
:10BE6000A0F6AB20A081E02029F06CFAA0F6AB2070
:10BE7000E08110BD10B504460120207000206070E4
:10BE80000820A0704FF4C2706060D92029F05AFADF
:10BE90002081DB2029F056FA6081DD2029F052FA5A
:10BEA000A081DF2029F04EFAE08110BD0121017050
:10BEB000002141700821817040F28511416000210C
:10BEC00081600022C2607047012101700021417031
:10BED000082181704FF4C37141600021018100226B
:10BEE00042810C49B1F84E10C1F300220273094996
:10BEF000B1F84E10C1F3802242730649B1F84E10DA
:10BF0000C1F3402282730349B1F84E10C1F3C0223D
:10BF1000C27370470CD200200121017000214170D2
:10BF20000821817040F287114160114991F84E104B
:10BF3000C1F3001101720E4991F84E10C1F3801245
:10BF400042720B49B1F84E10C1F3C03282720849F7
:10BF5000D1F84E10C1F30042C2720549D1F84E101B
:10BF6000C1F340420273002242738273C27370476E
:10BF70000CD2002010B50446012020700020607013
:10BF80000820A07040F20F306060032019F0F6FF27
:10BF900010B10120208101E0002020810021618179
:10BFA000A181E18110BD000038B504460020009059
:10BFB00001202070002060700820A07040F2113035
:10BFC00060604D48D0F82A00002806DDBDF800006A
:10BFD00020F00300801C009011E04748D0F82A00B0
:10BFE000002806DABDF8000020F00300C01C009015
:10BFF00005E0BDF8000020F00300401C0090BDF8F3
:10C00000000020F008000090BDF8000020F01000B3
:10C0100000903948D0F84E00800C3749D1F84E10C6
:10C0200040EA51503449D1F84E1040EA915032491B
:10C03000D1F84E1040EA91602F49D1F84E1040EAF5
:10C04000D1402D49D1F84E1040EA1150BDF80010F2
:10C0500060F382010091012019F090FFBDF80010FB
:10C0600060F345110091002019F088FFBDF8001021
:10C0700060F38611009120484088012805DCBDF856
:10C08000000020F44070009006E0BDF8000020F4AD
:10C09000407000F500700090022019F06FFFBDF8AD
:10C0A000001060F38A210091D32029F04BF905029A
:10C0B000D32029F047F905EB10202081D12029F069
:10C0C00041F90502D12029F03DF905EB10206081EE
:10C0D000D22029F037F90502D22029F033F905EBF7
:10C0E0001020A081BDF800000002BDF8001000EB98
:10C0F0001120E08138BD00000CD200201FB504469D
:10C1000000200290039000900190012020700020F8
:10C1100060700820A07040F212306060364890F8DD
:10C120004E000009344991F84E1040EA5110BDF814
:10C13000001060F38611ADF800102F4890F84E0003
:10C1400080092D4991F84E1040EAD110BDF8001039
:10C1500060F3C711ADF800102748B0F84E00000A90
:10C16000BDF8061060F38201ADF806102248B0F861
:10C170004E00800ABDF8061060F3C301ADF806104A
:10C180001D48B0F84E00400ABDF8061060F30001EB
:10C19000ADF806101848B0F84E00C00ABDF80610F9
:10C1A00060F34101ADF806101348D0F84E00800C42
:10C1B000BDF8001060F34511ADF80010BDF80000A7
:10C1C0000002BDF8001000EB11202081BDF808002E
:10C1D0000002BDF8081000EB11206081064881784C
:10C1E000217300216173A1733F201BF031FE0249CE
:10C1F00089784843E0731FBD0CD200202DE9F0413F
:10C200002DED048B04460025002700260120207018
:10C21000002060700820A07040F213306060C820D9
:10C2200029F090F84FEA0028C82029F08BF808EB95
:10C2300010202081CA2029F085F88046C92029F0E5
:10C2400081F808EB00473846FCF77CFA41EC190B03
:10C250009FED170B53EC102BFCF793F941EC180BE7
:10C26000FCF78EFA05B2C5F3072000EB05206081CC
:10C27000F62029F067F8A0F6AB20C0F30728F620D7
:10C2800029F060F8A0F6AB2008EB0020A081D020B8
:10C2900029F058F8A073E12029F054F8C6B2642EB2
:10C2A00000DD6426E673BDEC048BBDE8F081000080
:10C2B0009A9999999999B93F2DE9F0410446002539
:10C2C00001202070002060700820A0704FF445709D
:10C2D00060601D48D0F84A504FF6E850854200D9BA
:10C2E0000546C5F3072000EB052020811648D0F84D
:10C2F0003E504FF6E850854200D90546C5F3072069
:10C3000000EB05206081DA2029F01CF80646DC20CD
:10C3100029F018F8301AC0F30727DA2029F012F8AC
:10C320000646DC2029F00EF8301A07EB0020A08129
:10C33000F32029F007F80602F32029F003F806EBB2
:10C340001020E081BDE8F0810CD20020F8B5044651
:10C35000002000900025012020700020607008203F
:10C36000A07040F219306060002019F007FE9DF8BF
:10C37000001060F3C7110091012019F0FFFD9DF836
:10C38000001060F386110091022019F0F7FD9DF86E
:10C39000001060F345110091032019F0EFFD9DF8A6
:10C3A000001060F3041100919DF800002072DA2063
:10C3B00028F0C8FF0602DA2028F0C4FF06EB1020A0
:10C3C00085B265722912A172DC2028F0BBFF06023B
:10C3D000DC2028F0B7FF06EB102085B2E5722912A9
:10C3E0002173D92028F0AEFF6073DB2028F0AAFF6C
:10C3F000A0730021E173F8BD10B504460120207040
:10C40000002060700820A0704FF4487060604720E2
:10C41000207254216172492028F094FFA0720221F9
:10C42000E1720D212173022161730D21A17300219D
:10C43000E17310BD00210122027000224270082227
:10C4400082704FF4487242604B220272532343724F
:10C45000542383724123C37252230373FF23437314
:10C460008373C373704770B50446012020700020A9
:10C4700060700820A07040F222306060DE2028F05A
:10C4800061FFA0F6AB20C0F30725DE2028F05AFF9D
:10C49000A0F6AB2005EB00202081E02028F052FF21
:10C4A000A0F6AB20C0F30725E02028F04BFFA0F654
:10C4B000AB2005EB00206081DD2028F043FF2073D6
:10C4C000DF2028F03FFF6073D02028F03BFFA073EF
:10C4D000D02028F037FFE07370BD000010B504468F
:10C4E00001202070002060700820A07040F22330EE
:10C4F00060603F201BF0ACFC0949897848432072FA
:10C5000047201BF0A5FC010A617247201BF0A0FC2C
:10C51000A0720021E17221736173A173E17310BDF8
:10C520000CD200200146012008700020487008202D
:10C5300088704FF4497048600020087200224A72E7
:10C540008A72CA72CA6001207047014601200870D1
:10C55000002048700820887040F2723048604FF622
:10C56000FF70088102464A818A81CA810120704792
:10C5700010B500210022012303700023437008231B
:10C5800083704FF4547343604FF6FF7303811C466E
:10C5900044818481C48110BD10B5044601202070FF
:10C5A000002060700820A07040F251306060D320FD
:10C5B00028F0C8FE2081D12028F0C4FE6081D2205E
:10C5C00028F0C0FEA081D42028F0BCFEE08110BD80
:10C5D00010B5044601202070002060700820A07073
:10C5E00040F251306060D32028F0ACFE2081D12091
:10C5F00028F0A8FE6081D22028F0A4FEA081D420DB
:10C6000028F0A0FEE08110BD10B504460120207086
:10C61000002060700820A07040F251306060D3208C
:10C6200028F090FE2081D12028F08CFE6081D2205D
:10C6300028F088FEA081D42028F084FEE08110BD7F
:10C6400010B5044601202070002060700820A07002
:10C6500040F251306060D32028F074FE2081D12058
:10C6600028F070FE6081D22028F06CFEA081D420DA
:10C6700028F068FEE08110BD10B50446012020704E
:10C68000002060700820A07040F251306060D3201C
:10C6900028F058FE2081D12028F054FE6081D2205D
:10C6A00028F050FEA081D42028F04CFEE08110BD7F
:10C6B00010B5044601202070002060700820A07092
:10C6C00040F251306060D32028F03CFE2081D12020
:10C6D00028F038FE6081D22028F034FEA081D420DA
:10C6E00028F030FEE08110BD10B504460120207016
:10C6F000002060700820A07040F251306060D320AC
:10C7000028F020FE2081D12028F01CFE6081D2205C
:10C7100028F018FEA081D42028F014FEE08110BD7E
:10C7200010B5044601202070002060700820A07021
:10C7300040F251306060D32028F004FE2081D120E7
:10C7400028F000FE6081D22028F0FCFDA081D420DA
:10C7500028F0F8FDE08110BD10B5044601202070DE
:10C76000002060700820A07040F251306060D3203B
:10C7700028F0E8FD2081D12028F0E4FD6081D2205E
:10C7800028F0E0FDA0810021E18110BD10B5044634
:10C7900001202070002060700820A07040F251300D
:10C7A0006060D32028F0CEFD2081D12028F0CAFD82
:10C7B0006081D22028F0C6FDA081D42028F0C2FDDF
:10C7C000E08110BD10B5044601202070002060708B
:10C7D0000820A07040F251306060D32028F0B2FDF4
:10C7E0002081D12028F0AEFD6081D22028F0AAFD62
:10C7F000A081D42028F0A6FDE08110BD70B50446CC
:10C80000002501202070002060700820A07040F2F8
:10C8100055306060D02028F095FD2081E12028F07F
:10C8200091FDC5B2642D00DD642565810021A181E3
:10C83000E18170BD70B50446002501202070002004
:10C8400060700820A07040F255306060D02028F061
:10C8500079FD2081E12028F075FDC5B2642D00DD51
:10C8600064256581D02028F06DFD00EBC00101EB4F
:10C8700000104FF6FF7101EA8001A1810021E181E2
:10C8800070BD70B504460025012020700020607046
:10C890000820A07040F255306060D02028F052FD92
:10C8A0002081E12028F04EFDC5B2642D00DD642515
:10C8B00065810021A181E18170BD70B5044600252C
:10C8C00001202070002060700820A07040F25530D8
:10C8D0006060D02028F036FD2081E12028F032FD74
:10C8E000C5B2642D00DD642565810021A181E1814F
:10C8F00070BD70B5044600250120207000206070D6
:10C900000820A07040F255306060D02028F01AFD59
:10C910002081E12028F016FDC5B2642D00DD6425DC
:10C920006581DA2028F00EFDA081DC2028F00AFDC8
:10C93000E08170BD70B50446002501202070002004
:10C9400060700820A07040F255306060D02028F060
:10C95000F9FC2081E12028F0F5FCC5B2642D00DD52
:10C96000642565810021A181E18170BD70B5044617
:10C97000002501202070002060700820A07040F287
:10C9800055306060D02028F0DDFC2081E12028F0C7
:10C99000D9FCC5B2642D00DD64256581D02028F066
:10C9A000D1FC00EBC00101EB00104FF6FF7101EA72
:10C9B0008001A1810021E18170BD70B50446002590
:10C9C00001202070002060700820A07040F25530D7
:10C9D0006060D02028F0B6FC2081E12028F0B2FC75
:10C9E000C5B2642D00DD642565810021A181E1814E
:10C9F00070BD70B5044600250120207000206070D5
:10CA00000820A07040F255306060E12028F09AFCC8
:10CA1000C5B2642D00DD6425D02028F093FC208170
:10CA200065810021A181E18170BD70B504460025BA
:10CA300001202070002060700820A07040F2553066
:10CA40006060D02028F07EFC2081E12028F07AFC74
:10CA5000C5B2642D00DD642565810021A181E181DD
:10CA600070BD000070B52DED048B0446002501203B
:10CA70002070002060700820A07040F25530606087
:10CA8000D02028F05FFC2081E12028F05BFCC5B2BB
:10CA9000642D00DD642565810B49D1F84200FBF768
:10CAA00062FE41EC190B9FED090B53EC102BFBF7C9
:10CAB00068FD41EC180BFBF782FEA0810021E181AB
:10CAC000BDEC048B70BD00000CD200207B14AE477F
:10CAD000E17A843F2DE9F0412DED048B04460026D8
:10CAE000002501202070002060700820A07040F216
:10CAF00056306060C82028F025FC2081CA2028F02C
:10CB000021FC0746C92028F01DFC07EB00463046F3
:10CB1000FBF718FE41EC190B9FED0C0B53EC102B9F
:10CB2000FBF72FFD41EC180BFBF72AFE05B26581E0
:10CB3000F62028F007FCA0F6AB20A081F32028F017
:10CB400001FCE081BDEC048BBDE8F0819A999999D4
:10CB50009999B93F2DE9F0412DED048B044600264B
:10CB6000002501202070002060700820A07040F295
:10CB700056306060062028F0E5FB2081CA2028F0AE
:10CB8000E1FB0746C92028F0DDFB07EB00463046F5
:10CB9000FBF7D8FD41EC190B9FED0C0B53EC102B60
:10CBA000FBF7EFFC41EC180BFBF7EAFD05B26581E2
:10CBB000F62028F0C7FBA0F6AB20A081F32028F0D8
:10CBC000C1FBE081BDEC048BBDE8F0819A99999995
:10CBD0009999B93F2DE9F0412DED048B04460026CB
:10CBE000002501202070002060700820A07040F215
:10CBF00056306060C82028F0A5FB2081CA2028F0AC
:10CC0000A1FB0746C92028F09DFB07EB00463046F4
:10CC1000FBF798FD41EC190B9FED0B0B53EC102B20
:10CC2000FBF7AFFC41EC180BFBF7AAFD05B26581E1
:10CC3000F62028F087FBA0F6AB20A0810021E1813F
:10CC4000BDEC048BBDE8F0819A9999999999B93F07
:10CC50002DE9F0412DED048B04460025002601202E
:10CC60002070002060700820A07040F25630606094
:10CC70001448008D2081CA2028F064FB0746C92093
:10CC800028F060FB07EB00452846FBF75BFD41EC15
:10CC9000190B9FED0D0B53EC102BFBF772FC41ECC5
:10CCA000180BFBF76DFD06B26681F62028F04AFBF3
:10CCB000A0F6AB20A0810021E181BDEC048BBDE892
:10CCC000F08100000CD200209A9999999999B93F66
:10CCD0002DE9F0412DED048B044600250120207044
:10CCE000002060700820A07040F25630606000267E
:10CCF000C82028F027FB2081CA2028F023FB074604
:10CD0000C92028F01FFB07EB00452846FBF71AFD5A
:10CD100041EC190B9FED0D0B53EC102BFBF731FC85
:10CD200041EC180BFBF72CFD06B26681DE2028F0E3
:10CD300009FBA0F6AB20A081E02028F003FBA0F6C1
:10CD4000AB20E081BDEC048BBDE8F0819A99999904
:10CD50009999B93F2DE9F0412DED048B044600254A
:10CD600001202070002060700820A07040F2563032
:10CD700060600026C82028F0E5FA2081CA2028F04B
:10CD8000E1FA0746C92028F0DDFA07EB00452846FE
:10CD9000FBF7D8FC41EC190B9FED0B0B53EC102B60
:10CDA000FBF7EFFB41EC180BFBF7EAFC06B26681E0
:10CDB000F62028F0C7FAA0F6AB20A0810021E1817F
:10CDC000BDEC048BBDE8F0819A9999999999B93F86
:10CDD0002DE9F0412DED048B0446002600250120AD
:10CDE0002070002060700820A07040F25630606013
:10CDF000C82028F0A7FA2081CA2028F0A3FA074605
:10CE0000C92028F09FFA07EB00463046FBF79AFC52
:10CE100041EC190B9FED0D0B53EC102BFBF7B1FB05
:10CE200041EC180BFBF7ACFC05B26581F62028F04D
:10CE300089FAA0F6AB20A0814FF484701BF008F8AB
:10CE4000E081BDEC048BBDE8F08100009A999999CE
:10CE50009999B93F2DE9F0412DED048B0446002549
:10CE600001202070002060700820A07040F2563031
:10CE700060600026C82028F065FA2081CA2028F0CA
:10CE800061FA0746C92028F05DFA07EB00452846FD
:10CE9000FBF758FC41EC190B9FED0B0B53EC102BDF
:10CEA000FBF76FFB41EC180BFBF76AFC06B26681DF
:10CEB000F62028F047FAA0F6AB20A0810021E181FE
:10CEC000BDEC048BBDE8F0819A9999999999B93F85
:10CED0002DE9F0412DED048B0446002600250120AC
:10CEE0002070002060700820A07040F25630606012
:10CEF000C82028F027FA2081CA2028F023FA074604
:10CF0000C92028F01FFA07EB00463046FBF71AFC51
:10CF100041EC190B9FED0B0B53EC102BFBF731FB86
:10CF200041EC180BFBF72CFC05B26581F62028F0CC
:10CF300009FAA0F6AB20A0810021E181BDEC048BB1
:10CF4000BDE8F0819A9999999999B93F2DE9F041F5
:10CF50002DED048B044600250026012020700020C2
:10CF600060700820A07040F2563060601448008D58
:10CF70002081CA2028F0E6F90746C92028F0E2F906
:10CF800007EB00452846FBF7DDFB41EC190B9FED55
:10CF90000D0B53EC102BFBF7F4FA41EC180BFBF7DD
:10CFA000EFFB06B26681F62028F0CCF9A0F6AB20A4
:10CFB000A0810021E181BDEC048BBDE8F08100007F
:10CFC0000CD200209A9999999999B93F2DE9F0418D
:10CFD0002DED048B04460025002601202070002042
:10CFE00060700820A07040F2563060601448008DD8
:10CFF0002081CA2028F0A6F90746C92028F0A2F906
:10D0000007EB00452846FBF79DFB41EC190B9FED14
:10D010000D0B53EC102BFBF7B4FA41EC180BFBF79C
:10D02000AFFB06B26681F62028F08CF9A0F6AB20A3
:10D03000A0810021E181BDEC048BBDE8F0810000FE
:10D040000CD200209A9999999999B93F10B500216D
:10D05000002201230370002343700823837040F2F1
:10D060005733436000230381002444818481C481B9
:10D0700010BD00000CB5002101910091012101704B
:10D08000002141700821817040F2593141603949D5
:10D0900091F84E100909374A92F84E2041EA521190
:10D0A000BDF8042061F308220192324991F84E1034
:10D0B0008909BDF8042061F3C71201922D49B1F826
:10D0C0004E10090A2B4AB2F84E2041EA9221294A11
:10D0D000B2F84E2041EA1231264AB2F84E2041EA17
:10D0E0005231BDF8042061F3C30201922149B1F825
:10D0F0004E10490A1F4AB2F84E2041EAD2211D4A79
:10D10000B2F84E2041EA9231BDF8042061F30412D6
:10D1100001921849D1F84E10890C164AD2F84E20C7
:10D1200041EA5251134AD2F84E2041EA9251114A33
:10D13000D2F84E2041EA92610E4AD2F84E2041EADE
:10D14000D2410C4AD2F84E2041EA1251BDF80420D7
:10D1500061F3CB220192BDF804100181BDF80020DB
:10D16000428104498A780273002242738273C27337
:10D170000CBD00000CD200200CB5002101910091E3
:10D1800001210170002141700821817040F2593164
:10D1900041603A4991F84E100909384A92F84E20F8
:10D1A00041EA5211BDF8042061F30822019233498B
:10D1B00091F84E108909BDF8042061F3C71201925D
:10D1C0002E49B1F84E10090A2C4AB2F84E2041EA15
:10D1D00092212A4AB2F84E2041EA1231274AB2F887
:10D1E0004E2041EA5231BDF8042061F3C30201929E
:10D1F0002249B1F84E10490A204AB2F84E2041EABD
:10D20000D2211E4AB2F84E2041EA9231BDF80420E4
:10D2100061F3041201921949D1F84E10890C174A92
:10D22000D2F84E2041EA5251144AD2F84E2041EA37
:10D230009251124AD2F84E2041EA92610F4AD2F836
:10D240004E2041EAD2410D4AD2F84E2041EA125115
:10D25000BDF8042061F3CB220192BDF804100181D6
:10D26000BDF80020428105498A780273502242733A
:10D270004E2282730022C2730CBD00000CD200202B
:10D2800010B52DED048B82B0044600200190009073
:10D2900001202070002060700820A07040F25930FA
:10D2A00060604C4890F84E0000094A4991F84E10D1
:10D2B00040EA5110BDF8041060F30821019145487F
:10D2C00090F84E008009BDF8041060F3C711019179
:10D2D0004048B0F84E00000A3E49B1F84E1040EA0E
:10D2E00091203C49B1F84E1040EA11303949B1F86B
:10D2F0004E1040EA5130BDF8041060F3C3010191B3
:10D300003448B0F84E00400A3249B1F84E1040EAB5
:10D31000D1203049B1F84E1040EA9130BDF80410E8
:10D3200060F3041101912B48D0F84E00800C29497C
:10D33000D1F84E1040EA51502649D1F84E1040EA3B
:10D3400091502449D1F84E1040EA91602149D1F81A
:10D350004E1040EAD1401F49D1F84E1040EA11501A
:10D36000BDF8041060F3CB210191BDF804002081C9
:10D37000BDF8001061811748817821730146D1F80A
:10D380004200FBF7F0F941EC190B9FED130B53EC46
:10D39000102BFBF7F6F841EC180BFBF710FA607353
:10D3A0000C49D1F84200FBF7DEF941EC190B9FED77
:10D3B0000A0B53EC102BFBF7E4F841EC180BFBF7CE
:10D3C000FEF9010AA1730021E17302B0BDEC048BE8
:10D3D00010BD00000CD200207B14AE47E17A843FE0
:10D3E0000CB50021019100910121017000214170D3
:10D3F0000821817040F259314160294991F84E105D
:10D400000909274A92F84E2041EA5211BDF804203A
:10D4100061F308220192224991F84E108909BDF862
:10D42000042061F3C71201921D49B1F84E10090A98
:10D430001B4AB2F84E2041EA9221194AB2F84E2016
:10D4400041EA1231164AB2F84E2041EA5231BDF893
:10D45000042061F3C30201921149B1F84E10490A48
:10D460000F4AB2F84E2041EAD2210D4AB2F84E20BE
:10D4700041EA9231BDF8042061F304120192BDF833
:10D4800004100181BDF80020428105498A780273A9
:10D4900000224273827391F83820C2730CBD0000E1
:10D4A0000CD200200CB500210191009101210170E6
:10D4B000002141700821817040F2593141602949B1
:10D4C00091F84E100909274A92F84E2041EA52116C
:10D4D000BDF8042061F308220192224991F84E1010
:10D4E0008909BDF8042061F3C71201921D49B1F802
:10D4F0004E10090A1B4AB2F84E2041EA9221194AFD
:10D50000B2F84E2041EA1231164AB2F84E2041EAF2
:10D510005231BDF8042061F3C30201921149B1F800
:10D520004E10490A0F4AB2F84E2041EAD2210D4A64
:10D53000B2F84E2041EA9231BDF8042061F30412A2
:10D540000192BDF804100181BDF800204281054917
:10D550008A780273502242734E2282730022C27371
:10D560000CBD00000CD2002010B504460120207034
:10D57000002060700820A07040F2593060600BF00D
:10D580008BFD208100216181044881782173552120
:10D5900061735A21A1730021E17310BD0CD20020E8
:10D5A0000CB5002101910091012101700021417011
:10D5B0000821817040F2593141603A4991F84E108A
:10D5C0000909384A92F84E2041EA5211BDF8042068
:10D5D00061F308220192334991F84E108909BDF890
:10D5E000042061F3C71201922E49B1F84E10090AC6
:10D5F0002C4AB2F84E2041EA92212A4AB2F84E2033
:10D6000041EA1231274AB2F84E2041EA5231BDF8C0
:10D61000042061F3C30201922249B1F84E10490A75
:10D62000204AB2F84E2041EAD2211E4AB2F84E20DA
:10D6300041EA9231BDF8042061F3041201921949C4
:10D64000D1F84E10890C174AD2F84E2041EA5251B7
:10D65000144AD2F84E2041EA9251124AD2F84E2092
:10D6600041EA92610F4AD2F84E2041EAD2410D4A76
:10D67000D2F84E2041EA1251BDF8042061F3CB22CA
:10D680000192BDF804100181BDF8002042810549D6
:10D690008A780273502242734E2282730022C27330
:10D6A0000CBD00000CD200201CB5044600200190E7
:10D6B000009001202070002060700820A07040F2CF
:10D6C000593060600BF0CFFA0190019820720198F8
:10D6D000010A61720BF0CCFA0090BDF80000A07254
:10D6E000BDF80000010AE17204488178217301212C
:10D6F00061730021A173E1731CBD00000CD20020F6
:10D700000EB50021029100910191012101700021CB
:10D7100041700821817040F25A314160244991F8EA
:10D720004E10C1F30011224A92F84E20C2F340126B
:10D730001143029A61F3114202921D4991F84E1071
:10D74000C1F38012029962F38F3102911849B1F846
:10D750004E10C1F30022029962F38B210291144909
:10D76000B1F84E10C1F34022029962F30D310291DB
:10D770000F49D1F84E10C1F38042029962F315515E
:10D7800002910B49B1F84E10C1F38022029962F365
:10D79000871102910649B1F84E10C1F3C0220299D7
:10D7A00062F30921029102998160009AC2600EBD64
:10D7B0000CD200200EB500210291009101910121AF
:10D7C0000170002141700821817040F25A3141609E
:10D7D000274991F84E10C1F30011254A92F84E20C6
:10D7E000C2F340121143029A61F31142029220499E
:10D7F00091F84E10C1F380111D4A92F84E20C2F3E9
:10D80000C0121143029A61F38F3202921849B1F8A3
:10D810004E10C1F30022029962F38B210291144948
:10D82000B1F84E10C1F34022029962F30D3102911A
:10D830000F49D1F84E10C1F38042029962F315519D
:10D8400002910B49B1F84E10C1F38022029962F3A4
:10D85000871102910649B1F84E10C1F3C022029916
:10D8600062F30921029102998160009AC2600EBDA3
:10D870000CD200200EB500210291009101910121EE
:10D880000170002141700821817040F25A314160DD
:10D89000244991F84E10C1F30011224A92F84E200B
:10D8A000C2F340121143029A61F3114202921D49E0
:10D8B00091F84E10C1F38012029962F38F310291F8
:10D8C0001849B1F84E10C1F30022029962F38B217E
:10D8D00002911449B1F84E10C1F34022029962F34B
:10D8E0000D3102910F49D1F84E10C1F380420299D7
:10D8F00062F3155102910B49B1F84E10C1F3802229
:10D90000029962F3871102910649B1F84E10C1F3F2
:10D91000C022029962F30921029102998160009A62
:10D92000C2600EBD0CD200200121017000214170A7
:10D930000821817040F25B314160002101810022A9
:10D9400042818281C281704738B504460020009030
:10D9500001202070002060700820A0704FF45770E4
:10D960006060022018F00AFB9DF8001060F345117A
:10D970000091032018F002FB9DF8001060F30411E1
:10D980000091002018F0FAFA9DF8001060F3C7111A
:10D990000091012018F0F2FA9DF8001060F3861152
:10D9A00000919DF800002072002161726181A181C7
:10D9B000E18138BD38B50446012020700020607038
:10D9C0000820A0704FF45770606000200090022083
:10D9D00018F0D4FA9DF8001060F34511009103206F
:10D9E00018F0CCFA9DF8001060F3041100910020AB
:10D9F00018F0C4FA9DF8001060F3C71100910120DF
:10DA000018F0BCFA9DF8001060F3861100915320C5
:10DA100027F098FC9DF8001060F3C30100919DF879
:10DA200000002072002161726181A181E18138BD15
:10DA300038B5044601202070002060700820A070D6
:10DA40004FF45770606000200090022018F096FAA2
:10DA50009DF8001060F304110091032018F08EFA75
:10DA60009DF8001060F345110091002018F086FA2F
:10DA70009DF8001060F3C7110091012018F07EFAA4
:10DA80009DF8001060F386110091532027F05AFC96
:10DA90009DF8001060F3C30100919DF80000207212
:10DAA00000216172F32027F04DFC60810021A181EB
:10DAB000E18138BD38B50446012020700020607037
:10DAC0000820A0704FF45770606000200090022082
:10DAD00018F054FA9DF8001060F345118DF800100D
:10DAE000032018F04BFA9DF8001060F304118DF834
:10DAF0000010002018F042FA9DF8001060F3C711E2
:10DB00008DF80010012018F039FA9DF8001060F32C
:10DB100086118DF80010532027F014FCC0B28DF848
:10DB200001009DF800002072002161726181A181D5
:10DB3000E18138BD38B504460120207000206070B6
:10DB40000820A0704FF45770606000200090022001
:10DB500018F014FA9DF8001060F345118DF80010CC
:10DB6000032018F00BFA9DF8001060F304118DF8F3
:10DB70000010002018F002FA9DF8001060F3C711A1
:10DB80008DF80010012018F0F9F99DF8001060F3ED
:10DB900086118DF80010532027F0D4FBC0B28DF809
:10DBA00001009DF800002072002161726181A18155
:10DBB000E18138BD38B50446012020700020607036
:10DBC0000820A0704FF4577060600020009018F09B
:10DBD000D5F99DF8001060F3C7110091012018F0ED
:10DBE000CDF99DF8001060F386110091022018F025
:10DBF000C5F99DF8001060F345110091032018F05D
:10DC0000BDF99DF8001060F304110091532027F036
:10DC100099FB9DF8001060F3C30100910AF06EF9C2
:10DC20002072002161726181A181E18138BD38B526
:10DC3000044601202070002060700820A0704FF47E
:10DC40005770606000200090022018F097F99DF84E
:10DC5000001060F345110091032018F08FF99DF832
:10DC6000001060F304110091002018F087F99DF86E
:10DC7000001060F3C7110091012018F07FF99DF8A2
:10DC8000001060F386110091532027F05BFB9DF894
:10DC9000001060F3C30100919DF800002072002184
:10DCA00061726181A181E18138BD38B504460120EE
:10DCB0002070002060700820A0704FF457706060E2
:10DCC0000020009018F05AF99DF8001060F3C71179
:10DCD0000091012018F052F99DF8001060F38611B0
:10DCE0000091022018F04AF99DF8001060F34511E8
:10DCF0000091032018F042F99DF8001060F3041120
:10DD00000091532027F01EFB9DF8001060F3C30123
:10DD100000919DF800002072002161726181A18153
:10DD2000E18138BD10B504460120207000206070EC
:10DD30000820A07040F25E30606004F10802042107
:10DD4000EC201AF091F810BD10B5044601202070A7
:10DD5000002060700820A07040F25E30606004F126
:10DD600008020421EC201AF07FF810BD0121017097
:10DD7000002141700821817040F25E3141605021E4
:10DD80000172592242724C2282724F22C2724E227A
:10DD90000273202242738273C273704710B5044627
:10DDA00001202070002060700820A07040F25E30DA
:10DDB000606004F108020421EC201AF055F810BD4F
:10DDC00010B5044601202070002060700820A0706B
:10DDD00040F25E30606004F108020421EC201AF089
:10DDE00043F810BD10B5044601202070002060707B
:10DDF0000820A07040F25E30606004F10802042147
:10DE0000EC201AF031F810BD70B5044601202070E6
:10DE1000002060700820A07040F25E306060002535
:10DE200004F108020421EC201AF01EF870BD10B5B0
:10DE3000044601202070002060700820A07040F28D
:10DE40005E30606004F108020421EC201AF00CF846
:10DE500010BD000070B52DED048B0446012020702C
:10DE6000002060700820A07040F25F3060600020E9
:10DE7000208184216181D82027F064FA0546FAF7D1
:10DE800072FC41EC190B9FED080B53EC102BFAF7C9
:10DE900078FB41EC180BFAF792FCA0810021E1819C
:10DEA000BDEC048B70BD00007B14AE47E17A843F6B
:10DEB00001210170002141700821817040F25F3121
:10DEC00041604A210172422242720D228272022274
:10DED000C27200228281C28170470121017000213B
:10DEE00041700821817040F25F3141600021017270
:10DEF000002242720D2282720222C27200228281AC
:10DF0000C281704770B52DED048B0446012020704E
:10DF1000002060700820A07040F25F306060002038
:10DF2000208143F2CA216181D82027F00BFA0546EF
:10DF3000FAF719FC41EC190B9FED070B53EC102B72
:10DF4000FAF71FFB41EC180BFAF739FCA08100210E
:10DF5000E181BDEC048B70BD7B14AE47E17A843F58
:10DF600010B5044601202070002060700820A070C9
:10DF70004FF45C70606004F108020421C82019F0BD
:10DF800073FF10BD10B504460120207000206070A2
:10DF90000820A0704FF45C706060DE2027F0D2F99A
:10DFA000A0F6AB202081E02027F0CCF9A0F6AB2032
:10DFB0006081DA2027F0C6F9A081DC2027F0C2F9C1
:10DFC000E08110BD10B50446012020700020607073
:10DFD0000820A0704FF45C706060DE2027F0B2F97A
:10DFE000A0F6AB202081E02027F0ACF9A0F6AB2012
:10DFF0006081DA2027F0A6F9A081DC2027F0A2F9C1
:10E00000E08110BD10B50446012020700020607032
:10E010000820A0704FF45C706060DE2027F092F959
:10E02000A0F6AB202081E02027F08CF9A0F6AB20F1
:10E030006081DA2027F086F9A081DC2027F082F9C0
:10E04000E08110BD10B504460120207000206070F2
:10E050000820A07040F27130606004F108020421D1
:10E06000CC2019F001FF10BD10B50446012020702E
:10E07000002060700820A07040F271306060DD20E8
:10E0800027F060F92081DF2027F05CF96081D9203A
:10E0900027F058F9A081DB2027F054F9E08110BD6A
:10E0A00010B5044601202070002060700820A07088
:10E0B00040F271306060DD2027F044F92081DF20DC
:10E0C00027F040F96081D92027F03CF9A081DB20BE
:10E0D00027F038F9E08110BD10B50446012020700A
:10E0E000002060700820A07040F271306060DD2078
:10E0F00027F028F92081DF2027F024F96081D9203A
:10E1000027F020F9A081DB2027F01CF9E08110BD69
:10E1100001210170002141700821817040F27231AB
:10E120004160044949880181002242818281C28183
:10E13000704700000CD200200121017000214170C5
:10E140000821817040F2723141600449498801819F
:10E15000002242818281C281704700000CD20020DF
:10E1600070B52DED048B04460120207000206070F6
:10E170000820A07040F273306060DC2027F0E2F8E5
:10E180002081DA2027F0DEF86081E02027F0DAF83D
:10E190000546FAF7E8FA41EC190B9FED100B53EC2A
:10E1A000102BFAF7EEF941EC180BFAF708FBA081F7
:10E1B000DE2027F0C7F80546FAF7D5FA41EC190B2F
:10E1C0009FED060B53EC102BFAF7DBF941EC180B23
:10E1D000FAF7F5FAE081BDEC048B70BD9A99999934
:10E1E0009999B93F70B52DED048B0446012020703C
:10E1F000002060700820A07040F273306060DC2066
:10E2000027F0A0F82081DA2027F09CF86081E02038
:10E2100027F098F80546FAF7A6FA41EC190B9FED9E
:10E22000100B53EC102BFAF7ACF941EC180BFAF782
:10E23000C6FAA081DE2027F085F80546FAF793FAA2
:10E2400041EC190B9FED060B53EC102BFAF799F9E3
:10E2500041EC180BFAF7B3FAE081BDEC048B70BD0A
:10E260009A9999999999B93F70B52DED048B044607
:10E2700001202070002060700820A07040F27330F0
:10E280006060DC2027F05EF80546FAF76CFA41EC96
:10E29000190B9FED160B53EC102BFAF772F941ECAA
:10E2A000180BFAF78CFA2081DA2027F04BF8054694
:10E2B000FAF759FA41EC190B9FED0C0B53EC102BAC
:10E2C000FAF75FF941EC180BFAF779FA6081E02070
:10E2D00027F038F8A0F6AB20A081DE2027F032F836
:10E2E000A0F6AB20E081BDEC048B70BD7B14AE4783
:10E2F000E17A843F01210170002141700821817081
:10E300004FF45D71416049210172442242723A2208
:10E3100082721049B1F854100912302202EB111226
:10E32000C2720C49B1F85410C1F3032130310173AA
:10E330002E224273074991F85410C1F30311303172
:10E340008173044991F8541001F00F013031C17309
:10E35000704700000CD2002010B5002100220123DC
:10E36000037000234370082383704FF45D73436090
:10E37000124BB3F854301912104B93F854200A235F
:10E3800091FBF3F3303303720A2391FBF3F403FBA5
:10E390001413303343720A2392FBF3F33033837246
:10E3A0000A2392FBF3F403FB14233033C3720024DB
:10E3B000047344738473C47310BD00000CD2002036
:10E3C00010B5044601202070002060700820A07065
:10E3D0004FF45D706060DB2026F0B4FF2081D9200F
:10E3E00026F0B0FF6081DF2026F0ACFFA081DD20A9
:10E3F00026F0A8FFE08110BD0121017000214170CD
:10E400000821817040F27531416049210172442236
:10E4100042723A2282721049B1F852100912302227
:10E4200002EB1112C2720C49B1F85210C1F3032170
:10E43000303101732E224273074991F85210C1F313
:10E44000031130318173044991F8521001F00F012A
:10E450003031C173704700000CD2002010B500218C
:10E46000002201230370002343700823837040F2CD
:10E4700075334360124BB3F852301912104B93F8B6
:10E4800052200A2391FBF3F3303303720A2391FBEA
:10E49000F3F403FB1413303343720A2392FBF3F3B8
:10E4A000303383720A2392FBF3F403FB14233033DB
:10E4B000C3720024047344738473C47310BD0000DA
:10E4C0000CD2002070B504460025012020700020E9
:10E4D00060700820A07040F275306060D22026F095
:10E4E00031FF00B102252572002161726181A18195
:10E4F000E18170BD10B504460120207000206070DD
:10E500000820A07040F276306060492020724421DB
:10E5100061723A21A1723021E172312121732E21E1
:10E5200061732A2026F00EFFC0F303103030A07371
:10E530002A2026F007FF00F00F003030E07310BDF6
:10E5400010B500210022012303700023437008232B
:10E55000837040F276334360124BB3F85C3019128B
:10E56000104B93F85C200A2391FBF3F330330372D2
:10E570000A2391FBF3F403FB1413303343720A2391
:10E5800092FBF3F3303383720A2392FBF3F403FB21
:10E5900014233033C3720024047344738473C4732C
:10E5A00010BD00000CD2002010B5044601202070E0
:10E5B000002060700820A07040F277306060492031
:10E5C0002072442161723A21A1723021E17231211D
:10E5D00021732E216173282026F0B4FEC0F30310AE
:10E5E0003030A073282026F0ADFE00F00F00303050
:10E5F000E07310BD10B50021002201230370002339
:10E6000043700823837040F277334360124BB3F8B2
:10E610005C301912104B93F85C200A2391FBF3F342
:10E62000303303720A2391FBF3F403FB14133033EA
:10E6300043720A2392FBF3F3303383720A2392FB73
:10E64000F3F403FB14233033C372002404734473C4
:10E650008473C47310BD00000CD20020012101702E
:10E6600000214170082181704FF45E7141600021EA
:10E6700081600022C260704770B52DED048B0446A6
:10E6800001202070002060700820A07040F27930D6
:10E6900060604FF4827019F0DBFB0D49498800FB84
:10E6A00001F52846FAF74EF841EC190B9FED090BDE
:10E6B00053EC102BF9F765FF41EC180BFAF77FF8D4
:10E6C000208100216181A181E181BDEC048B70BDBD
:10E6D0000CD200207B14AE47E17A843F70B52DED5B
:10E6E000048B044601202070002060700820A07078
:10E6F00040F2793060604FF4827019F0A9FB0D4947
:10E70000498800FB01F52846FAF71CF841EC190B83
:10E710009FED090B53EC102BF9F733FF41EC180B6D
:10E72000FAF74DF8208100216181A181E181BDECE2
:10E73000048B70BD0CD200207B14AE47E17A843F7D
:10E7400010B52DED048B0446012020700020607070
:10E750000820A07040F2793060600C49D1F8420086
:10E76000FAF701F841EC190B9FED090B53EC102B54
:10E77000F9F707FF41EC180BFAF721F8208103485D
:10E7800041886181BDEC048B10BD00000CD20020DB
:10E790007B14AE47E17A843F10B504460120207017
:10E7A000002060700820A0704FF46070606004F179
:10E7B00008020421DA2019F057FB10BD0121017075
:10E7C00000214170082181704FF460714160002187
:10E7D0000181002242818281C281704710B50446C6
:10E7E00001202070002060700820A07040F281306D
:10E7F000606004F108020421DE2019F035FB10BD31
:10E8000001210170002141700821817040F28131A5
:10E81000416000210181002242818281C2817047D2
:10E8200001210170002141700821817040F2823184
:10E8300041604A21017242224272442282720022C5
:10E84000C272027342738273C27370472DE9F04340
:10E85000ADF5497D074688464FF0000900250026A2
:10E8600000244FF4F07151A8F9F7C9FD4FF4A071DD
:10E8700001A8F9F7C4FD012F03DD0DF5497DBDE8C1
:10E88000F083FB2019F0E4FA00F0FF0901A93846F3
:10E89000FBF7A6FC06463EB10021582026F05EFD9F
:10E8A0000021592026F05AFD00240AE001A80FC8D3
:10E8B0000DF024FC012802D1B2200DF0DDF9601C1E
:10E8C000C4B2B442F2DBB9F1100F7DD2DFE809F037
:10E8D0000826466484A2C0DEFDFCFBFAF9F8F7F6D0
:10E8E00051A940461BF0EAFD0546002411E051A85D
:10E8F00000EB0410C068009051A800EB041C3846DF
:10E900009CE80E00FBF78CFC142026F0E7F9601C55
:10E91000C4B2AC4201DA1E2CE9DBEEE1F2B201AB8B
:10E9200051A940460BF072F90546002411E051A8A8
:10E9300000EB0410C068009051A800EB041C38469E
:10E940009CE80E00FBF76CFC142026F0C7F9601C55
:10E95000C4B2AC4201DA1E2CE9DBCEE151A940463B
:10E960000BF016F90546002411E051A800EB041045
:10E97000C068009051A800EB041C38469CE80E00CB
:10E98000FBF74EFC142026F0A9F9601CC4B2AC427F
:10E9900001DA1E2CE9DBB0E151A9404623F0B0F8C2
:10E9A0000546002413E051A800EB0410C068009055
:10E9B00051A800EB041C38469CE80E00FBF730FC25
:10E9C000142026F08BF900E079E1601CC4B2AC425F
:10E9D00001DA1E2CE7DB90E151A9404626F0CCFC81
:10E9E0000546002411E051A800EB0410C068009017
:10E9F00051A800EB041C38469CE80E00FBF710FC05
:10EA0000142026F06BF9601CC4B2AC4201DA1E2C53
:10EA1000E9DB72E151A9404611F0FCFE05460024F5
:10EA200011E051A800EB0410C068009051A800EB61
:10EA3000041C38469CE80E00FBF7F2FB142026F07D
:10EA40004DF9601CC4B2AC4201DA1E2CE9DB54E182
:10EA500051A9404612F068F90546002411E051A87A
:10EA600000EB0410C068009051A800EB041C38466D
:10EA70009CE80E00FBF7D4FB142026F02FF9601C55
:10EA8000C4B2AC4201DA1E2CE9DB36E151A94046A2
:10EA900005F06EF8054600241AE051A800EB0410BA
:10EAA000C068009051A800EB041C38469CE80E009A
:10EAB000FBF7B6FB142026F011F907E0E1E0C2E015
:10EAC000A3E082E063E044E025E006E0601CC4B21D
:10EAD000AC4201DA1E2CE0DB0FE151A940461BF0ED
:10EAE000EDFC0546002411E051A800EB0410C068BD
:10EAF000009051A800EB041C38469CE80E00FBF780
:10EB00008FFB142026F0EAF8601CC4B2AC4201DA94
:10EB10001E2CE9DBF1E051A9404621F05DF80546E5
:10EB2000002411E051A800EB0410C068009051A827
:10EB300000EB041C38469CE80E00FBF771FB142028
:10EB400026F0CCF8601CC4B2AC4201DA1E2CE9DB22
:10EB5000D3E051A94046FCF773FC0546002411E0C0
:10EB600051A800EB0410C068009051A800EB041CF1
:10EB700038469CE80E00FBF753FB142026F0AEF855
:10EB8000601CC4B2AC4201DA1E2CE9DBB5E051A92D
:10EB9000404623F045FB0546002411E051A800EB58
:10EBA0000410C068009051A800EB041C38469CE893
:10EBB0000E00FBF735FB142026F090F8601CC4B261
:10EBC000AC4201DA1E2CE9DB97E0F2B201AB51A9AD
:10EBD00040460DF067F90546002411E051A800EB0E
:10EBE0000410C068009051A800EB041C38469CE853
:10EBF0000E00FBF715FB142026F070F8601CC4B261
:10EC0000AC4201DA1E2CE9DB77E051A9404622F044
:10EC100077FF0546002411E051A800EB0410C068FE
:10EC2000009051A800EB041C38469CE80E00FBF74E
:10EC3000F7FA142026F052F8601CC4B2AC4201DA94
:10EC40001E2CE9DB59E051A9404612F0ABF905460C
:10EC5000002411E051A800EB0410C068009051A8F6
:10EC600000EB041C38469CE80E00FBF7D9FA142090
:10EC700026F034F8601CC4B2AC4201DA1E2CE9DB89
:10EC80003BE051A94046FCF7CFFD0546002411E0CA
:10EC900051A800EB0410C068009051A800EB041CC0
:10ECA00038469CE80E00FBF7BBFA142026F016F855
:10ECB000601CC4B2AC4201DA1E2CE9DB1DE051A994
:10ECC00040461BF0FBFB0546002411E051A800EB79
:10ECD0000410C068009051A800EB041C38469CE862
:10ECE0000E00FBF79DFA142025F0F8FF601CC4B25B
:10ECF000AC4201DA1E2CE9DB00BF00BF00BFBCE55F
:10ED000010B5029C2046FCF7C1FF10342046FCF7EA
:10ED1000CDFF022010BD10B5029C002010BD10B523
:10ED2000029C002010BD10B5029C012010BD10B542
:10ED3000029C20461034FDF7F5FB20461034FDF709
:10ED400004FC022010BD10B5029C012010BD30B59E
:10ED50000446481C60434FF47A7590FBF5F5481C57
:10ED6000401B1860186808B9012018601868082846
:10ED700001D9082018601868081A10601068102857
:10ED800004D9102010601068081A1860481C1D680B
:10ED9000401B4FF47A7568434D1C90FBF5F030BD75
:10EDA0002DE9F04704460F4615464FF00008C146CE
:10EDB0000026B81E81B2204600F022FC8046B81E14
:10EDC000215C781E205C01EB00201FFA80F9C84509
:10EDD00002D00220BDE8F087207828706078687043
:10EDE000E078A17800EB012068806079217900EB60
:10EDF0000120A880E079A17900EB0120E8800026BD
:10EE000010E0092000EB4600205C082101EB4601E0
:10EE1000615C00EB012081B205F1080020F81610BA
:10EE2000701C86B2E888B04201DD802EE9DB01204B
:10EE3000D0E701460022C1F30320C1F303131844B5
:10EE400001F00F03C218D043401C00F00F02B2EBD8
:10EE5000113F01D1012070470020FCE710B508F0F8
:10EE6000C9FF01210C4808F0A2F8012812D1402165
:10EE70004FF0402008F0A3F80A2011F0E6FF8021AF
:10EE80004FF0402008F09BF808F0B4FF4FF4FA7000
:10EE900011F0DBFF10BD00004040004070B586B0AF
:10EEA00006460C460020059014216846F9F7A7FA9B
:10EEB00000255748407800287ED15548807820B1F9
:10EEC00001282ED0022878D17EE051488068204465
:10EED0004F49886008468068C82805D300208860AC
:10EEE0000021304600F0BEF84948C0682044484937
:10EEF000C8600846C068B0F5FA6F11D3002088607A
:10EF0000012088700220C87000200861C86008468F
:10EF1000C178304600F0A6F801210020FBF746FC3E
:10EF200073E03B488068204439498860084680681F
:10EF3000C82806D3002088600846C178304600F013
:10EF400091F83046FBF7E2F9012820D13046FBF773
:10EF5000A9F9C5B2142D00DB14252A4669463046AE
:10EF6000FBF77AF905AA2946684600F053F801280C
:10EF70000DD12748C0789DF81410884204D1244848
:10EF8000C078401C2249C8700020214908612048EF
:10EF9000006920441E49086108460069B0F57A7F7F
:10EFA00011D30220887000210846FBF7FFFBFF21E8
:10EFB000304600F057F801E028E025E00020144931
:10EFC00088600861C86020E0114800692044104949
:10EFD0000861084680682044886008460069B0F5EA
:10EFE0007A7F05D3552048700020887088600AE039
:10EFF00007488068C82806D3002005498860FF219B
:10F00000304600F02FF800E000BF00BF06B070BD32
:10F01000B4F900202DE9F04104460D4616460027BC
:10F02000B846052D02D00020BDE8F0812078DD280B
:10F0300016D16078BB2813D1A81E81B2204611F0EA
:10F0400051FF0746A81E215C681E205C01EB0020D2
:10F050001FFA80F8474503D1A07830700120E3E71C
:10F060000020E1E7FEB507460D46002400260020FB
:10F07000009001900290DD222146641C0DF80120D1
:10F08000AA222146641C0DF801202146641C0DF8BB
:10F0900001502146684611F025FF0646F2B221468E
:10F0A000641C0DF8012032122146641C0DF8012069
:10F0B000224669463846FBF75FF9FEBD2DE9F04769
:10F0C0002DED048B04460F460025A8460026AA46CF
:10F0D000A946522026F036F929466D1C605451226B
:10F0E00029466D1C6254002229466D1C6254294633
:10F0F0006D1C6254FF2229466D1C625429466D1C0A
:10F100006254002229466D1C625429466D1C6254CB
:10F11000AA48068D320A29466D1C625429466D1C88
:10F1200066540146D1F82A00F9F70CFB41EC190BA3
:10F130009FEDA30B53EC102BF9F723FA41EC180BBE
:10F14000F9F71EFB82460FFA8AF9C9F3072229460E
:10F150006D1C625429466D1C04F801909748468E38
:10F16000320A29466D1C625429466D1C6654868EEF
:10F17000320A29466D1C62542846691C8DB22654F9
:10F180000A2026F0DFF800F6B706C6F30722284665
:10F19000691C8DB222542846691C8DB226548748BA
:10F1A000868C320A2846691C8DB222542846691C76
:10F1B0008DB226548148C68C320A2846691C8DB20D
:10F1C00022542846691C8DB226547C48C68D320ACA
:10F1D0002846691C8DB222542846691C8DB22654DB
:10F1E0007648068E320A2846691C8DB2225428467B
:10F1F000691C8DB22654714890F85E60320A284628
:10F20000691C8DB222542846691C8DB226546B4964
:10F21000D1F84A00F9F7A7FA41EC190B9FED680BFA
:10F2200053EC102BF9F7ADF941EC180BF9F7C7FACD
:10F230000646C6F307222846691C8DB2225428468A
:10F24000691C8DB226545D49D1F83E00F9F78BFA5E
:10F2500041EC190B9FED5A0B53EC102BF9F791F978
:10F2600041EC180BF9F7ABFA0646C6F3072228461D
:10F27000691C8DB222542846691C8DB226544F4811
:10F280004688320A2846691C8DB222542846691CD9
:10F290008DB226544948866BC6F307222846691C5E
:10F2A0008DB222542846691C8DB226544348C68E1E
:10F2B000320A2846691C8DB222542846691C8DB238
:10F2C00026543E48D0F84E60320E2846691C8DB256
:10F2D0002254C6F307422846691C8DB22254C6F355
:10F2E00007222846691C8DB222542846691C8DB21B
:10F2F00026543248B0F85260320A2846691C8DB252
:10F3000022542846691C8DB226542C48B0F854600B
:10F31000320A2846691C8DB222542846691C8DB2D7
:10F3200026542648B0F85A60320A2846691C8DB225
:10F3300022542846691C8DB226542048B0F85C60DF
:10F34000320A2846691C8DB222542846691C8DB2A7
:10F350002654FB2018F07CFD0646320A2846691C1C
:10F360008DB222542846691C8DB22654FD2018F017
:10F370006FFD0646320A2846691C8DB22254284683
:10F38000691C8DB22654A5F10806300AA071E671F9
:10F390002946204600F034F980462846691C8DB283
:10F3A00004F800804FEA28222846691C8DB22254B6
:10F3B0003D80BDEC048BBDE8F08700000CD200203E
:10F3C0009A9999999999B93FF0B587B006460C4634
:10F3D00000200690142101A8F9F711F800255D48D6
:10F3E0004078002871D15B48807820B101280ED088
:10F3F00002286BD193E000210846FBF7D7F90021E2
:10F40000522025F0ABFF0120524988709EE0304623
:10F41000FAF77CFF012869D13046FAF743FFC5B2FD
:10F42000142D00DB14252A4601A93046FAF714FFF3
:10F4300006AA294601A800F08FF8012856D19DF8A8
:10F440001800FF2805D155204249487000208870D7
:10F4500049E09DF8180020B900210846FBF7A6F9FD
:10F4600041E09DF8180000281FDD522025F06AFFBA
:10F47000D8B90920FBF7FAF8012834D19DF8181003
:10F48000522025F06BFF9DF81810FE2018F044FE66
:10F4900000210846FBF78AF9522025F053FFC7B236
:10F4A0003946304600F080F81DE0522025F04AFF32
:10F4B0009DF8181088420AD1522025F043FFC7B2A8
:10F4C0003946304600F070F80DE040E03DE0522053
:10F4D00025F038FF401C9DF81810884203D1012107
:10F4E0000020FBF763F900201A49086119480069F8
:10F4F0002044184908610846006940F6B83188423E
:10F500000CD302201349887055204870002108460A
:10F51000FBF74CF900200F498860086116E00D48A0
:10F52000806820440B49886008468068B0F57A7F7F
:10F530000AD3552048700020887000210846FBF748
:10F5400035F900200349886000E000BF00BF07B024
:10F55000F0BD0000B4F900202DE9F04104460D464D
:10F5600016460027B846052D02D00020BDE8F081E0
:10F570002078DD2816D16078AA2813D1A81E81B280
:10F58000204611F0AFFC0746A81E215C681E205CD7
:10F5900001EB00201FFA80F8474503D1A0783070B6
:10F5A0000120E3E70020E1E7FEB507460D46002411
:10F5B00000260020009001900290DD222146641C6C
:10F5C0000DF80120BB222146641C0DF801202146C4
:10F5D000641C0DF801502146684611F083FC064674
:10F5E000F2B22146641C0DF8012032122146641C3F
:10F5F0000DF80120224669463846FAF7BDFEFEBDE9
:10F6000030B502460B4600214FF6FF7010E012F8AD
:10F61000014B6040002109E000F0010424B14AF2EE
:10F62000010484EA600000E04010491C0829F3DB73
:10F630001C1EA3F10105ABB2E9D130BD10B501210B
:10F64000084603F03EFE00211820FBF7AFF800212A
:10F650001520FBF7ABF84FF4967025F03FFB012027
:10F660000749087001211820FBF7A0F80121152097
:10F67000FBF79CF80021084603F023FE10BD0000B4
:10F680003A3200200FB42DE9F041499F489D0024F3
:10F690000026522025F056FE012804D00020BDE8A7
:10F6A000F0015DF814FB45F6A3214A2025F056FE33
:10F6B0009DF818202046611C8CB22A549DF8192010
:10F6C0002046611C8CB22A54BDF81A000212204652
:10F6D000611C8CB22A54BDF81A00C2B22046611CCB
:10F6E0008CB22A54BDF81C0002122046611C8CB258
:10F6F0002A54BDF81C00C2B22046611C8CB22A54A8
:10F7000000222046611C8CB22A5401222046611C32
:10F710008CB22A5421462846FFF772FF064620463F
:10F72000611C8CB22E5432122046611C8CB22A54B9
:10F730003C800120B3E70FB42DE9F041499F489D7B
:10F7400000240026522025F0FDFD012804D00020D1
:10F75000BDE8F0015DF814FB45F6A4214A2025F030
:10F76000FDFD9DF818202046611C8CB22A549DF89E
:10F7700019202046611C8CB22A54BDF81A000212CE
:10F780002046611C8CB22A54BDF81A00C2B2204631
:10F79000611C8CB22A54BDF81C0002122046611C68
:10F7A0008CB22A54BDF81C00C2B22046611C8CB237
:10F7B0002A5400222046611C8CB22A540122204681
:10F7C000611C8CB22A5421462846FFF719FF0646D1
:10F7D0002046611C8CB22E5432122046611C8CB221
:10F7E0002A543C800120B3E70FB42DE9F041499F32
:10F7F000489D00240026522025F0A4FD9DF81810F5
:10F80000884204D00020BDE8F0015DF814FB45F605
:10F81000A6214A2025F0A2FD9DF818202046611C53
:10F820008CB22A549DF819202046611C8CB22A54AF
:10F83000BDF81A0002122046611C8CB22A54BDF891
:10F840001A00C2B22046611C8CB22A54BDF81C00BA
:10F8500002122046611C8CB22A54BDF81C00C2B2B0
:10F860002046611C8CB22A5400222046611C8CB2B6
:10F870002A5401222046611C8CB22A542146284673
:10F88000FFF7BEFE06462046611C8CB22E54321293
:10F890002046611C8CB22A543C800120B3E70FB48F
:10F8A0002DE9F041499F489D00240026522025F073
:10F8B00049FD9DF81810884204D00020BDE8F001F1
:10F8C0005DF814FB45F6A5214A2025F047FD9DF87B
:10F8D00018202046611C8CB22A549DF8192020461D
:10F8E000611C8CB22A54BDF81A0002122046611C19
:10F8F0008CB22A54BDF81A00C2B22046611C8CB2E8
:10F900002A54BDF81C0002122046611C8CB22A54F5
:10F91000BDF81C00C2B22046611C8CB22A540022E1
:10F920002046611C8CB22A5401222046611C8CB2F4
:10F930002A5421462846FFF763FE06462046611CEE
:10F940008CB22E5432122046611C8CB22A543C8058
:10F950000120B3E70FB42DE9F041499F489D0024F1
:10F960000026522025F0EEFC9DF81810884204D0A5
:10F970000020BDE8F0015DF814FB45F6A0214A2007
:10F9800025F0ECFC9DF818202046611C8CB22A540E
:10F990009DF819202046611C8CB22A54BDF81A002B
:10F9A00002122046611C8CB22A54BDF81A00C2B261
:10F9B0002046611C8CB22A54BDF81C00021220465D
:10F9C000611C8CB22A54BDF81C00C2B22046611CD6
:10F9D0008CB22A5400222046611C8CB22A54012287
:10F9E0002046611C8CB22A5421462846FFF708FEA7
:10F9F00006462046611C8CB22E5432122046611CF1
:10FA00008CB22A543C800120B3E700000FB42DE9EA
:10FA1000F04F2DED048B83B0DDF854B2949D00249B
:10FA20000026A146002002900190804600278246D1
:10FA30007E222146641C6A5429199DF84100FCF776
:10FA400011F8A41C29199DF84200FCF70BF8A41C1E
:10FA500029199DF84300FCF705F8A41C291900207A
:10FA6000FCF700F8A41C291900200AF02FFB241D24
:10FA700029199DF842000AF029FB241D9DF8420037
:10FA8000022807D0002003B0BDEC048BBDE8F00FC6
:10FA90005DF814FB4FF000083F2018F0D9F900F092
:10FAA000FF0ABAF1100F01DB4FF0100A2919504676
:10FAB000FBF7D8FFA01C84B200260FE0C8EB0813A8
:10FAC000684A02EBC302921C02EB46021088291915
:10FAD0000AF0FCFA201D84B2701C86B25645EDDB9C
:10FAE0004FF0060929194846FBF7BCFFA01C84B259
:10FAF00000260FE0C8EB08135A4A02EBC3026C322F
:10FB000002EB4602108829190AF0E0FA201D84B29F
:10FB1000701C86B2042EEDDB2919C8EB0813514A7C
:10FB200002EBC302B2F868000AF0D0FA201D84B2DA
:10FB30002919C8EB08134B4A02EBC302B2F866005E
:10FB40000AF0C4FA201D84B246486938D0F82A0069
:10FB500002900298F8F7F6FD41EC190B9FED420B6D
:10FB600053EC102BF8F70DFD41EC180BF8F727FEBE
:10FB700080B2291900900AF0A9FA201D84B23948F0
:10FB80006938008D00EB80004FF6FF7101EA4009F3
:10FB9000291948460AF09AFA201D84B2314869387A
:10FBA000D0F84A702919C7F30720FBF75BFFA01CA8
:10FBB00084B22919F8B2FBF755FFA01C84B22919A9
:10FBC0000320FBF74FFFA01C84B226486938D0F809
:10FBD0003E702919C7F30720FBF744FFA01C84B22D
:10FBE0002919F8B2FBF73EFFA01C84B22919C8EB13
:10FBF00008131C4A02EBC302908E0AF067FA201D1C
:10FC000084B218486938D0F83E702919C7F3072024
:10FC1000FBF728FFA01C84B22919F8B2FBF722FFDA
:10FC2000A01C84B2A4F10D0188B227F0B7FE0190A8
:10FC300005F1090101980AF049FA601E81B2681CB9
:10FC400027F0C2FE8146291948460AF03FFA201DD6
:10FC500084B20D222046611C8CB22A54ABF80040BD
:10FC6000012010E775D200209A9999999999B93F86
:10FC70000FB42DE9F04F2DED048B83B0DDF854B2B5
:10FC8000949D00240026A146002002900190804609
:10FC9000002782467E222146641C6A5429199DF859
:10FCA0004100FBF7DFFEA41C29199DF84200FBF779
:10FCB000D9FEA41C29199DF84300FBF7D3FEA41C10
:10FCC00029190020FBF7CEFEA41C291900200AF0F8
:10FCD000FDF9241D29199DF842000AF0F7F9241DA9
:10FCE0009DF8420012280BD09DF84200022807D050
:10FCF000002003B0BDEC048BBDE8F00F5DF814FBF1
:10FD00004FF000083F2018F0A3F800F0FF0ABAF106
:10FD1000100F01DB4FF0100A29195046FBF7A2FE25
:10FD2000A01C84B200260FE0C8EB08138A4A02EB3D
:10FD3000C302921C02EB4602108829190AF0C6F988
:10FD4000201D84B2701C86B25645EDDB4FF00609CB
:10FD500029194846FBF786FEA01C84B200260FE056
:10FD6000C8EB08137C4A02EBC3026C3202EB46027A
:10FD7000108829190AF0AAF9201D84B2701C86B2D5
:10FD8000042EEDDB2919C8EB0813734A02EBC302FA
:10FD9000B2F868000AF09AF9201D84B22919C8EB5C
:10FDA00008136D4A02EBC302B2F866000AF08EF93E
:10FDB000201D84B268486938D0F82A000290029861
:10FDC000F8F7C0FC41EC190B9FED640B53EC102BC2
:10FDD000F8F7D7FB41EC180BF8F7F1FC80B22919C2
:10FDE00000900AF073F9201D84B25B486938008DD9
:10FDF00000EB80004FF6FF7101EA400929194846DF
:10FE00000AF064F9201D84B253486938D0F83E00E6
:10FE100041F66411884252D929194FF6FF700AF051
:10FE200055F9201D84B229190420FBF71BFEA01CE4
:10FE300084B229194FF6FF700AF048F9201D84B2E8
:10FE40002919454A693AD08E0AF040F9201D84B23A
:10FE500041486938D0F84A0000EB80004700291972
:10FE6000C7F30740FBF7FEFDA01C84B22919C7F3B6
:10FE70000720FBF7F7FDA01C84B22919F8B2FBF7A5
:10FE8000F1FDA01C84B234486938D0F83E0000EB84
:10FE9000800047002919C7F30740FBF7E3FDA01CCA
:10FEA00084B22919C7F30720FBF7DCFDA01C84B23C
:10FEB0002919F8B2FBF7D6FDA01C84B22BE0291952
:10FEC000254A693AD2F84A2002EB82024FF6FF73C4
:10FED00003EA42000AF0FAF8201D84B22919022030
:10FEE000FBF7C0FDA01C84B229191B4A693AD2F85D
:10FEF0003E2002EB82024FF6FF7303EA42000AF053
:10FF0000E5F8201D84B22919134A693AD08E0AF007
:10FF1000DDF8201D84B2A4F10D0188B227F03EFD6A
:10FF2000019005F1090101980AF0D0F8601E81B234
:10FF3000681C27F049FD8146291948460AF0C6F891
:10FF4000201D84B20D222046611C8CB22A54ABF8CD
:10FF500000400120CDE6000075D200209A999999C1
:10FF60009999B93F0FB42DE9F04F2DED048B83B073
:10FF7000DDF854B2949D00240026A1460020029092
:10FF800001908046002782467E222146641C6A54E6
:10FF900029199DF84100FBF765FDA41C29199DF85E
:10FFA0004200FBF75FFDA41C29199DF84300FBF7F5
:10FFB00059FDA41C29190020FBF754FDA41C291984
:10FFC00000200AF083F8241D29199DF842000AF048
:10FFD0007DF8241D00BF3F2017F03AFF00F0FF0A14
:10FFE000BAF1100F01DB4FF0100A29195046FBF748
:10FFF00039FDA01C84B200260FE0C8EB08136C4A40
:020000040001F9
:1000000002EBC302921C02EB4602108829190AF087
:100010005DF8201D84B2701C86B25645EDDB4FF0B2
:10002000060929194846FBF71DFDA01C84B20026CD
:100030000FE0C8EB08135E4A02EBC3026C3202EB1E
:100040004602108829190AF041F8201D84B2701C5C
:1000500086B2042EEDDB2919C8EB0813544A02EBD3
:10006000C302B2F868000AF031F8201D84B22919E1
:10007000C8EB08134E4A02EBC302B2F866000AF05E
:1000800025F8201D84B24A486938D0F82A00029029
:100090000298F8F757FB41EC190B9FED460B53EC18
:1000A000102BF8F76EFA41EC180BF8F788FB80B2CA
:1000B000291900900AF00AF8201D84B23C486938DA
:1000C000008D00EB80004FF6FF7101EA400929190D
:1000D000484609F0FBFF201D84B235486938D0F846
:1000E0004A702919C7F30720FBF7BCFCA01C84B297
:1000F0002919F8B2FBF7B6FCA01C84B22919032019
:10010000FBF7B0FCA01C84B229486938D0F83E70D7
:100110002919C7F30720FBF7A5FCA01C84B22919F5
:10012000F8B2FBF79FFCA01C84B22919C8EB081396
:100130001F4A02EBC302908E09F0C8FF201D84B253
:100140001B486938D0F83E702919C7F30720FBF720
:1001500089FCA01C84B22919F8B2FBF783FCA01C0F
:1001600084B2A4F10D0188B227F018FC019005F1CA
:100170000901019809F0AAFF601E81B2681C27F0EE
:1001800023FC81462919484609F0A0FF201D84B2AE
:100190000D222046611C8CB22A54ABF8004001208D
:1001A00003B0BDEC048BBDE8F00F5DF814FB00005C
:1001B00075D200209A9999999999B93F0FB42DE970
:1001C000F04F2DED028B83B0DDF84CB2929D0024F0
:1001D000002700200290019000268146804682463A
:1001E0007E222146641C6A5429199DF83900FBF7C8
:1001F00039FCA41C29199DF83A00FBF733FCA41C18
:1002000029199DF83B00FBF72DFCA41C291900209F
:10021000FBF728FCA41C2919002009F057FF241D16
:1002200029199DF83A0009F051FF241D9DF83A0064
:10023000022807D0002003B0BDEC028BBDE8F00F10
:100240005DF814FB4FF000083F2017F001FE00F0AE
:10025000FF09B9F1100F01DB4FF0100929194846C9
:10026000FBF700FCA01C84B2002707E0291900203E
:10027000FBF7F8FBA01C84B2781C87B24F45F5DB76
:100280001EF042FD8246BAF1040F01DB4FF0040A72
:1002900029190AF10202D0B2FBF7E4FBA01C84B2D8
:1002A0002919C8EB08138C4A02EBC30292F86800C4
:1002B000FBF7D8FBA01C84B200270EE0C8EB0813A4
:1002C000854A02EBC3026C3212F817002919FBF7BA
:1002D000C9FBA01C84B2781C87B25745EEDB2919F4
:1002E000C8EB08137C4A02EBC30292F86600FBF7E6
:1002F000B9FBA01C84B27848693890F84E00C0F36E
:10030000001020B129190220FBF7ACFB03E02919EA
:100310000020FBF7A7FBA01C84B26F48693890F857
:100320004E00C0F3800020B129190220FBF79AFB90
:100330000FE06948693890F84E00C0F3C00020B162
:1003400029190120FBF78EFB03E029190020FBF798
:1003500089FBA01C84B26048693890F84E00C0F355
:10036000801020B129190220FBF77CFB03E029193A
:100370000020FBF777FBA01C84B2002656486938A2
:1003800090F84E00C0F3001030B95348693890F827
:100390004E00C0F3401008B146F004064E486938DC
:1003A00090F84E00C0F3801030B94B48693890F88F
:1003B0004E00C0F3C01008B146F010064648693838
:1003C000B0F84E00C0F3802008B146F02006424845
:1003D0006938B0F84E00C0F3002008B146F040067E
:1003E00029193046FBF73EFBA01C84B200263A4890
:1003F000693890F85E0000F0010008B146F004068C
:100400003548693890F85E0000F0020008B146F007
:10041000020629193046FBF725FBA01C84B20026F2
:100420002D496939D1F82A00F8F78CF941EC180BFD
:100430009FED2A0B53EC102BF8F706FA01D246F089
:10044000800625496939D1F82A00F8F77BF941EC93
:10045000180B9FED240B53EC102BF8F7DDF901D2AC
:1004600046F040061C486938408E642801D146F0A9
:10047000080629193046FBF7F5FAA01C84B22919A1
:100480000020FBF7EFFAA01C84B229190020FBF72B
:10049000E9FAA01C84B2A4F10D0188B227F07EFA1B
:1004A000019005F10901019809F010FE601E81B26A
:1004B000681C27F089FA02902919029809F006FEB3
:1004C000201D84B20D222046611C8CB22A54ABF848
:1004D00000400120AFE6000075D200209A9999995A
:1004E0009999B93F9A9999999999B9BF0FB42DE9FA
:1004F000F04F2DED028B83B0DDF84CB2929D0024BD
:100500000027002002900190002681468046824606
:100510007E222146641C6A5429199DF83900FBF794
:10052000A1FAA41C29199DF83A00FBF79BFAA41C18
:1005300029199DF83B00FBF795FAA41C2919002006
:10054000FBF790FAA41C2919002009F0BFFD241D17
:1005500029199DF83A0009F0B9FD241D00BF3F207C
:1005600017F076FC00F0FF09B9F1100F01DB4FF036
:10057000100929194846FBF775FAA01C84B2002718
:1005800007E029190020FBF76DFAA01C84B2781C43
:1005900087B24F45F5DB1EF0B7FB8246BAF1040F78
:1005A00001DB4FF0040A29190AF10202D0B2FBF76D
:1005B00059FAA01C84B22919C8EB08138E4A02EB21
:1005C000C30292F86800FBF74DFAA01C84B2002722
:1005D0000EE0C8EB0813884A02EBC3026C3212F833
:1005E00017002919FBF73EFAA01C84B2781C87B2C9
:1005F0005745EEDB2919C8EB08137F4A02EBC3020B
:1006000092F86600FBF72EFAA01C84B27A4869388B
:1006100090F84E00C0F3001020B129190220FBF71A
:1006200021FA03E029190020FBF71CFAA01C84B270
:100630007148693890F84E00C0F3800020B1291944
:100640000220FBF70FFA0FE06B48693890F84E0074
:10065000C0F3C00020B129190120FBF703FA03E021
:1006600029190020FBF7FEF9A01C84B26248693802
:1006700090F84E00C0F3801020B129190220FBF73A
:10068000F1F903E029190020FBF7ECF9A01C84B272
:1006900000265948693890F84E00C0F3001030B970
:1006A0005548693890F84E00C0F3401008B146F044
:1006B00004065148693890F84E00C0F3801030B9F4
:1006C0004D48693890F84E00C0F3C01008B146F0AC
:1006D000100649486938B0F84E00C0F3802008B1D0
:1006E00046F0200644486938B0F84E00C0F30020B8
:1006F00008B146F0400629193046FBF7B3F9A01CB3
:1007000084B200263C48693890F85E0000F0010091
:1007100008B146F004063848693890F85E0000F0E9
:10072000020008B146F0020629193046FBF79AF993
:10073000A01C84B2002630496939D1F82A00F8F7A4
:1007400001F841EC180B9FED2D0B53EC102BF8F733
:100750007BF801D246F0800627496939D1F82A0092
:10076000F7F7F0FF41EC180B9FED260B53EC102B25
:10077000F8F752F801D246F040061F486938408E1B
:10078000642801D146F0080629193046FBF76AF9BA
:10079000A01C84B229190020FBF764F9A01C84B2C4
:1007A00029190020FBF75EF9A01C84B2A4F10D0109
:1007B00088B227F0F3F8019005F10901019809F0DA
:1007C00085FC601E81B2681C27F0FEF80290291992
:1007D000029809F07BFC201D84B20D222046611C8A
:1007E0008CB22A54ABF80040012003B0BDEC028B60
:1007F000BDE8F00F5DF814FB75D200209A99999925
:100800009999B93F9A9999999999B9BF0FB42DE9D6
:10081000F04F2DED028B83B0DDF84CB2929D002499
:1008200000270020029001900026814680468246E3
:100830007E222146641C6A5429199DF83900FBF771
:1008400011F9A41C29199DF83A00FBF70BF9A41C17
:1008500029199DF83B00FBF705F9A41C2919002074
:10086000FBF700F9A41C2919002009F02FFC241D16
:1008700029199DF83A0009F029FC241D00BF3F20EA
:1008800017F0E6FA00F0FF09B9F1100F01DB4FF0A5
:10089000100929194846FBF7E5F8A01C84B2002787
:1008A00007E029190020FBF7DDF8A01C84B2781CB2
:1008B00087B24F45F5DB1EF027FA8246BAF1040FE6
:1008C00001DB4FF0040A29190AF10202D0B2FBF74A
:1008D000C9F8A01C84B22919C8EB08138E4A02EB90
:1008E000C30292F86800FBF7BDF8A01C84B2002791
:1008F0000EE0C8EB0813884A02EBC3026C3212F810
:1009000017002919FBF7AEF8A01C84B2781C87B237
:100910005745EEDB2919C8EB08137F4A02EBC302E7
:1009200092F86600FBF79EF8A01C84B27A486938FA
:1009300090F84E00C0F3001020B129190220FBF7F7
:1009400091F803E029190020FBF78CF8A01C84B271
:100950007148693890F84E00C0F3800020B1291921
:100960000220FBF77FF80FE06B48693890F84E00E3
:10097000C0F3C00020B129190120FBF773F803E090
:1009800029190020FBF76EF8A01C84B26248693870
:1009900090F84E00C0F3801020B129190220FBF717
:1009A00061F803E029190020FBF75CF8A01C84B271
:1009B00000265948693890F84E00C0F3001030B94D
:1009C0005548693890F84E00C0F3401008B146F021
:1009D00004065148693890F84E00C0F3801030B9D1
:1009E0004D48693890F84E00C0F3C01008B146F089
:1009F000100649486938B0F84E00C0F3802008B1AD
:100A000046F0200644486938B0F84E00C0F3002094
:100A100008B146F0400629193046FBF723F8A01C20
:100A200084B200263C48693890F85E0000F001006E
:100A300008B146F004063848693890F85E0000F0C6
:100A4000020008B146F0020629193046FBF70AF801
:100A5000A01C84B2002630496939D1F82A00F7F782
:100A600071FE41EC180B9FED2D0B53EC102BF7F79B
:100A7000EBFE01D246F0800627496939D1F82A00F9
:100A8000F7F760FE41EC180B9FED260B53EC102B93
:100A9000F7F7C2FE01D246F040061F486938408E83
:100AA000642801D146F0080629193046FAF7DAFF22
:100AB000A01C84B229190020FAF7D4FFA01C84B22C
:100AC00029190020FAF7CEFFA01C84B2A4F10D0171
:100AD00088B226F063FF019005F10901019809F041
:100AE000F5FA601E81B2681C26F06EFF029029198B
:100AF000029809F0EBFA201D84B20D222046611CF9
:100B00008CB22A54ABF80040012003B0BDEC028B3C
:100B1000BDE8F00F5DF814FB75D200209A99999901
:100B20009999B93F9A9999999999B9BF0FB42DE9B3
:100B3000F0478D9E8C9D00240027A0469DF8220042
:100B4000022804D00020BDE8F0075DF814FB7E22E7
:100B50002046611C8CB22A5429199DF82100FAF70D
:100B600081FFA01C84B229199DF82200FAF77AFFB0
:100B7000A01C84B229199DF82300FAF773FFA01C6A
:100B800084B229190020FAF76DFFA01C84B229193C
:100B9000002009F09BFA201D84B24A2017F058F972
:100BA0008146291909F092FA201D84B24D2017F0D0
:100BB0004FF98146291909F089FA201D84B2502085
:100BC00017F046F98146291909F080FA201D84B2F0
:100BD000782017F03DF900F6B7001FFA80F82919C0
:100BE000404609F073FA201D84B27E2017F030F9D8
:100BF00000F6B7001FFA80F82919404609F066FA96
:100C0000201D84B2622017F023F900EB80004FF61C
:100C1000FF7101EA40092919484609F057FA201DD9
:100C200084B2562017F014F900EB80004FF6FF71E4
:100C300001EA40092919484609F048FA201D84B202
:100C4000592017F005F900EB80004FF6FF7101EA1B
:100C500040092919484609F039FA201D84B25C2060
:100C600017F0F6F800EB80004FF6FF7101EA40093B
:100C70002919484609F02AFA201D84B2842017F069
:100C8000E7F800F6B7001FFA80F92919484609F07D
:100C90001DFA201D84B28A2017F0DAF800F6B7009A
:100CA0001FFA80F92919484609F010FA201D84B26C
:100CB0006D2017F0CDF8404200EB80004FF6FF7139
:100CC00001EA40092919484609F000FA201D84B2BA
:100CD000A4F10D0188B226F061FE074605F1090175
:100CE000384609F0F3F9601E81B2681C26F06CFEEC
:100CF00080462919404609F0E9F9201D84B20D22E9
:100D00002046611C8CB22A54348001201BE70FB4AA
:100D10002DE9F0478D9E8C9D00240027A0467E2261
:100D20002146641C6A5429199DF82100FAF79AFE9D
:100D3000A41C29199DF82200FAF794FEA41C291975
:100D40009DF82300FAF78EFEA41C29190020FAF75B
:100D500089FEA41C2919002009F0B8F9241D4A2095
:100D600017F076F88146291909F0B0F9241D4D20B5
:100D700017F06EF88146291909F0A8F9241D5020B2
:100D800017F066F88146291909F0A0F9241D78208A
:100D900017F05EF800F6B7001FFA80F829194046F0
:100DA00009F094F9241D7E2017F052F800F6B700E0
:100DB0001FFA80F82919404609F088F9241D62209D
:100DC00017F046F800EB80004FF6FF7101EA40098A
:100DD0002919484609F07AF9241D562017F038F8E9
:100DE00000EB80004FF6FF7101EA400929194846DF
:100DF00009F06CF9241D592017F02AF800EB800047
:100E00004FF6FF7101EA40092919484609F05EF9D9
:100E1000241D5C2017F01CF800EB80004FF6FF71DA
:100E200001EA40092919484609F050F9241D842097
:100E300017F00EF800F6B7001FFA80F92919484696
:100E400009F044F9201D84B28A2017F001F800F659
:100E5000B7001FFA80F92919484609F037F9201D13
:100E600084B26D2016F0F4FF404200EB80004FF694
:100E7000FF7101EA40092919484609F027F9201DA8
:100E800084B2A4F10D0188B226F088FD074605F171
:100E90000901384609F01AF9601E81B2681C26F073
:100EA00093FD80462919404609F010F9201D84B2AF
:100EB0000D222146601C84B26A5434800120BDE8B2
:100EC000F0075DF814FB0FB42DE9F0478D9E8C9D63
:100ED00000240027A0467E222146641C6A5429195A
:100EE0009DF82100FAF7BEFDA41C29199DF82200E7
:100EF000FAF7B8FDA41C29199DF82300FAF7B2FDF2
:100F0000A41C29190020FAF7ADFDA41C2919002002
:100F100009F0DCF8241D4A2016F09AFF81462919B1
:100F200009F0D4F8241D4D2016F092FF81462919AE
:100F300009F0CCF8241D502016F08AFF81462919AB
:100F400009F0C4F8241D782016F082FF00F6B700DF
:100F50001FFA80F82919404609F0B8F8241D7E20B0
:100F600016F076FF00F6B7001FFA80F82919404600
:100F700009F0ACF8241D622016F06AFF00EB800037
:100F80004FF6FF7101EA40092919484609F09EF819
:100F9000241D562016F05CFF00EB80004FF6FF7119
:100FA00001EA40092919484609F090F8241D592002
:100FB00016F04EFF00EB80004FF6FF7101EA40098A
:100FC0002919484609F082F8241D5C2016F040FFDC
:100FD00000EB80004FF6FF7101EA400929194846ED
:100FE00009F074F8241D842016F032FF00F6B700D3
:100FF0001FFA80F92919484609F068F8201D84B2C3
:101000008A2016F025FF00F6B7001FFA80F929198B
:10101000484609F05BF8201D84B26D2016F018FFD9
:10102000404200EB80004FF6FF7101EA40092919A8
:10103000484609F04BF8201D84B2A4F10D0188B296
:1010400026F0ACFC074605F10901384609F03EF8E8
:10105000601E81B2681C26F0B7FC80462919404604
:1010600009F034F8201D84B20D222146601C84B2A0
:101070006A5434800120BDE8F0075DF814FB0FB41A
:101080002DE9F0418B9E8A9D00240027A0469DF803
:101090001A00022804D00020BDE8F0015DF814FB1E
:1010A0007E222046611C8CB22A5429192020FAF78E
:1010B000D9FCA01C84B229199DF81A00FAF7D2FCB9
:1010C000A01C84B229199DF81B00FAF7CBFCA01CC8
:1010D00084B229190020FAF7C5FCA01C84B2291992
:1010E000002008F0F3FF201D84B2A4F10D0188B2A6
:1010F00026F054FC074605F10901384608F0E6FFE2
:10110000601E81B2681C26F05FFC804629194046AB
:1011100008F0DCFF201D84B20D222146601C84B241
:101120006A5434800120B7E70FB42DE9F0418B9E5B
:101130008A9D00240027A0467E222146641C6A5412
:1011400029192020FAF78EFCA41C29199DF81A00F1
:10115000FAF788FCA41C29199DF81B00FAF782FCF9
:10116000A41C29190020FAF77DFCA41C29190020D1
:1011700008F0ACFF241DA4F10D0188B226F00EFC8E
:10118000074605F10901384608F0A0FF601E81B24C
:10119000681C26F019FC80462919404608F096FF85
:1011A000241D0D222146641C6A5434800120BDE8B0
:1011B000F0015DF814FB0FB42DE9F0418B9E8A9D80
:1011C00000240027A0467E222146641C6A54291967
:1011D0002020FAF747FCA41C29199DF81A00FAF7F9
:1011E00041FCA41C29199DF81B00FAF73BFCA41C28
:1011F00029190020FAF736FCA41C2919002008F050
:1012000065FF241DA4F10D0188B226F0C7FB074637
:1012100005F10901384608F059FF601E81B2681CCB
:1012200026F0D2FB80462919404608F04FFF241DC6
:101230000D222146641C6A5434800120BDE8F0016F
:101240005DF814FB0FB42DE9F0438DB0999F989D84
:101250000024A046A14614223C4908A8F7F7B6F896
:1012600020223A4914316846F7F7B0F800269DF875
:101270005200022805D000200DB0BDE8F0035DF853
:1012800014FB7E222046611C8CB22A5429199DF839
:101290005100FAF7E7FBA01C84B229199DF852000F
:1012A000FAF7E0FBA01C84B229199DF85300FAF765
:1012B000D9FBA01C84B229190020FAF7D3FBA01C8B
:1012C00084B22919002008F001FF201D84B20026F5
:1012D00008E0291908AA905DFAF7C4FBA01C84B2A3
:1012E000701CC6B20A2EF4DB2919002008F0EEFEAD
:1012F000201D84B2002608E029191DF80600FAF71F
:10130000B1FBA01C84B2701CC6B2142EF4DBA4F195
:101310000D0188B226F042FB804605F109014046E6
:1013200008F0D4FE601E81B2681C26F04DFB814699
:101330002919484608F0CAFE201D84B20D22204615
:10134000611C8CB22A543C80012095E78C860300F6
:101350000FB42DE9F0438DB0999F989D0024A046CD
:10136000A1461422364908A8F7F730F8202234495C
:1013700014316846F7F72AF800267E222146641CBD
:101380006A5429199DF85100FAF76CFBA41C29191D
:101390009DF85200FAF766FBA41C29199DF853002A
:1013A000FAF760FBA41C29190020FAF75BFBA41CC8
:1013B0002919002008F08AFE241D00BF08E0291921
:1013C00008AA905DFAF74EFBA01C84B2701CC6B24E
:1013D0000A2EF4DB2919002008F078FE201D84B2C3
:1013E000002608E029191DF80600FAF73BFBA01CAF
:1013F00084B2701CC6B2142EF4DBA4F10D0188B2C5
:1014000026F0CCFA804605F10901404608F05EFE60
:10141000601E81B2681C26F0D7FA81462919484619
:1014200008F054FE201D84B20D222046611C8CB2AF
:101430002A543C8001200DB0BDE8F0035DF814FB98
:10144000CC8603000FB42DE9F0438DB0999F989D91
:101450000024A046A1461422364908A8F6F7B6FF94
:101460002022344914316846F6F7B0FF00267E2268
:101470002146641C6A5429199DF85100FAF7F2FAC2
:10148000A41C29199DF85200FAF7ECFAA41C29199A
:101490009DF85300FAF7E6FAA41C29190020FAF780
:1014A000E1FAA41C2919002008F010FE241D00BF39
:1014B00008E0291908AA905DFAF7D4FAA01C84B2B2
:1014C000701CC6B20A2EF4DB2919002008F0FEFDBC
:1014D000201D84B2002608E029191DF80600FAF73D
:1014E000C1FAA01C84B2701CC6B2142EF4DBA4F1A5
:1014F0000D0188B226F052FA804605F109014046F6
:1015000008F0E4FD601E81B2681C26F05DFA814699
:101510002919484608F0DAFD201D84B20D22204624
:10152000611C8CB22A543C8001200DB0BDE8F00350
:101530005DF814FB888903000FB42DE9FF5FDDF827
:101540004C92929D0024A24600200390604AD2E96A
:1015500000109268CDE9010200910026A346A04642
:1015600000279DF83A00022805D0002004B0BDE80D
:10157000F01F5DF814FB7E222046611C8CB22A54B9
:1015800029199DF83900FAF76DFAA01C84B22919BF
:101590009DF83A00FAF766FAA01C84B229199DF862
:1015A0003B00FAF75FFAA01C84B229190020FAF771
:1015B00059FAA01C84B22919002008F087FD201DCB
:1015C00084B2002608E029191DF80600FAF74AFA45
:1015D000A01C84B2701CC6B20A2EF4DB002612E0F6
:1015E00006F1EC0016F034FC07462919F8B2FAF7B8
:1015F00039FAA01C84B229193812FAF733FAA01C60
:1016000084B2701CC6B20A2EEADB29190D20FAF743
:1016100029FAA01C84B229190220FAF723FAA01C87
:1016200084B229192B4A9078FAF71CFAA01C84B2CC
:10163000D52023F087FE8346002626E00120B04017
:1016400000EA0B00F8B14FF0000819E0C6EB0611F4
:101650002048693000EBC100423000EB48000788A9
:101660002919F8B2FAF7FEF9A01C84B22919381228
:10167000FAF7F8F9A01C84B208F1010000F0FF08A5
:10168000B8F1080FE2DB701CC6B2202ED6DBA4F145
:101690000D0188B226F082F9824605F10901504613
:1016A00008F014FD601E81B2681C26F08DF90390CD
:1016B0002919039808F00AFD201D84B20D22204646
:1016C000611C8CB22A54A9F8004001204EE70000AA
:1016D000C08603000CD200200FB42DE9FF5FDDF8B7
:1016E0004C92929D0024A246002003905A4AD2E9CF
:1016F00000109268CDE9010200910026A346A046A1
:1017000000277E222146641C6A5429199DF839005D
:10171000FAF7A8F9A41C29199DF83A00FAF7A2F9DA
:10172000A41C29199DF83B00FAF79CF9A41C29195F
:101730000020FAF797F9A41C2919002008F0C6FC2C
:10174000241D00BF08E029191DF80600FAF78AF9E0
:10175000A01C84B2701CC6B20A2EF4DB002612E074
:1017600006F1EC0016F074FB07462919F8B2FAF7F7
:1017700079F9A01C84B229193812FAF773F9A01C60
:1017800084B2701CC6B20A2EEADB29190D20FAF7C2
:1017900069F9A01C84B229190220FAF763F9A01C88
:1017A00084B229192D4A9078FAF75CF9A01C84B20A
:1017B000D52023F0C7FD8346002626E00120B04057
:1017C00000EA0B00F8B14FF0000819E0C6EB061173
:1017D0002248693000EBC100423000EB4800078826
:1017E0002919F8B2FAF73EF9A01C84B22919381267
:1017F000FAF738F9A01C84B208F1010000F0FF08E4
:10180000B8F1080FE2DB701CC6B2202ED6DBA4F1C3
:101810000D0188B226F0C2F8824605F10901504652
:1018200008F054FC601E81B2681C26F0CDF80390CD
:101830002919039808F04AFC201D84B20D22204685
:10184000611C8CB22A54A9F80040012004B0BDE804
:10185000F01F5DF814FB0000008703000CD200208D
:101860000FB42DE9FF5FDDF84C92929D0024A24653
:10187000002003905A4AD2E900109268CDE9010293
:1018800000910026A346A04600277E222146641C24
:101890006A5429199DF83900FAF7E4F8A41C2919AB
:1018A0009DF83A00FAF7DEF8A41C29199DF83B00D0
:1018B000FAF7D8F8A41C29190020FAF7D3F8A41CC9
:1018C0002919002008F002FC241D00BF08E0291996
:1018D0001DF80600FAF7C6F8A01C84B2701CC6B248
:1018E0000A2EF4DB002612E006F1EC0016F0B0FA46
:1018F00007462919F8B2FAF7B5F8A01C84B22919DD
:101900003812FAF7AFF8A01C84B2701CC6B20A2EC7
:10191000EADB29190D20FAF7A5F8A01C84B22919D1
:101920000220FAF79FF8A01C84B229192D4A90785A
:10193000FAF798F8A01C84B2D52023F003FD834663
:10194000002626E00120B04000EA0B00F8B14FF07D
:10195000000819E0C6EB06112248693000EBC1000F
:10196000423000EB480007882919F8B2FAF77AF8F4
:10197000A01C84B229193812FAF774F8A01C84B29A
:1019800008F1010000F0FF08B8F1080FE2DB701C5D
:10199000C6B2202ED6DBA4F10D0188B225F0FEFFE1
:1019A000824605F10901504608F090FB601E81B2A5
:1019B000681C26F009F803902919039808F086FBA3
:1019C000201D84B20D222046611C8CB22A54A9F835
:1019D0000040012004B0BDE8F01F5DF814FB0000DA
:1019E000BC8903000CD200200FB42DE9F047DDF8CC
:1019F00034828C9D0024A146002600279DF82200F9
:101A0000022804D00020BDE8F0075DF814FB7E2218
:101A10002046611C8CB22A5429199DF82100FAF73E
:101A200021F8A01C84B229199DF82200FAF71AF8AF
:101A3000A01C84B229199DF82300FAF713F8A01C02
:101A400084B229190020FAF70DF8A01C84B22919D4
:101A5000002008F03BFB201D84B2F22023F072FC32
:101A600000EB80004FF6FF7101EA400A2919504649
:101A700008F02CFB201D84B28448408D06B2291941
:101A8000B0B208F023FB201D84B2D02023F05AFC12
:101A900000F0FF0A29195046F9F7E4FFA01C84B2B0
:101AA000F32023F04FFC8246291908F00FFB201D7C
:101AB00084B2F42023F046FC8246291908F006FB84
:101AC000201D84B2E12023F03DFC0746642F00DB9B
:101AD00064272919F8B2F9F7C5FFA01C84B2F520D4
:101AE00023F030FC00F0FF0A29195046F9F7BAFF3D
:101AF000A01C84B2DA2023F025FC8246291908F0C4
:101B0000E5FA201D84B2D92023F01CFC8246291955
:101B100008F0DCFA201D84B2DC2023F013FC82469E
:101B2000291908F0D3FA201D84B2DB2023F00AFC27
:101B30008246291908F0CAFA201D84B2F62023F043
:101B400001FC8246291908F0C1FA201D84B2DE206A
:101B500023F0F8FB8246291908F0B8FA201D84B258
:101B6000DD2023F0EFFB8246291908F0AFFA201D93
:101B700084B2E02023F0E6FB8246291908F0A6FA99
:101B8000201D84B2DF2023F0DDFB8246291908F0F6
:101B90009DFA201D84B2F72023F0D4FB8246291938
:101BA00008F094FA201D84B2F92023F0CBFB824682
:101BB000291908F08BFA201D84B2F82023F0C2FB0B
:101BC0008246291908F082FA201D84B2FB2023F0F6
:101BD000B9FB8246291908F079FA201D84B2FA204F
:101BE00023F0B0FB8246291908F070FA201D84B258
:101BF000FC2023F0A7FB8246291908F067FA201D74
:101C000084B2FE2023F09EFB8246291908F05EFA7A
:101C1000201D84B2FD2023F095FB8246291908F08F
:101C200055FA201D84B24FF4807023F08BFB82465E
:101C3000291908F04BFA201D84B2FF2023F082FB03
:101C40008246291908F042FA201D84B2A4F10D0140
:101C500088B225F0A3FE814605F10901484608F047
:101C600035FA601E81B2681C25F0AEFE06B2291955
:101C7000B0B208F02BFA201D84B20D222046611C60
:101C80008CB22A54A8F800400120BCE60CD20020F7
:101C90000FB42DE9F047DDF834828C9D0024A14675
:101CA000002600277E222146641C6A5429199DF8CB
:101CB0002100F9F7D7FEA41C29199DF82200F9F795
:101CC000D1FEA41C29199DF82300F9F7CBFEA41C12
:101CD00029190020F9F7C6FEA41C2919002008F0D4
:101CE000F5F9241DF22023F02DFB00EB80004FF6C8
:101CF000FF7101EA400A2919504608F0E7F9241D4E
:101D00008448408D06B22919B0B208F0DFF9241DCD
:101D1000D02023F017FB00F0FF0A29195046F9F7ED
:101D2000A1FEA41CF32023F00DFB8246291908F024
:101D3000CDF9241DF42023F005FB8246291908F073
:101D4000C5F9241DE12023F0FDFA0746642F00DBCE
:101D500064272919F8B2F9F785FEA01C84B2F52092
:101D600023F0F0FA00F0FF0A29195046F9F77AFE3D
:101D7000A01C84B2DA2023F0E5FA8246291908F083
:101D8000A5F9201D84B2D92023F0DCFA8246291956
:101D900008F09CF9201D84B2DC2023F0D3FA82469F
:101DA000291908F093F9201D84B2DB2023F0CAFA28
:101DB0008246291908F08AF9201D84B2F62023F002
:101DC000C1FA8246291908F081F9201D84B2DE206B
:101DD00023F0B8FA8246291908F078F9201D84B258
:101DE000DD2023F0AFFA8246291908F06FF9201D93
:101DF00084B2E02023F0A6FA8246291908F066F999
:101E0000201D84B2DF2023F09DFA8246291908F0B4
:101E10005DF9201D84B2F72023F094FA8246291937
:101E200008F054F9201D84B2F92023F08BFA824681
:101E3000291908F04BF9201D84B2F82023F082FA0A
:101E40008246291908F042F9201D84B2FB2023F0B4
:101E500079FA8246291908F039F9201D84B2FA204E
:101E600023F070FA8246291908F030F9201D84B257
:101E7000FC2023F067FA8246291908F027F9201D73
:101E800084B2FE2023F05EFA8246291908F01EF97A
:101E9000201D84B2FD2023F055FA8246291908F04E
:101EA00015F9201D84B24FF4807023F04BFA82465E
:101EB000291908F00BF9201D84B2FF2023F042FA03
:101EC0008246291908F002F9201D84B2A4F10D01FF
:101ED00088B225F063FD814605F10901484608F006
:101EE000F5F8601E81B2681C25F06EFD06B2291956
:101EF000B0B208F0EBF8201D84B20D222046611C20
:101F00008CB22A54A8F800400120BDE8F0075DF823
:101F100014FB00000CD200200FB42DE9F047DDF8CF
:101F200034828C9D0024A146002600277E22214673
:101F3000641C6A5429199DF82100F9F793FDA41C2B
:101F400029199DF82200F9F78DFDA41C29199DF887
:101F50002300F9F787FDA41C29190020F9F782FD59
:101F6000A41C2919002008F0B1F8241DF22023F048
:101F7000E9F900EB80004FF6FF7101EA400A2919E8
:101F8000504608F0A3F8241D8448408D06B2291954
:101F9000B0B208F09BF8241DD02023F0D3F900F054
:101FA000FF0A29195046F9F75DFDA41CF32023F020
:101FB000C9F98246291908F089F8241DF42023F074
:101FC000C1F98246291908F081F8241DE12023F087
:101FD000B9F90746642F00DB64272919F8B2F9F72D
:101FE00041FDA01C84B2F52023F0ACF900F0FF0AFB
:101FF00029195046F9F736FDA01C84B2DA2023F0E7
:10200000A1F98246291908F061F8201D84B2D9206F
:1020100023F098F98246291908F058F8201D84B257
:10202000DC2023F08FF98246291908F04FF8201D93
:1020300084B2DB2023F086F98246291908F046F89D
:10204000201D84B2F62023F07DF98246291908F07C
:102050003DF8201D84B2DE2023F074F98246291950
:1020600008F034F8201D84B2DD2023F06BF982469D
:10207000291908F02BF8201D84B2E02023F062F922
:102080008246291908F022F8201D84B2DF2023F0AF
:1020900059F98246291908F019F8201D84B2F72051
:1020A00023F050F98246291908F010F8201D84B257
:1020B000F92023F047F98246291908F007F8201D76
:1020C00084B2F82023F03EF98246291907F0FEFF7A
:1020D000201D84B2FB2023F035F98246291907F030
:1020E000F5FF201D84B2FA2023F02CF9824629192D
:1020F00007F0ECFF201D84B2FC2023F023F9824678
:10210000291907F0E3FF201D84B2FE2023F01AF9FD
:102110008246291907F0DAFF201D84B2FD2023F042
:1021200011F98246291907F0D1FF201D84B24FF41E
:10213000807023F007F98246291907F0C7FF201D98
:1021400084B2FF2023F0FEF88246291907F0BEFF73
:10215000201D84B2A4F10D0188B225F01FFC814638
:1021600005F10901484607F0B1FF601E81B2681C05
:1021700025F02AFC06B22919B0B207F0A7FF201DEE
:1021800084B20D222046611C8CB22A54A8F800406B
:102190000120BDE8F0075DF814FB00000CD2002020
:1021A0000FB42DE9F047DDF834828C9D0024A14660
:1021B00000260027A2469DF82200022804D0002015
:1021C000BDE8F0075DF814FB7E222046611C8CB24E
:1021D0002A5429199DF82100F9F744FCA01C84B267
:1021E00029199DF82200F9F73DFCA01C84B2291999
:1021F0009DF82300F9F736FCA01C84B229190020B1
:10220000F9F730FCA01C84B22919002007F05EFF0A
:10221000201D84B206F072FA06462919F0B2F9F7C9
:1022200021FCA01C84B229193012F9F71BFCA01C58
:1022300084B206F045FE07462919F8B2F9F712FCF8
:10224000A01C84B229193812F9F70CFCA01C84B226
:10225000A4F10D0188B225F0A1FB814605F1090129
:10226000484607F033FF601E81B2681C25F0ACFBC6
:1022700082462919504607F029FF201D84B20D22FD
:102280002046611C8CB22A54A8F80040012097E730
:102290000FB42DE9F047DDF834828C9D0024A1466F
:1022A00000260027A2467E222146641C6A54291972
:1022B0009DF82100F9F7D6FBA41C29199DF82200EE
:1022C000F9F7D0FBA41C29199DF82300F9F7CAFBE4
:1022D000A41C29190020F9F7C5FBA41C291900200A
:1022E00007F0F4FE241D06F00BFA06462919F0B299
:1022F000F9F7B8FBA41C29193012F9F7B3FBA41C99
:1023000006F04EFE07462919F8B2F9F7ABFBA41CFC
:1023100029193812F9F7A6FBA41CA4F10D0188B203
:1023200025F03CFB814605F10901484607F0CEFE49
:10233000601E81B2681C25F047FB82462919504671
:1023400007F0C4FE241D0D222146641C6A54A8F81F
:1023500000400120BDE8F0075DF814FB0FB42DE943
:10236000F047DDF834828C9D0024A146002600272A
:10237000A2467E222146641C6A5429199DF8210038
:10238000F9F770FBA41C29199DF82200F9F76AFBE4
:10239000A41C29199DF82300F9F764FBA41C291932
:1023A0000020F9F75FFBA41C2919002007F08EFE1E
:1023B000241D06F0ABF9064629193012F9F752FB35
:1023C000A41C2919F0B2F9F74DFBA41C06F01EFE5F
:1023D000074629193812F9F745FBA41C2919F8B248
:1023E000F9F740FBA41CA4F10D0188B225F0D6FA40
:1023F000814605F10901484607F068FE601E81B27A
:10240000681C25F0E1FA82462919504607F05EFE65
:10241000241D0D222146641C6A54A8F800400120A6
:10242000BDE8F0075DF814FB0FB42DE9F0478D9F70
:102430008C9D00240026A046A1469DF8220002287B
:1024400004D00020BDE8F0075DF814FB7E22204692
:10245000611C8CB22A5429199DF82100F9F702FB5E
:10246000A01C84B229199DF82200F9F7FBFAA01CE0
:1024700084B229199DF82300F9F7F4FAA01C84B25C
:1024800029190020F9F7EEFAA01C84B229190020BE
:1024900007F01CFE201D84B2D32022F053FF00EB76
:1024A000C00101EB00104FF6FF7101EA800A291903
:1024B000504607F00BFE201D84B2D42022F042FFCC
:1024C00000EBC00101EB00104FF6FF7101EA800A3A
:1024D0002919504607F0FAFD201D84B2D12022F0C0
:1024E00031FF8246291907F0F1FD201D84B2D22068
:1024F00022F028FF8246291907F0E8FD201D84B24A
:102500000026002013F03AFD08B146F080060120B5
:1025100013F034FD08B146F04006022013F02EFD02
:1025200018B9032013F02AFD08B146F02006532005
:1025300022F008FF08B146F0100629193046F9F7D5
:1025400091FAA01C84B2A4F10D0188B225F026FAFC
:10255000804605F10901404607F0B8FD601E81B2D2
:10256000681C25F031FA81462919484607F0AEFD6E
:10257000201D84B20D222046611C8CB22A543C805E
:1025800001205FE70FB42DE9F0478D9F8C9D00245B
:1025900000BFA046A1467E222146641C6A54291928
:1025A0009DF82100F9F75EFAA41C29199DF8220074
:1025B000F9F758FAA41C29199DF82300F9F752FAE3
:1025C000A41C29190020F9F74DFAA41C2919002090
:1025D00007F07CFD241DD32022F0B4FE00EBC001E7
:1025E00001EB00104FF6FF7101EA800A29195046ED
:1025F00007F06CFD241DD42022F0A4FE00EBC001E6
:1026000001EB00104FF6FF7101EA800A29195046CC
:1026100007F05CFD241DD12022F094FE824629198A
:1026200007F054FD241DD22022F08CFE8246291989
:1026300007F04CFD241D0026002013F09FFC08B17C
:1026400046F08006012013F099FC08B146F04006E0
:10265000022013F093FC18B9032013F08FFC08B18B
:1026600046F02006532022F06DFE08B146F0100619
:1026700029193046F9F7F6F9A01C84B2A4F10D012E
:1026800088B225F08BF9804605F10901404607F034
:102690001DFD601E81B2681C25F096F9814629193E
:1026A000484607F013FD201D84B20D222046611C10
:1026B0008CB22A543C800120BDE8F0075DF814FB81
:1026C0000FB42DE9F0478D9F8C9D002400BFA046DC
:1026D000A1467E222146641C6A5429199DF82100D6
:1026E000F9F7C0F9A41C29199DF82200F9F7BAF9E5
:1026F000A41C29199DF82300F9F7B4F9A41C291981
:102700000020F9F7AFF9A41C2919002007F0DEFC1E
:10271000241DD32022F016FE00EBC00101EB0010B7
:102720004FF6FF7101EA800A2919504607F0CEFCE6
:10273000241DD42022F006FE00EBC00101EB0010A6
:102740004FF6FF7101EA800A2919504607F0BEFCD6
:10275000241DD12022F0F6FD8246291907F0B6FC8F
:10276000241DD22022F0EEFD8246291907F0AEFC8E
:10277000241D0026002013F001FC08B146F080065D
:10278000012013F0FBFB08B146F04006022013F0D5
:10279000F5FB18B9032013F0F1FB08B146F0200651
:1027A000532022F0CFFD08B146F01006291930461B
:1027B000F9F758F9A01C84B2A4F10D0188B225F0F4
:1027C000EDF8804605F10901404607F07FFC601EE8
:1027D00081B2681C25F0F8F881462919484607F0AF
:1027E00075FC201D84B20D222046611C8CB22A5437
:1027F0003C800120BDE8F0075DF814FB0FB42DE923
:10280000F0418B9E8A9D00240027A0467E2221460F
:10281000641C6A5429199DF81900F9F723F9A41CBE
:1028200029199DF81A00F9F71DF9A41C29199DF81A
:102830001B00F9F717F9A41C29190020F9F712F960
:10284000A41C2919002007F041FC241D29199DF81A
:102850001A00F9F707F9A41CA4F10D0188B225F0BC
:102860009DF8074605F10901384607F02FFC601E68
:1028700081B2681C25F0A8F880462919404607F067
:1028800025FC241D0D222146641C6A54348001203D
:10289000BDE8F0015DF814FB0FB42DE9F0478D9F02
:1028A0008C9D00240026A046A1469DF82200022807
:1028B00004D00020BDE8F0075DF814FB7E2220461E
:1028C000611C8CB22A5429199DF82100F9F7CAF825
:1028D000A01C84B229199DF82200F9F7C3F8A01CA6
:1028E00084B229199DF82300F9F7BCF8A01C84B222
:1028F00029190020F9F7B6F8A01C84B22919002084
:1029000007F0E4FB201D84B229199DF82200F9F795
:10291000A9F8A01C84B2D32022F014FD00EBC00162
:1029200001EB00104FF6FF7101EA800A29195046A9
:1029300007F0CCFB201D84B2D42022F003FD00EB75
:10294000C00101EB00104FF6FF7101EA800A29195E
:10295000504607F0BBFB201D84B2D12022F0F2FCD0
:102960008246291907F0B2FB201D84B2D22022F042
:10297000E9FC40421FFA80FA2919504607F0A6FBED
:10298000201D84B2002013F0F9FA08B146F0800649
:10299000012013F0F3FA08B146F04006022013F0CC
:1029A000EDFA08B146F02006032013F0E7FA08B16B
:1029B00046F01006532022F0C5FC08B146F0080688
:1029C00029193046F9F74EF8A01C84B2A4F10D0184
:1029D00088B224F0E3FF804605F10901404607F084
:1029E00075FB601E81B2681C24F0EEFF8146291938
:1029F000484607F06BFB201D84B20D222046611C67
:102A00008CB22A543C80012054E70FB42DE9F047E2
:102A10008D9F8C9D00240026A046A1467E22214643
:102A2000641C6A5429199DF82100F9F71BF8A41CAD
:102A300029199DF82200F9F715F8A41C29199DF809
:102A40002300F9F70FF8A41C29190020F9F70AF858
:102A5000A41C2919002007F039FB241D29199DF811
:102A60002200F8F7FFFFA41CD32022F06BFC00EB40
:102A7000C00101EB00104FF6FF7101EA800A29192D
:102A8000504607F023FB241DD42022F05BFC00EB12
:102A9000C00101EB00104FF6FF7101EA800A29190D
:102AA000504607F013FB241DD12022F04BFC824638
:102AB000291907F00BFB241DD22022F043FC4042D1
:102AC0001FFA80FA2919504607F000FB241D002048
:102AD00013F054FA08B146F08006012013F04EFAC4
:102AE00008B146F04006022013F048FA08B146F05B
:102AF0002006032013F042FA08B146F010065320D6
:102B000022F020FC08B146F0080629193046F8F7F3
:102B1000A9FFA01C84B2A4F10D0188B224F03EFFED
:102B2000804605F10901404607F0D0FA601E81B2E7
:102B3000681C24F049FF81462919484607F0C6FA67
:102B4000201D84B20D222046611C8CB22A543C8088
:102B50000120BDE8F0075DF814FB0FB42DE9F04744
:102B60008D9F8C9D00240026A046A1467E222146F2
:102B7000641C6A5429199DF82100F8F773FFA41CFE
:102B800029199DF82200F8F76DFFA41C29199DF85A
:102B90002300F8F767FFA41C29190020F8F762FF4B
:102BA000A41C2919002007F091FA241D29199DF869
:102BB0002200F8F757FFA41CD32022F0C3FB00EB40
:102BC000C00101EB00104FF6FF7101EA800A2919DC
:102BD000504607F07BFA241DD42022F0B3FB00EB13
:102BE000C00101EB00104FF6FF7101EA800A2919BC
:102BF000504607F06BFA241DD12022F0A3FB824639
:102C0000291907F063FA241DD22022F09BFB4042D1
:102C10001FFA80FA2919504607F058FA241D00209F
:102C200013F0ACF908B146F08006012013F0A6F9C4
:102C300008B146F04006022013F0A0F908B146F0B2
:102C40002006032013F09AF908B146F0100653202D
:102C500022F078FB08B146F0080629193046F8F74B
:102C600001FFA01C84B2A4F10D0188B224F096FEED
:102C7000804605F10901404607F028FA601E81B23E
:102C8000681C24F0A1FE81462919484607F01EFA67
:102C9000201D84B20D222046611C8CB22A543C8037
:102CA0000120BDE8F0075DF814FB0FB42DE9F047F3
:102CB000DDF834828C9D0024A146002600279DF873
:102CC0002200022804D00020BDE8F0075DF814FBC4
:102CD0007E222046611C8CB22A5429199DF82100BD
:102CE000F8F7C0FEA01C84B229199DF82200F8F75D
:102CF000B9FEA01C84B229199DF82300F8F7B2FE92
:102D0000A01C84B229190020F8F7ACFEA01C84B2E4
:102D10002919002007F0DAF9201D84B229199DF83D
:102D20002200F8F79FFEA01C84B2002713E007F1F1
:102D3000DA0188B215F08CF806462919F0B2F8F7D6
:102D400091FEA01C84B229193012F8F78BFEA01C4A
:102D500084B2781C87B2082FE9DBA4F10D0188B298
:102D600024F01CFE814605F10901484607F0AEF942
:102D7000601E81B2681C24F027FE064629193046E1
:102D800007F0A4F9201D84B20D222046611C8CB2EC
:102D90002A54A8F80040012096E70FB42DE9F04727
:102DA000DDF834828C9D0024A146002600277E2277
:102DB0002146641C6A5429199DF82100F8F752FE37
:102DC000A41C29199DF82200F8F74CFEA41C29190F
:102DD0009DF82300F8F746FEA41C29190020F8F7F7
:102DE00041FEA41C2919002007F070F9241D29199F
:102DF0009DF82200F8F736FEA41C00BF13E007F18F
:102E0000DA0188B215F024F806462919F0B2F8F76D
:102E100029FEA01C84B229193012F8F723FEA01C49
:102E200084B2781C87B2082FE9DBA4F10D0188B2C7
:102E300024F0B4FD814605F10901484607F046F942
:102E4000601E81B2681C24F0BFFD06462919304679
:102E500007F03CF9201D84B20D222046611C8CB283
:102E60002A54A8F800400120BDE8F0075DF814FBE3
:102E70000FB42DE9F047DDF834828C9D0024A14683
:102E8000002600277E222146641C6A5429199DF8D9
:102E90002100F8F7E7FDA41C29199DF82200F8F796
:102EA000E1FDA41C29199DF82300F8F7DBFDA41C03
:102EB00029190020F8F7D6FDA41C2919002007F0D5
:102EC00005F9241D29199DF82200F8F7CBFDA41C53
:102ED00000BF13E007F1DA0188B214F0B9FF06462B
:102EE0002919F0B2F8F7BEFDA01C84B229193012DE
:102EF000F8F7B8FDA01C84B2781C87B2082FE9DB74
:102F0000A4F10D0188B224F049FD814605F10901C3
:102F1000484607F0DBF8601E81B2681C24F054FDBF
:102F200006462919304607F0D1F8201D84B20D223B
:102F30002046611C8CB22A54A8F800400120BDE84C
:102F4000F0075DF814FB30B5849D839C012030BDF3
:102F500030B5849D839C012030BD30B5849D839C19
:102F6000012030BD30B5849D839C012030BD30B53B
:102F7000849D839C012030BD30B5849D839C0120BD
:102F800030BD0FB42DE9F0478D9E8C9D00240027A5
:102F9000A0467E222146641C6A5429199DF821000E
:102FA000F8F760FDA41C29199DF82200F8F75AFDD6
:102FB000A41C29199DF82300F8F754FDA41C291915
:102FC0000020F8F74FFDA41C2919002007F07EF817
:102FD000241D29199DF82200F8F744FDA41C9DF832
:102FE0002200022804D00020BDE8F0075DF814FBA1
:102FF00029190220F8F736FDA01C84B229190420F3
:10300000F8F730FDA01C84B229190D20F8F72AFD2D
:10301000A01C84B20220F8F719FD1FFA80F92919C3
:10302000484607F053F8201D84B2A4F10D0188B280
:1030300024F0B4FC074605F10901384607F046F8CC
:10304000601E81B2681C24F0BFFC804629194046EE
:1030500007F03CF8201D84B20D222146601C84B28A
:103060006A5434800120BFE70FB42DE9F0478D9EEC
:103070008C9D00240027A0467E222146641C6A54B1
:1030800029199DF82100F8F7EDFCA41C29199DF8D9
:103090002200F8F7E7FCA41C29199DF82300F8F793
:1030A000E1FCA41C29190020F8F7DCFCA41C291958
:1030B000002007F00BF8241D29199DF82200F8F7CD
:1030C000D1FCA41C29190220F8F7CCFCA41C291956
:1030D0000420F8F7C7FCA41C29190D20F8F7C2FC3E
:1030E000A41C0220F8F7B2FC1FFA80F929194846FF
:1030F00006F0ECFF241DA4F10D0188B224F04EFC73
:10310000074605F10901384606F0E0FF601E81B26E
:10311000681C24F059FC80462919404606F0D6FF69
:10312000241D0D222146641C6A5434800120BDE810
:10313000F0075DF814FB0FB42DE9F0478D9E8C9DD0
:1031400000240027A0467E222146641C6A542919C7
:103150009DF82100F8F786FCA41C29199DF822008F
:10316000F8F780FCA41C29199DF82300F8F77AFCD5
:10317000A41C29190020F8F775FCA41C29190020AB
:1031800006F0A4FF241D29199DF82200F8F76AFC17
:10319000A41C29190220F8F765FCA41C2919042095
:1031A000F8F760FCA41C29190D20F8F75BFCA41C9F
:1031B0000220F8F74BFC1FFA80F92919484606F05F
:1031C00085FF241DA4F10D0188B224F0E7FB07461A
:1031D00005F10901384606F079FF601E81B2681CCE
:1031E00024F0F2FB80462919404606F06FFF241DAB
:1031F0000D222146641C6A5434800120BDE8F0078A
:103200005DF814FB08B500200090694661200EF0BF
:1032100046FABDF8000000F0040048B1002017494C
:103220000870BDF8001061200EF0D0FA012008BD32
:1032300012480078401C11490870084600780A2896
:1032400019DB0020009047F2177156200EF0BEFAED
:1032500012215A200EF0BAFA072158200EF0B6FAC1
:10326000D82130200EF0B2FA002156200EF0AEFA2E
:103270000020024908700020D9E700001401002056
:1032800010B500240EF09EF90446204610BD000043
:1032900010B500240EF0AFF9012803D102480EF05A
:1032A000EBF80446204610BD1001002070B504461E
:1032B0000D460026294620460DF014FF06463046EE
:1032C00070BD70B504460D460026294620460EF016
:1032D00039F80646304670BD70B504460D460026E6
:1032E000294620460EF0C0F90646304670BD000063
:1032F0002DE9F0432DED048B81B006460F464FF0CB
:103300000009C846002000900024002500BF38E0D6
:10331000694653200EF0C3F98146B9F1010F2CD153
:10332000BDF800008513681C4400BDF8000000F0E3
:103330000F05681C14FB00F000EB8000400000EE5D
:10334000100AB8EEC00ADFED140A80EE201ABCEEB7
:10335000C10A10EE100A3080BDF80000C0F303155A
:10336000681CF5F7EFF99FED0D0B53EC102BF5F7FB
:1033700008F9F5F724FA388006E008F1010000F0BA
:10338000FF08B8F1030FC3DB00BF484601B0BDEC36
:10339000048BBDE8F0830000AB3E573E0000000008
:1033A00000404F4010B504460DF0E8FF10BD00008E
:1033B00070B50446002504480EF05EF80546024844
:1033C00000682060284670BD1001002070B50446DA
:1033D000002520460EF022F90546284670BD000063
:1033E00002480088C0F34020704700001001002010
:1033F00038B5002400200090694657200EF04FF9A0
:103400000446012C08D1BDF8000000F0800008B986
:10341000002038BD2046FCE703480088401C0249D4
:1034200008802046F5E700000E01002070B5044634
:103430000D460026214628460EF03AF9064630464B
:1034400070BD10B5A021012003F078FE10BD2DE95C
:10345000F04105460F461646012003F039FFA02132
:10346000012004F007F8012003F0A0FE28B9012094
:1034700003F076FF0020BDE8F081C5F307210120AD
:1034800003F0F8FF012003F091FE20B9012003F0C2
:1034900067FF0020EFE7E9B2012003F0EBFF012016
:1034A00003F084FE20B9012003F05AFF0020E2E778
:1034B000012003F00DFFA121012003F0DBFF01201B
:1034C00003F074FE20B9012003F04AFF0020D2E788
:1034D00000240FE0012003F0B1FE3855701EA04219
:1034E00003D9012003F084FF02E0012004F016F864
:1034F000601C84B2B442EDD3012003F031FF0120FF
:10350000B9E72DE9F0470746884691460025002493
:1035100000263E4600BF54E01DB106F01F00002803
:103520003ED1012003F01CFF032021F0D7FB002433
:103530000EE0012003F0CCFEA021012003F09AFF51
:10354000012003F033FE012800D104E0601C84B2A6
:10355000B4F57A7FEDDB00BFB4F57A7F05D10120A9
:1035600003F0FEFE0020BDE8F087C6F3072101202E
:1035700003F080FF012003F019FE20B9012003F0C1
:10358000EFFE0020EFE7F1B2012003F073FF01200E
:1035900003F00CFE20B9012003F0E2FE0020E2E778
:1035A00018F80510012003F065FF012003F0FEFD6F
:1035B00020B9012003F0D4FE0020D4E7761C681C5B
:1035C00085B24D45A8D3012003F0CAFE00240EE0C9
:1035D000012003F07DFEA021012003F04BFF01201C
:1035E00003F0E4FD012800D104E0601C84B2B4F5CE
:1035F0007A7FEDDB00BFB4F57A7F04D1012003F0C0
:10360000AFFE0020AFE7012003F0AAFE052021F065
:1036100065FB0120A7E713B582B0002400200190CC
:1036200003F0A2FD00208DF80400012201A900F0A2
:1036300063FA0446012201A9022000F06FF9044652
:10364000012C09D19DF8040000F0800020B1DDE9D3
:10365000020100F052F80446204604B010BD1CB52B
:10366000044600200090019007226946022000F0E5
:1036700055F99DF8000000F0800050B19DF8000061
:1036800000F07F008DF8000001226946022000F062
:1036900033FA9DF8001001F07F00F8F739F9207037
:1036A0009DF8011001F07F00F8F732F960709DF885
:1036B000021001F03F00F8F72BF9A0709DF80310FD
:1036C00001F03F00F8F724F920719DF8041001F093
:1036D0000700F8F71DF9401CE0709DF8051001F097
:1036E0001F00F8F715F960719DF80600F8F710F95A
:1036F00000F5FA60E08001201CBD13B582B0002007
:103700000090019000249DF8080006F0A8FF8DF8B5
:1037100000009DF8090006F0A2FF8DF801009DF859
:103720000A0006F09CFF40F080008DF802009DF832
:103730000C0006F094FF8DF803009DF80B0006F0D6
:103740008EFF8DF804009DF80D0006F088FF8DF8BF
:103750000500BDF80E10A1F5FA61C8B206F07FFFB2
:103760008DF8060007226946022000F0C5F90446DC
:10377000204604B010BD000033B581B00020009099
:103780000024002503F0F0FC00BF684600F016F9A5
:103790000446012C08D180208DF8000001226946E2
:1037A000072000F06DF904462846691CCDB20228B6
:1037B00001DA002CE9D0012C03D101200A4908705C
:1037C00011E000BFDDE90101FFF725FF04462846AF
:1037D000691CCDB2022801DA002CF3D0012C02D1F1
:1037E0000020014908703EBD0D0100201CB50446B3
:1037F00000200090019020480078B0B3072269466D
:10380000002000F03BF89DF8001001F07F00F8F771
:1038100075F820709DF8011001F07F00F8F76EF840
:1038200060709DF8021001F03F00F8F767F8A07093
:103830009DF8031001F03F00F8F760F820719DF843
:10384000041001F01F00F8F759F860719DF80500A9
:10385000F8F754F800F5FA60E0809DF8061001F0E2
:103860000F00F8F74BF8E07003E0FFE72046FFF7A2
:10387000F6FE01201CBD00000D0100202DE9F041E5
:1038800006460F461446002514B90020BDE8F08115
:10389000002003F01DFDDE21002003F0EBFD0020E1
:1038A00003F084FC20B9002003F05AFD0020EDE76E
:1038B0003146002003F0DEFD002003F077FC20B944
:1038C000002003F04DFD0020E0E7002003F000FDA4
:1038D000DF21002003F0CEFD002003F067FC20B9BB
:1038E000002003F03DFD0020D0E700250FE0002080
:1038F00003F0A4FC7855601EA84203DD002003F00D
:1039000077FD02E0002003F009FE681CC5B2A54265
:10391000EDDB002003F024FD0120B7E72DE9F041A5
:1039200006460F461446002514B90020BDE8F08174
:10393000002003F0CDFCA221002003F09BFD00201D
:1039400003F034FC20B9002003F00AFD0020EDE76D
:103950003146002003F08EFD002003F027FC20B943
:10396000002003F0FDFC0020E0E7002003F0B0FCA5
:10397000A321002003F07EFD002003F017FC20B9F6
:10398000002003F0EDFC0020D0E700250FE0002030
:1039900003F054FC7855601EA84203DD002003F0BC
:1039A00027FD02E0002003F0B9FD681CC5B2A54266
:1039B000EDDB002003F0D4FC0120B7E710B504468E
:1039C000012221460720FFF759FF10BD13B582B031
:1039D000002000900190002428480078002845D05D
:1039E00090208DF8000001226946072000F048F879
:1039F0009DF8080006F026FE8DF800009DF80900ED
:103A000006F020FE8DF801009DF80A0006F01AFE6F
:103A100040F080008DF802009DF80C0006F012FEC8
:103A20008DF803009DF80D0006F00CFE8DF80400E3
:103A3000BDF80E10A1F5FA61C8B206F003FE8DF8CC
:103A400005009DF80B0006F0FDFD8DF8060007222D
:103A50006946002000F014F880208DF80000012253
:103A60006946072000F00CF8044603E0DDE9020196
:103A7000FFF743FE204604B010BD00000D010020FA
:103A80002DE9F04105460E4617460024002003F0BC
:103A90001FFCDE21002003F0EDFC002003F086FB7C
:103AA00028B9002003F05CFC0020BDE8F081294625
:103AB000002003F0DFFC002003F078FB20B9002099
:103AC00003F04EFC0020F0E700240EE0315D002002
:103AD00003F0D0FC002003F069FB20B9002003F0C4
:103AE0003FFC0020E1E7601CC4B2BC42EEDB0020DA
:103AF00003F036FC0120D8E72DE9F04105460E46DB
:103B000017460024002003F0E3FBA221002003F06D
:103B1000B1FC002003F04AFB28B9002003F020FC90
:103B20000020BDE8F0812946002003F0A3FC00201E
:103B300003F03CFB20B9002003F012FC0020F0E76A
:103B400000240EE0315D002003F094FC002003F01F
:103B50002DFB20B9002003F003FC0020E1E7601CEE
:103B6000C4B2BC42EEDB002003F0FAFB0120D8E730
:103B70002DE9F04105460E460024002700BF2DE048
:103B800004EB4400184901EB80008088284404EBD2
:103B90004401154A02EB8101888004EB4400114680
:103BA00001EB8000808804EB440102EB810149882D
:103BB000884211DB002004EB440102EB8101888084
:103BC0003A467B1CDFB206EB021004EB4402064BC4
:103BD00003EB820291688847601CC4B2082CCFD3E3
:103BE0003846BDE8F0810000343700200FB42DE9DD
:103BF000F047DDF82CA28A9F4FF00008C14600254F
:103C000000263C469DF8200004F8010B9DF8210099
:103C100004F8010B2B2004F8010B804600BF0BE0D9
:103C200005F1C80014F014F90646301204F8010B2F
:103C300004F8016B681CC5B2072DF1DB05F1C80063
:103C400014F006F90646301204F8010B2A2004F895
:103C5000010B0D2004F8010B022004F8010B2A20AF
:103C600004F8010B002004F8010B492021F06AFB45
:103C700004F8010B2A2004F8010B00250BE005F1E4
:103C8000DA0014F0E5F80646301204F8010B04F8E7
:103C9000016B681CC5B20A2DF1DB2A2004F8010B68
:103CA00008F1030081B238460DF01CF9814604F892
:103CB000019B4FEA292004F8010B08F10500AAF83E
:103CC00000000120BDE8F0075DF814FB0FB42DE9FA
:103CD000F047DDF82C928A9D0027B84600262C4636
:103CE0009DF8200004F8010B9DF8210004F8010B59
:103CF000BDF824004006000E04F8010BBDF82400B6
:103D00004FF6FF7101EA400700BF11E0BDF8220045
:103D10003044134931F81000001204F8010BBDF8CB
:103D20002200304411F8100004F8010B701CC6B2D8
:103D3000BDF82400B042E9DCF81C81B228460DF041
:103D4000D1F8804604F8018B4FEA282004F8010BD3
:103D5000781DA9F800000120BDE8F0075DF814FB0C
:103D6000ECE80020F0B5ADF20C4D06460F461446C7
:103D70001D464FF4027181A8F4F741FB81AA394630
:103D800030460DF0C5F8012844D19DF80402012801
:103D90003ED1BDF80602BDF808120844B0F5805FB8
:103DA00023DBBDF80602BDF808120844B0F5815FB8
:103DB0001BDC9DF80502042817D1BDF80602A0F50A
:103DC000805080B2ADF8060200F026F84FF4FC7285
:103DD00085A968467F957E94F4F7F8FA81A80FC804
:103DE000FFF774FF0DF20C4DF0BD9DF80502112890
:103DF0000CD14FF4FC7285A968467F957E94F4F748
:103E0000E5FA81A80FC8FFF7F1FEEBE70020E9E72C
:103E10000020E7E70020E5E770B500250024C82072
:103E200021F090FA484908804848408D488047482A
:103E3000D0F84A404FF6DC70844200D30446424931
:103E40008C80F62021F07EFAA0F6AB203E49C88097
:103E50000A2021F077FAA0F5FA703B49088100208A
:103E6000488105F063F8384988810020C881D02056
:103E700021F068FA00EB80004FF6FF7101EA400084
:103E800031490882E12021F05DFA0546642D00DD0C
:103E9000642505EB85004FF6FF7101EA40002A49D1
:103EA00048822A48D0F83E404FF6DC70844200D366
:103EB000044625498C82F32021F044FA2249C88225
:103EC000D12021F03FFA00EB80004FF6FF7101EAAC
:103ED00040001D490883DA2021F034FA1A4948834A
:103EE000DC2021F02FFA184988834FF6FF70C88331
:103EF000DE2021F027FAA0F6AB2013490884E02049
:103F000021F020FAA0F6AB200F494884092021F0C7
:103F100019FAA0F5FA700C4988840020C884D320CF
:103F200021F010FA00EB80004FF6FF7101EA40002B
:103F300005490885D82021F005FA03494885002065
:103F40008885012070BD0000ECE800200CD2002024
:103F50002DE9F0412DED068B8EB004461C2107A8FB
:103F6000F4F74DFA1C216846F4F749FA00BF002621
:103F70001BF06CFAB0EE408A352021F0E3F9C5B2AF
:103F80005F2013F065FF0746F4F7EDFB9FEDF30BA1
:103F900053EC102BF4F7F5FAF4F76EFC0890602060
:103FA00013F056FF0746F4F7DEFB9FEDEC0B53ECE6
:103FB000102BF4F7E6FAF4F75FFC0990612013F098
:103FC00047FFADF82800622013F042FF0746F4F7E0
:103FD000CAFB9FEDE20B53EC102BF4F7D2FAF4F787
:103FE0004BFC0B90632013F033FFADF834006420DA
:103FF00013F02EFF4FF47A71484300EE100AB8EE2A
:10400000C00A8DED0C0A652013F022FFADF81C00EC
:10401000662013F01DFF0746F4F7A5FB9FEDCF0BBD
:1040200053EC102BF4F7ADFAF4F726FC049067205C
:1040300013F00EFFADF81800682013F009FF4FF4DD
:104040007A71484300EE100AB8EEC00A8DED050AF9
:10405000692013F0FDFEADF80000C248007868BB8F
:104060009DED080AB4EEC80AF1EE10FA22D8BD4858
:1040700040682044BB49486008464068BDF82810A5
:10408000884241D30120B74908705F2013F0E0FE59
:104090000746082021F056F980463A464146252039
:1040A00003F04EFF0020AF49486088600120AE4910
:1040B000087029E00020AB49486025E0022D0ED1B0
:1040C000B1EE480AF0EE080AB4EEE00AF1EE10FA9A
:1040D00005DB0020A34908704860886014E0A1480F
:1040E000806820449F498860084690ED020AB8EE37
:1040F000400ADDED0C0AB4EEE00AF1EE10FA03DB43
:10410000002008704860886096480178042000F01C
:1041100067FB9448407800287DD194484078002877
:10412000FAD19DED040AB4EEC80AF1EE10FA7AD87D
:104130008C48C06820448B49C8608C48C0682044C3
:104140008A49C8600846C068BDF81810884230D354
:10415000662013F07DFE0746082021F0F3F8804624
:104160003A464146462003F0EBFE01207F49487065
:104170000020C8604FF4937013F06AFE401C86B2B2
:1041800031464FF4937013F0C7FFBDF81C0060B1C7
:104190007448008ABDF81C10884206D1BDF81C2066
:1041A0007048018A5A2003F0CBFE01206E49087046
:1041B000C4E06C48C068BDF834108842F8D362206F
:1041C00013F046FE0746082021F0BCF880463A4628
:1041D0004146452003F0B4FE0120624948700020AA
:1041E000C8604FF4937013F033FE401C86B2314622
:1041F0004FF4937013F090FFBDF81C0078B159484C
:10420000008ABDF81C10884209D1BDF81C20554811
:10421000018A5A2001E052E005E003F091FE0120FE
:10422000514908708AE09DED0B0AB4EEC80AF1EE20
:1042300010FA3ED800204D49C8604A48C068204462
:104240004849C8600846C068BDF83410884275D334
:10425000622013F0FDFD0746082021F073F8804628
:104260003A464146452003F06BFE01203D49487027
:104270000020C8604FF4937013F0EAFD401C86B232
:1042800031464FF4937013F047FFBDF81C0060B146
:104290003448008ABDF81C10884206D1BDF81C20A5
:1042A0003048018A5A2003F04BFE01202E49087045
:1042B00044E000202B49C8602C49C8603EE0022D34
:1042C00014D1B1EE480AF0EE080AB4EEE00AF1EEBD
:1042D00010FA0BDB002023494870C860088223498C
:1042E0004870C86008821F49886027E01D48008A1E
:1042F000BDF81C10884221DA1A4840692044194947
:104300004861084690ED050AB8EE400ADDED0C0A5A
:10431000B4EEE00AF1EE10FA10DB002048614870BC
:10432000124948700F48008A401C0E490882BDF8A7
:104330001C200846018A5C2003F002FE09484178EF
:10434000042000F061FA09484178052000F05CFA89
:104350000EB0BDEC068BBDE8F08100009A999999EA
:104360009999B93FA84A0020EC320020C04A0020A9
:104370002DE9F0412DED068B8EB004461C2107A8D7
:10438000F4F73DF81C216846F4F739F8002635208B
:1043900020F0D8FFC5B200BF1BF058F8B1EE400ABC
:1043A000B0EE408A6A2013F053FD0746F4F7DBF9BC
:1043B0009FEDF20B53EC102BF4F7E3F8F4F75CFAF3
:1043C00008906B2013F044FD0746F4F7CCF99FEDFD
:1043D000EB0B53EC102BF4F7D4F8F4F74DFA0990EB
:1043E0006C2013F035FDADF828006D2013F030FD82
:1043F0000746F4F7B8F99FEDE10B53EC102BF4F7F7
:10440000C0F8F4F739FA0B906E2013F021FDADF8E7
:1044100034006F2013F01CFD4FF47A71484300EE16
:10442000100AB8EEC00A8DED0C0A702013F010FDD2
:10443000ADF81C00712013F00BFD0746F4F793F95B
:104440009FEDCE0B53EC102BF4F79BF8F4F714FA16
:104450000490722013F0FCFCADF818006F2013F0EC
:10446000F7FC4FF47A71484300EE100AB8EEC00A28
:104470008DED050A742013F0EBFCADF80000C14887
:10448000007860BB9DED080AB4EEC80AF1EE10FAA0
:1044900021D8BC4840682044BA4948600846406872
:1044A000BDF82810884240D36A2013F0D1FC07469B
:1044B000082020F047FF80463A464146262003F078
:1044C0003FFD0120AF49087000204860886001204E
:1044D000AD49087029E00020AA49486025E0012D77
:1044E0000ED1B1EE480AF7EE000AB4EEE00AF1EEA2
:1044F00010FA05DB0020A34908704860886014E0CA
:10450000A048806820449F498860084690ED020AD0
:10451000B8EE400ADDED0C0AB4EEE00AF1EE10FA56
:1045200003DB002008704860886096480178052009
:1045300000F056F99348407800287DD193484078A0
:104540000028FAD19DED040AB4EEC80AF1EE10FA83
:104550007AD88C48C06820448A49C8608B48C068B3
:1045600020448A49C8600846C068BDF818108842CF
:1045700030D30120854948700020C86040F22710E0
:1045800013F066FC401C86B2314640F2271013F04F
:10459000C3FD712013F05CFC0746082020F0D2FE1A
:1045A00080463A464146482003F0CAFCBDF81C004C
:1045B00060B17448008ABDF81C10884206D1BDF86D
:1045C0001C207048018A5B2003F0BAFC01206E4970
:1045D0000870C4E06B48C068BDF834108842F8D356
:1045E0000120684948700020C86040F2271013F08D
:1045F0002FFC401C86B2314640F2271013F08CFD90
:104600006D2013F025FC0746082020F09BFE804615
:104610003A464146472003F093FCBDF81C0078B1B0
:104620005848008ABDF81C10884209D1BDF81C20EA
:104630005448018A5B2001E052E005E003F080FC71
:104640000120514908708AE09DED0B0AB4EEC80ABA
:10465000F1EE10FA3CD800204C49C8604948C068C7
:1046600020444849C8600846C068BDF834108842F4
:1046700075D30120434948700020C86040F22710DC
:1046800013F0E6FB401C86B2314640F2271013F0CF
:1046900043FD6D2013F0DCFB0746082020F052FE9E
:1046A00080463A464146472003F04AFCBDF81C00CC
:1046B000002854D03348008ABDF81C1088424ED1DF
:1046C000BDF81C202F48018A5B2003F039FC46E02E
:1046D00000202C494870C8602C494870C8603EE0F2
:1046E000012D14D1B1EE480AF7EE000AB4EEE00A4B
:1046F000F1EE10FA0BDB002022494870C8600882F6
:1047000022494870C86048701E49486127E01D482A
:10471000008ABDF81C10884221DA1A4840692044FA
:1047200018494861084690ED050AB8EE400ADDEDEB
:104730000C0AB4EEE00AF1EE10FA10DB002048613A
:104740004870124948700F48008A401C0D49088281
:10475000BDF81C200846018A5D2003F0F1FB0948E2
:104760004178062000F050F808484178072000F012
:104770004BF80EB0BDEC068BBDE8F0819A99999983
:104780009999B93FD84A0020EC320020F04A002025
:10479000014601208840044A1268104008B10120F7
:1047A00070470020FCE70000F0310020014800685D
:1047B00070470000F0310020014800687047000099
:1047C000F4310020014601208840044A126810405C
:1047D00008B1012070470020FCE70000F431002000
:1047E00039B1084A1268012383401A43054B1A6005
:1047F00006E0044A1268012383409A43014B1A6081
:1048000070470000F031002039B1084A12680123D6
:1048100083401A43054B1A6006E0044A12680123DC
:1048200083409A43014B1A6070470000F431002026
:10483000F0B52DED068B87B005461C216846F3F7D1
:10484000DEFD312020F07EFD0746F3F78CFF41ECC2
:104850001A0B9FED2C0B53EC102BF3F792FE41EC4F
:10486000190BF4F709F808EE100A0026352020F09D
:1048700069FDC6B2254CAB2013F0EAFA00EE100A2F
:10488000B8EE400A8DED010AAC2013F0E1FA00EE1B
:10489000100AB8EE400A8DED020AAD2013F0D8FAE6
:1048A000ADF80C002078C0B9012E16D09DED010A9C
:1048B000B4EEC80AF1EE10FA0CDB606828446060C0
:1048C000BDF80C106068884213D3012020700020CE
:1048D00060600EE0002060600BE09DED020AB4EE27
:1048E000C80AF1EE10FA01D3012E02D10020207087
:1048F000606021780F20FFF773FF07B0BDEC068BD7
:10490000F0BD00007B14AE47E17A843FB04B00203D
:1049100070B505463A2020F015FD04461948407848
:10492000E8B9C4B11748C06828441649C8600846A9
:10493000C06841F2883188421ED301201149487075
:104940000020C86001222146522003F0F9FA01201C
:104950000D49087010E000200A49C8600CE024B13D
:104960005D2020F0EFFC012806D1002005494870A9
:1049700000215D2020F0F2FC024841781320FFF76F
:1049800043FF70BD084B0020EC3200202DE9F047BA
:104990002DED088B04469FEDAF0AB0EE408A00264D
:1049A00000250027A846A9469FEDAA0AF0EE408AF6
:1049B000252020F0C7FC0646372020F0C3FC054622
:1049C000082020F0BFFC00EE100AF8EE400A9FED30
:1049D000A21A9FEDA20A10EE810AB0EE408A0620CC
:1049E00020F0B0FC8246F3F7BEFE41EC1A0B9FEDBF
:1049F0009C0B53EC102BF3F7C4FD41EC190BF3F7B0
:104A0000DEFE1FFA80F9292020F09CFC8246F3F795
:104A1000AAFE41EC1B0B9FED920B53EC102BF3F70E
:104A2000B0FD41EC1A0B9FED900B53EC102BF3F7FC
:104A3000A2FD41EC190BF3F71FFF08EE900A30209E
:104A400020F080FC00F0010000B10127302020F0B0
:104A500079FC00F0020008B14FF00108844840786A
:104A6000002876D1002F6ED11120F5F723FE012802
:104A700069D1B0EE080AB4EEC08AF1EE10FA2EDD6C
:104A800040F67A5085420DDAB9F50A7F0ADC9FEDCF
:104A9000790AF4EEC08AF1EE10FA03DC0C20FFF77D
:104AA00091FEE0B17248C06820447149C860084670
:104AB000C06842F2107188426BD301206C49487083
:104AC000082020F03FFC824652463146542003F035
:104AD00037FA012068490870FAF7B0FD59E040F64E
:104AE000AC50854227DDB5EEC08AF1EE10FA22DD2A
:104AF0004A2013F0ADF93230B0421CDA5F48C0688A
:104B000020445E49C8600846C06842F2107188427D
:104B10003FD3012056494870082020F013FC8246FC
:104B200052463146542003F00BFA012052490870D6
:104B3000FAF784FD2DE000204D49C8604F49C86058
:104B400027E006E0FFE700204949C8604B49C860FC
:104B50001FE04B480078E0B10C20F5F787FD0128F5
:104B600017D1484800682044464908600846006854
:104B700041F2883188420CD901211820FFF744FE08
:104B8000082020F0DFFB8246524631460C2003F01D
:104B9000D7F9374841781520FFF736FE3A48407874
:104BA00070BBB8F1000F27D140F6B830854223DC46
:104BB000B8EE080AB4EEC08AF1EE10FA1CD2324800
:104BC000C06820443049C8600846C06842F210718D
:104BD000884235D301202C494870082020F0B2FBD0
:104BE000824652463146552003F0AAF90120224957
:104BF0000870FAF723FD23E000202349C8601FE076
:104C00001F480078E0B10C20F5F730FD012817D1DE
:104C10001C48006820441B4908600846006841F2AF
:104C2000883188420CD901211820FFF7EDFD0820BA
:104C300020F088FB8246524631460C2003F080F972
:104C4000114841781620FFF7DFFDBDEC088BBDE869
:104C5000F0870000000000000AD7233C00009643C4
:104C60009A9999999999B93F00000000000049402C
:104C7000684B002000005C42EC320020804B00209A
:104C80003A320020E4310020984B002070B52DED21
:104C9000028B0446002500269FED510AB0EE408AA3
:104CA0001AF0D4FBB0EE408A352020F04BFBC5B2A1
:104CB0004C484078002851D1FEF792FB012839D1A9
:104CC0001AF056FC002835D14748008A02280CDC2F
:104CD0001AF03EFC642020F001F81AF0C7F94248AF
:104CE000008A401C4049088224E001203D49487068
:104CF00000203D4908823B49486100221146562068
:104D000003F01EF940F2251013F0A2F8401C86B201
:104D1000314640F2251013F0FFF93248008A03288B
:104D200005D13048018A0322592003F009F90120F6
:104D30002E490870012D4BD1B0EE080AB4EEC08A9E
:104D4000F1EE10FA44DD0020264908822649088247
:104D5000002140F2251013F0DFF939E05D2020F04A
:104D6000F1FA012810D100201E4948701E4908821E
:104D70001C4908821AF07AF900201A49486100217A
:104D80005D2020F0EBFA23E01648008A03281FDAA2
:104D900014484069204413494861084640694EF66A
:104DA0006021884214D300200E4948701AF05EF941
:104DB0001AF0CEFB0B48008A401C0A4908820846BC
:104DC000018A03225E2003F0BBF8002005494861F8
:104DD000044841781220FFF717FDBDEC028B70BD2F
:104DE00000000000384B0020504B0020EC32002027
:104DF00070B505463B2020F0A5FA0446002604F4D1
:104E0000404000B10126C4F30B000CF00BF804463F
:104E10001B484078F8B90EB9012C18DD1848C06855
:104E200028441749C8600846C06841F28831884262
:104E300020D30120124948700020C8600122214679
:104E4000532003F07DF801200E49087012E0002085
:104E50000B49C8600EE00EB9012C04DD5D2020F086
:104E600071FA012806D100200549487000215D2013
:104E700020F074FA024841781420FFF7C5FC70BD99
:104E8000204B0020EC3200202DE9F0432DED0A8B61
:104E900087B006461C216846F3F7B1FA292020F0B6
:104EA00051FA8046F3F75FFC41EC1C0B9FED830B3E
:104EB00053EC102BF3F765FB41EC1B0B9FED810BC3
:104EC00053EC102BF3F757FB41EC1A0BF3F7D4FC20
:104ED00008EE100A7D4C00279FED7D0BB0EE409A46
:104EE000F0EE609A352020F02DFAC5B2752012F050
:104EF000AFFF80464146002012F0BEFE8DED010A54
:104F0000762012F0A5FF80464146002012F0B4FE44
:104F10008DED020A772012F09BFFADF80C0078208F
:104F200012F096FF80464146002012F0A5FE8DED5E
:104F3000040A792012F08CFF80464146002012F0CE
:104F40009BFE8DED050A7A2012F082FFADF8180065
:104F5000082020F0F7F900EE100AF8EE400A9FED65
:104F60005E1A9FED5E0A10EE810A10EE108A40462E
:104F7000F3F73EFC41EC190B207840BB012D23D107
:104F80009DED010AB4EEC80AF1EE10FA1CD8606873
:104F900030446060BDF80C106068884230D3012056
:104FA000207000206060752012F052FF804629209A
:104FB00020F0C8F9814642464946272002F0C0FF4A
:104FC0000120474908701BE00020606018E0022DB6
:104FD0000CD151EC190B81F0004141EC1A0B9FED03
:104FE000410B53EC102BF3F72FFC06D39DED020A77
:104FF000B4EEC80AF1EE10FA02DB00202070606007
:1050000021780620FFF7ECFB607880BB012D2FD1C3
:105010009DED040AB4EEC80AF1EE10FA28D8E06853
:105020003044E060BDF81810E06888423CD30120AD
:1050300060704FF4967012F00BFF401C87B2394637
:105040004FF4967013F068F8782012F001FF804654
:10505000292020F077F9814642464946492002F04E
:105060006FFF0020E06001201D4908701CE002E095
:105070000020E06018E0022D0CD151EC190B81F0FA
:10508000004141EC1A0B9FED170B53EC102BF3F77B
:10509000DBFB06D39DED050AB4EEC80AF1EE10FA6B
:1050A00002DB00206070E06061780820FFF7ACFB55
:1050B00007B0BDEC0A8BBDE8F08300009A9999997E
:1050C0009999B93F0000000000004940C84B0020FA
:1050D00000000000000000000AD7233C00009643B7
:1050E000EC32002000000000000008402DE9F043F1
:1050F0002DED088B87B006461C216846F3F77FF933
:10510000824C352020F01EF9C5B20027292020F05E
:1051100019F98046F3F727FB41EC1B0B9FED7C0B45
:1051200053EC102BF3F72DFA41EC1A0B9FED7A0B91
:1051300053EC102BF3F71FFA41EC190BF3F79CFB20
:1051400008EE100A9FED760AF0EE408A082020F063
:10515000F9F800EE100AF8EE400A9FED721A9FED82
:10516000720A10EE810AF0EE408A812012F070FE81
:1051700080464146002012F07FFD8DED010A82201D
:1051800012F066FE80464146002012F075FD8DED5E
:10519000020A832012F05CFEADF80C00842012F0AD
:1051A00057FE80464146002012F066FD8DED040A50
:1051B000852012F04DFE80464146002012F05CFD35
:1051C0008DED050A862012F043FEADF81800207818
:1051D00040BB022D23D19DED010AB4EEC80AF1EEC9
:1051E00010FA1CD8606830446060BDF80C1060682C
:1051F00088422AD301202070812012F029FE8046A7
:10520000292020F09FF8814642464946292002F095
:1052100097FE0020606001204449087015E00020DE
:10522000606012E0012D06D1B7EE000AF4EEC08AEC
:10523000F1EE10FA06DA9DED020AB4EEC80AF1EEBC
:1052400010FA02DB00202070606021780820FFF750
:10525000C7FA607880BB022D2FD19DED040AB4EE11
:10526000C80AF1EE10FA28D8E0683044E060BDF8D2
:105270001810E06888423FD3012060704FF49770A7
:1052800012F0E6FD401C87B239464FF4977012F0D9
:1052900043FF842012F0DCFD8046292020F052F8E4
:1052A0008146424649464B2002F04AFE0020E0601B
:1052B00001201E4908701FE002E00020E0601BE0B2
:1052C000012D06D1B7EE000AF4EEC08AF1EE10FA15
:1052D0000BDA9DED050AB4EEC80AF1EE10FA04DA15
:1052E0005D2020F02FF8012806D100206070E060DA
:1052F00000215D2020F032F861780A20FFF784FA5F
:1053000007B0BDEC088BBDE8F0830000F84B00202F
:105310009A9999999999B93F000000000000494075
:10532000000000000AD7233C00009643EC32002026
:10533000F0B52DED088B87B005461C216846F3F7C4
:105340005EF8644C0A201FF0FDFF0646F3F70BFAE7
:1053500041EC1B0B9FED600B53EC102BF3F711F995
:1053600041EC1A0B9FED5E0B53EC102BF3F703F996
:1053700041EC190BF3F780FA08EE100A8D2012F0B9
:1053800067FD06463146002012F076FC8DED010ADD
:105390008E2012F05DFD06463146002012F06CFCB6
:1053A0008DED020A8F2012F053FDADF80C00902015
:1053B00012F04EFD06463146002012F05DFC8DEDE8
:1053C000040A912012F044FD06463146002012F0F6
:1053D00053FC8DED050A922012F03AFDADF818004D
:1053E000207830BB9DED010AB4EEC80AF1EE10FA48
:1053F0001CD8606828446060BDF80C106068884262
:1054000020D3012020708D2012F022FD06460A20B4
:105410001FF098FF0746324639462B2002F090FDD8
:10542000002060600120304908700BE000206060BF
:1054300008E09DED020AB4EEC80AF1EE10FA01DBB5
:105440000020207021780B20FFF7CAF9607830BB6C
:105450009DED040AB4EEC80AF1EE10FA1CD8E0681B
:105460002844E060BDF81810E068884229D3012084
:105470006070902012F0ECFC06460A201FF062FFDC
:105480000746324639464D2002F05AFD0020E060C2
:1054900001201549087014E00020E06011E09DED46
:1054A000050AB4EEC80AF1EE10FA04DA5D201FF026
:1054B00049FF012805D10020607000215D201FF008
:1054C0004DFF61780D20FFF79FF907B0BDEC088B09
:1054D000F0BD0000404C00209A9999999999B93FE4
:1054E0000000000000004940EC320020F0B52DED36
:1054F000088B87B005461C216846F2F780FF644C94
:1055000009201FF01FFF0646F3F72DF941EC1B0B96
:105510009FED600B53EC102BF3F733F841EC1A0BB3
:105520009FED5E0B53EC102BF3F725F841EC190BB4
:10553000F3F7A2F908EE100A992012F089FC06464A
:105540003146002012F098FB8DED010A9A2012F0EE
:105550007FFC06463146002012F08EFB8DED020ADC
:105560009B2012F075FCADF80C009C2012F070FC32
:1055700006463146002012F07FFB8DED040A9D2087
:1055800012F066FC06463146002012F075FB8DEDE8
:10559000050A9E2012F05CFCADF81800207830BBA4
:1055A0009DED010AB4EEC80AF1EE10FA1CD860684D
:1055B00028446060BDF80C106068884220D3012048
:1055C0002070992012F044FC064609201FF0BAFE14
:1055D0000746324639462C2002F0B2FC00206060BB
:1055E0000120304908700BE00020606008E09DED6C
:1055F000020AB4EEC80AF1EE10FA01DB00202070B6
:1056000021780A20FFF7ECF8607830BB9DED040AA2
:10561000B4EEC80AF1EE10FA1CD8E0682844E06045
:10562000BDF81810E068884229D3012060709C20E2
:1056300012F00EFC064609201FF084FE0746324693
:1056400039464F2002F07CFC0020E0600120154923
:10565000087014E00020E06011E09DED050AB4EE52
:10566000C80AF1EE10FA04DA5D201FF06BFE012883
:1056700005D10020607000215D201FF06FFE617871
:105680000C20FFF7C1F807B0BDEC088BF0BD00009F
:10569000704C00209A9999999999B93F000000009F
:1056A00000004940EC3200202DE9F0432DED0A8B3B
:1056B00087B006461C216846F2F7A1FE884C3520CB
:1056C0001FF040FEC5B200272B201FF03BFE804696
:1056D000F3F749F841EC1C0B9FED820B53EC102BB8
:1056E000F2F74FFF41EC1B0B9FED800B53EC102B9F
:1056F000F2F741FF41EC1A0BF3F7BEF808EE100A7F
:105700009FED7C0BB0EE409AF0EE609A08201FF0FF
:1057100019FE00EE100AF8EE400A9FED781A9FED90
:10572000780A10EE810A10EE108A4046F3F760F80E
:1057300041EC190B7B2012F08BFB80464146002088
:1057400012F09AFA8DED010A7C2012F081FB80465E
:105750004146002012F090FA8DED020A7D2012F0F1
:1057600077FBADF80C007E2012F072FB80464146BC
:10577000002012F081FA8DED040A7F2012F068FB00
:1057800080464146002012F077FA8DED050A802010
:1057900012F05EFBADF81800207840BB012D23D13C
:1057A0009DED010AB4EEC80AF1EE10FA1CDB606848
:1057B00030446060BDF80C106068884230D301202E
:1057C00020707B2012F044FB80462B201FF0BAFD96
:1057D000814642464946282002F0B2FB0020606024
:1057E0000120484908701BE00020606018E0022D8D
:1057F0000CD151EC190B81F0004141EC1A0B9FEDDB
:10580000420B53EC102BF3F71FF806D39DED020A61
:10581000B4EEC80AF1EE10FA02D8002020706060E1
:1058200021780720FEF7DCFF607890BB012D31D195
:105830009DED040AB4EEC80AF1EE10FA2ADBE06826
:105840003044E060BDF81810E06888423ED3012083
:1058500060700020E06040F22D1012F0F9FA401C58
:1058600087B2394640F22D1012F056FC7E2012F01D
:10587000EFFA80462B201FF065FD814642464946DF
:105880004A2002F05DFB0020606001201D49087085
:105890001CE002E00020E06018E0022D0CD151EC89
:1058A000190B81F0004141EC1A0B9FED170B53ECE3
:1058B000102BF2F7C9FF06D39DED050AB4EEC80A16
:1058C000F1EE10FA02D800206070E06061780920E3
:1058D000FEF79AFF07B0BDEC0A8BBDE8F08300002D
:1058E000E04B00209A9999999999B93F00000000DE
:1058F0000000494000000000000000000AD7233CDF
:1059000000009643EC320020000000000000084038
:105910002DE9F0432DED0A8B87B006461C21684621
:10592000F2F76DFD874C002735201FF00BFDC5B247
:105930002B201FF007FD8046F2F715FF41EC1C0BF2
:105940009FED810B53EC102BF2F71BFE41EC1B0B70
:105950009FED7F0B53EC102BF2F70DFE41EC1A0B71
:10596000F2F78AFF08EE100A9FED7B0BB0EE409A2B
:10597000F0EE609A08201FF0E5FC00EE100AF8EE49
:10598000400A9FED771A9FED770A10EE810A10EE1C
:10599000108A4046F2F72CFF41EC190B872012F0D9
:1059A00057FA80464146002012F066F98DED010A53
:1059B000882012F04DFA80464146002012F05CF932
:1059C0008DED020A892012F043FAADF80C008A200E
:1059D00012F03EFA80464146002012F04DF98DED5E
:1059E000040A8B2012F034FA80464146002012F05F
:1059F00043F98DED050A8C2012F02AFAADF8180053
:105A0000207840BB022D23D19DED010AB4EEC80AD7
:105A1000F1EE10FA1CDD606830446060BDF80C10D7
:105A2000606888422CD301202070872012F010FA81
:105A300080462B201FF086FC8146424649462A209C
:105A400002F07EFA0020606001204749087017E0EC
:105A50000020606014E0012D08D19FED440B53EC51
:105A6000102B51EC190BF2F7EFFE06D99DED020A4F
:105A7000B4EEC80AF1EE10FA02D80020207060607F
:105A800021780920FEF7ACFE607880BB022D2FD173
:105A90009DED040AB4EEC80AF1EE10FA28DBE068C6
:105AA0003044E060BDF81810E068884241D301201E
:105AB000607040F22F1012F0CBF9401C87B23946CB
:105AC00040F22F1012F028FB8A2012F0C1F9804614
:105AD0002B201FF037FC8146424649464C2002F0FD
:105AE0002FFA0020E06001201F49087021E002E049
:105AF0000020E0601DE0012D08D19FED1C0B53EC50
:105B0000102B51EC190BF2F79FFE0BD99DED050AF6
:105B1000B4EEC80AF1EE10FA04D95D201FF012FCB1
:105B2000012806D100206070E06000215D201FF098
:105B300015FC61780B20FEF767FE07B0BDEC0A8B01
:105B4000BDE8F083104C00209A9999999999B93F32
:105B500000000000000049400000000000000000BC
:105B60000AD7233C00009643EC32002000000000DE
:105B70000000F03FF0B52DED088B87B005461C21E5
:105B80006846F2F73CFC704C0A201FF0DBFB06462F
:105B9000F2F7E9FD41EC1B0B9FED6C0B53EC102B66
:105BA000F2F7EFFC41EC1A0B9FED6A0B53EC102B54
:105BB000F2F7E1FC41EC190BF2F75EFE08EE100A79
:105BC000932012F045F906463146002012F054F8B1
:105BD0008DED010A942012F03BF906463146002073
:105BE00012F04AF88DED020A952012F031F9ADF865
:105BF0000C00962012F02CF906463146002012F0D7
:105C00003BF88DED040A972012F022F90646314642
:105C1000002012F031F88DED050A982012F018F9E5
:105C2000ADF81800207870BB9DED010AB4EEC80AEB
:105C3000F1EE10FA28DBB2EE040A28EE000ADFEDDE
:105C4000470AB4EE600AF1EE10FA1DD060682844ED
:105C50006060BDF80C106068884221D3012020707C
:105C6000932012F0F5F806460A201FF06BFB07465A
:105C7000324639462F2002F063F90020606001208F
:105C8000374908700CE002E00020606008E09DEDFC
:105C9000020AB4EEC80AF1EE10FA01D80020207012
:105CA00021780C20FEF79CFD607870BB9DED040A06
:105CB000B4EEC80AF1EE10FA28DBB2EE040A28EEC0
:105CC000000ADFED260AB4EE600AF1EE10FA1DD0EC
:105CD000E0682844E060BDF81810E06888422AD3E4
:105CE00001206070962012F0B3F806460A201FF0DB
:105CF00029FB0746324639464E2002F021F90020A2
:105D0000E06001201649087015E002E00020E06024
:105D100011E09DED050AB4EEC80AF1EE10FA04D9BF
:105D20005D201FF00FFB012805D1002060700021CD
:105D30005D201FF013FB61780E20FEF765FD07B0B4
:105D4000BDEC088BF0BD0000584C00209A99999941
:105D50009999B93F00000000000049400000CDC300
:105D6000EC3200202DE9F0432DED068B87B005467F
:105D70001C216846F2F743FB9F4C35201FF0E2FAE6
:105D8000C6B2002706201FF0DDFA8046F2F7EBFCD2
:105D900041EC1A0B9FED990B53EC102BF2F7F1FB32
:105DA00041EC190BF2F768FD08EE100A9FED950A19
:105DB000F0EE408A19F04AFBF0EE408A532012F0D0
:105DC00047F880464146032011F056FF8DED010A49
:105DD000542012F03DF880464146032011F04CFF5C
:105DE0008DED020A552012F033F8ADF80C00562064
:105DF00012F02EF880464146032011F03DFF8DED54
:105E0000040A572012F024F880464146032011F07E
:105E100033FF8DED050A582012F01AF8ADF818007E
:105E20002078A8BB022E34D09DED010AB4EEC80A3A
:105E3000F1EE10FA2DD8606828446060BDF80C10AF
:105E40006068884257D301202070532012F000F878
:105E5000804606201FF076FA8146424649462320B6
:105E600002F06EF8002060601320FEF7ABFC58B91A
:105E700042F210701BF086FB01211920FEF7C4FCD2
:105E800001211220FEF7ACFC01205F49087032E0CE
:105E900002E0002060602EE035201FF053FA022857
:105EA00008D1B1EE680AF0EE080AB4EEE00AF1EEAD
:105EB00010FA1DDC31201FF045FA8046F2F753FC42
:105EC00041EC1A0B9FED4D0B53EC102BF2F759FBE5
:105ED00041EC190B9FED4D0B53EC102BF2F79CFC92
:105EE00006D39DED020AB4EEC80AF1EE10FA02DB09
:105EF00000202070606021780220FEF771FC60783D
:105F0000F0BB022E40D09DED040AB4EEC80AF1EEBB
:105F100010FA39D8E0682844E060BDF81810E0684D
:105F2000884260D3012060704FF4957011F090FFAB
:105F3000401C87B239464FF4957012F0EDF85620A8
:105F400011F086FF804606201FF0FCF9814642468C
:105F50004946432001F0F4FF0020E0601320FEF7E3
:105F600031FC58B942F210701BF00CFB01211920D2
:105F7000FEF74AFC01211220FEF732FC012000E06E
:105F800005E0214908702EE00020E0602BE0022EA1
:105F900008D1B1EE680AF0EE080AB4EEE00AF1EEBC
:105FA00010FA1DDC31201FF0CDF98046F2F7DBFB43
:105FB00041EC1A0B9FED110B53EC102BF2F7E1FAA9
:105FC00041EC190B9FED110B53EC102BF2F724FC55
:105FD00006D39DED050AB4EEC80AF1EE10FA02DB15
:105FE00000206070E06061780220FEF70DFC07B0D1
:105FF000BDEC068BBDE8F083B84C00207B14AE47A7
:10600000E17A843F00000000EC3200200000000034
:10601000000058402DE9F0432DED068B87B0064671
:106020001C216846F2F7EBF9874C35201FF08AF9FE
:10603000C5B2002706201FF085F98046F2F793FBD2
:1060400041EC1A0B9FED810B53EC102BF2F799FAF0
:1060500041EC190BF2F710FC08EE100A9FED7D0AD7
:10606000F0EE408A19F0F2F9F0EE408A592011F072
:10607000EFFE80464146032011F0FEFD8DED010A42
:106080005A2011F0E5FE80464146032011F0F4FD50
:106090008DED020A5B2011F0DBFEADF80C005C20F8
:1060A00011F0D6FE80464146032011F0E5FD8DED4E
:1060B000040A5D2011F0CCFE80464146032011F019
:1060C000DBFD8DED050A5E2011F0C2FEADF8180073
:1060D000207888BB012D30D09DED010AB4EEC80AAE
:1060E000F1EE10FA29DB606830446060BDF80C10F6
:1060F0006068884237D3012020701320FEF762FBCE
:1061000038B927201FF01EF9642802DD00201BF09B
:1061100039FA592011F09CFE804606201FF012F932
:10612000814642464946242001F00AFF0020606073
:1061300001204949087016E002E00020606012E08A
:10614000012D06D1B7EE000AF4EEC08AF1EE10FA86
:1061500006DC9DED020AB4EEC80AF1EE10FA02D890
:1061600000202070606021780320FEF739FB607802
:10617000F0BB3A480078E0B3012D3DD09DED040A14
:10618000B4EEC80AF1EE10FA36DBE0683044E060A5
:10619000BDF81810E06888424DD30120607040F2CD
:1061A0002B1011F055FE401C87B2394640F22B10DF
:1061B00011F0B2FF5C2011F04BFE804606201FF06C
:1061C000C1F8814642464946442001F0B9FE00200C
:1061D000E0601320FEF7F6FA38B927201FF0B2F876
:1061E000642802DD00201BF0CDF901201A4901E0EE
:1061F00005E001E008701EE00020E0601BE0012DDA
:1062000006D1B7EE000AF4EEC08AF1EE10FA0BDC0C
:106210009DED050AB4EEC80AF1EE10FA04D95D202E
:106220001FF090F8012806D100206070E060002186
:106230005D201FF093F861780320FEF7E5FA07B0C0
:10624000BDEC068BBDE8F083D04C00207B14AE473C
:10625000E17A843F00000000EC320020E8310020A9
:106260002DE9F0432DED068B87B005461C216846CD
:10627000F2F7C5F89A4C00279FED9A0AF0EE408A93
:1062800019F0E4F8F0EE408A35201FF05BF8C6B252
:1062900025201FF057F808EE100A472011F0D8FD0E
:1062A00000EE100AB8EE400A8DED010A482011F008
:1062B000CFFD00EE100AB8EE400A8DED020A49202B
:1062C00011F0C6FDADF80C004A2011F0C1FD00EE42
:1062D000100AB8EE400A8DED040A4B2011F0B8FD0B
:1062E00000EE100AB8EE400A8DED050A4C2011F0C0
:1062F000AFFDADF818002078B8BB022E36D09DED6A
:10630000010AF8EE480AB4EEE00AF1EE10FA2DD8D0
:10631000606828446060BDF80C106068884259D3FA
:10632000012020701320FEF74DFA58B942F2107088
:106330001BF028F901211920FEF766FA012112202D
:10634000FEF74EFA472011F083FD804625201EF00F
:10635000F9FF814642464946212001F0F1FD002027
:10636000606001206049087034E002E00020606055
:1063700030E035201EF0E6FF022808D1B1EE680AB1
:10638000F0EE080AB4EEE00AF1EE10FA1FDC31205C
:106390001EF0D8FF8046F2F7E6F941EC1A0B9FEDAC
:1063A000530B53EC102BF2F7ECF841EC190B9FED6B
:1063B000510B53EC102BF2F72FFA08D39DED020A84
:1063C000F8EE480AB4EEE00AF1EE10FA02DB002023
:1063D0002070606021780020FEF702FA6078E8BB48
:1063E000022E42D09DED040AF8EE480AB4EEE00A0F
:1063F000F1EE10FA39D8E0682844E060BDF81810D2
:10640000E068884262D3012060701320FEF7DAF959
:1064100058B942F210701BF0B5F801211920FEF7AF
:10642000F3F901211220FEF7DBF94FF4947011F01B
:106430000FFD401C87B239464FF4947011F06CFE8A
:106440004A2011F005FD804625201EF07BFF814685
:1064500042464946412001F073FD00E008E000207B
:10646000E06001202049087030E00020E0602DE06D
:10647000022E08D1B1EE680AF0EE080AB4EEE00A86
:10648000F1EE10FA1FDC31201EF05CFF8046F2F7BF
:106490006AF941EC1A0B9FED150B53EC102BF2F738
:1064A00070F841EC190B9FED130B53EC102BF2F726
:1064B000B3F908D39DED050AF8EE480AB4EEE00AF8
:1064C000F1EE10FA02DB00206070E06061780020DD
:1064D000FEF79AF907B0BDEC068BBDE8F08300002B
:1064E000884C002000000000EC3200207B14AE47F6
:1064F000E17A843F00000000000058402DE9F0439D
:106500002DED028B87B005461C216846F1F777FF19
:10651000954C002735201EF015FFC6B227201EF02F
:1065200011FF08EE100A9FED910AF0EE408A18F074
:106530008DFFF0EE408A4D2011F08AFC00EE100A2B
:10654000B8EE400A8DED010A4E2011F081FC00EEFC
:10655000100AB8EE400A8DED020A4F2011F078FCC7
:10656000ADF80C00502011F073FC00EE100AB8EEEC
:10657000400A8DED040A512011F06AFC00EE100A69
:10658000B8EE400A8DED050A522011F061FCADF81D
:1065900018007748007800BB7648006828447549A1
:1065A0000860B1EE680AF1EE040AB4EEE00AF1EE1A
:1065B00010FA05DD0846006842F21071884205D2E3
:1065C0006C4800684EF66021884209D30020694972
:1065D000086001206649087002E0002065490860F3
:1065E000207898BB012E32D09DED010AF8EE480AC2
:1065F000B4EEE00AF1EE10FA29DB6068284460602E
:10660000BDF80C106068884239D301202070132037
:10661000FEF7D8F838B927201EF094FE642802DD72
:1066200000201AF0AFFF4D2011F012FC8046272009
:106630001EF088FE814642464946222001F080FC39
:106640000020606001204C49087018E002E0002042
:10665000606014E0012E06D1B7EE000AF4EEC08AA5
:10666000F1EE10FA08DA9DED020AF8EE480AB4EEEF
:10667000E00AF1EE10FA02D8002020706060217864
:106680000120FEF7ADF86078F0BB39480078E0B340
:10669000012E3FD09DED040AF8EE480AB4EEE00A60
:1066A000F1EE10FA36DBE0682844E060BDF818101F
:1066B000E06888424FD3012060701320FEF782F813
:1066C00038B927201EF03EFE642802DD00201AF0B3
:1066D00059FF40F2291011F0BBFB401C87B239462C
:1066E00040F2291011F018FD502011F0B1FB804646
:1066F00027201EF027FE814642464946422001F0EF
:106700001FFC0020E06001E007E003E001201A49DF
:10671000087020E00020E0601DE0012E06D1B7EEF9
:10672000000AF4EEC08AF1EE10FA0DDA9DED050ACA
:10673000F8EE480AB4EEE00AF1EE10FA04D95D2052
:106740001EF000FE012806D100206070E0600021EC
:106750005D201EF003FE61780120FEF755F807B0BA
:10676000BDEC028BBDE8F083A04C002000000000CF
:10677000E8310020EC310020EC320020F0B587B089
:1067800006461C216846F1F73AFE5C4C25201EF0B7
:10679000D9FD074627201EF0D5FD381A85B2A52061
:1067A00011F056FB00EE100AB8EE400A8DED010A1A
:1067B000A62011F04DFB00EE100AB8EE400A8DED58
:1067C000020AA72011F044FBADF80C00A82011F03C
:1067D0003FFB00EE100AB8EE400A8DED040AA92036
:1067E00011F036FB00EE100AB8EE400A8DED050AF6
:1067F000AA2011F02DFBADF81800207830BBDDED9C
:10680000010A00EE105AB8EE400AF4EEC00AF1EEAA
:1068100010FA18D8606830446060BDF80C106068E9
:10682000884220D301202070A52011F011FB0746DB
:106830003A4629462D2001F083FB002060600120AC
:106840002F4908700FE0002060600CE0DDED020AC7
:1068500000EE105AB8EE400AF4EEC00AF1EE10FA5B
:1068600001DB0020207021780D20FDF7B9FF607852
:1068700030BBDDED040A00EE105AB8EE400AF4EE2B
:10688000C00AF1EE10FA18D8E0683044E060BDF8B4
:106890001810E06888422AD301206070A82011F007
:1068A000D7FA07463A462946502001F049FB002016
:1068B000E06001201249087019E00020E06016E055
:1068C000DDED050A00EE105AB8EE400AF4EEC00AFB
:1068D000F1EE10FA04DA5D201EF034FD012806D135
:1068E00000206070E06000215D201EF037FD6178BF
:1068F0000F20FDF789FF07B0F0BD0000E84C002035
:10690000EC32002010B53548F2F7D8FE4FF43022B3
:1069100000213248F3F71CF94FF08040806B20F0E3
:106920007F404FF0804188630846806B40F088507C
:1069300088630846C06B0020C8630846C06B40F0FF
:106940001130C8634FF04020406C254908434FF098
:106950004021486400212348F3F7DCF90623002294
:1069600011462048F3F7BEF90723002201211D48F4
:10697000F3F7B8F90823002202211A48F3F7B2F915
:106980000923002203211748F3F7ACF90A23002258
:1069900004211448F3F7A6F90B230022052111481E
:1069A000F3F7A0F90C23002206210E48F3F79AF919
:1069B0000D23002207210B48F3F794F90E23002240
:1069C00008210848F3F78EF90F2300220921054812
:1069D000F3F788F900F02EF810BD00001CFE03400C
:1069E0000000C0FF00300440014600220A2901DBFC
:1069F00000207047074B53F8210082B240F6E44371
:106A000002FB03F0C31700EB1353C3F30F3210461E
:106A1000EFE7000000300440014600220A2901DBB4
:106A200000207047024B53F8210082B21046F8E76D
:106A30000030044040F2FF70014948657047000093
:106A40000030044098B94FF08041C96841F080712E
:106A50004FF08042D1601146C96821F08071D16049
:106A60000D49096821F08071C2F8081212E001286E
:106A700010D18107C96841F000718207D160810798
:106A8000C96821F00071D1600349096821F00071E3
:106A9000C2F80812704700000802004070B50446B2
:106AA0000D46022C00DB70BD94BB0020FFF7CAFF2F
:106AB0004120334908600846006820F04100086022
:106AC0000E2008602F48006840F080704903C1F82C
:106AD00008020846C06C20F4706040F48060C8640E
:106AE0000846C06C20F4704040F48040C864002226
:106AF00029462348F2F768F90E212148F2F72BF9CD
:106B00000D213820F3F794FF3820F3F76FFF34E0BE
:106B1000FFE7012C31D10120FFF794FF41201A49F2
:106B200008600846006820F0410008600E200860F8
:106B30001448006840F000708904C1F80802084653
:106B4000406C20F4700040F4A00048640846C06C1B
:106B500020F4702040F4A020C864002229460A488E
:106B6000F2F732F90E210848F2F7F5F80E21392034
:106B7000F3F75EFF3920F3F739FF00BF93E700001A
:106B800000000A400802004000100A4070B586B0BC
:106B900004460D4600200290039004900590022CBC
:106BA00001DB06B070BD02AA2946204600F014F8A9
:106BB00000B9F6E7074850F8240040B10598009066
:106BC000044850F82460204602A90EC9B04700BF0F
:106BD000E7E7000084000020F0B58BB005460F46C3
:106BE0001646182105A8F1F70AFC00200190029032
:106BF000039004900024022D01DB0BB0F0BD164978
:106C000051F8250005AA3946F2F7C6F920B90698C9
:106C1000C0B28DF80400F0E70598C0B28DF8050009
:106C2000079802909DF820008DF80600002406E0E9
:106C30000DF12100015D03A80155601CC4B2082CB0
:106C400003DA9DF80600A042F2DC01A80FC886E82E
:106C50000F000120D1E700007C0000200FB470B5C8
:106C600086B0044618216846F1F7C9FB00250A26BC
:106C7000022C04DB002006B070BC5DF814FB012080
:106C800001909DF82D0000900C9802909DF82E0028
:106C90008DF80C00002505E00DA8415D2738415511
:106CA000681CC5B2082D03DA9DF82E00A842F3DC5B
:106CB000124951F824006A460121F2F720FC08B974
:106CC0000020D8E705E006B90BE001201EF006F829
:106CD000761E0A4850F82400406800F0080000289A
:106CE000F1D000BF054850F82400406820F00800AB
:106CF000024951F8241048600120BCE77C000020C4
:106D0000022800DB7047024A42F8201000BFF9E772
:106D1000840000202DE9F84304460D4616461F4620
:106D2000DDF82080022C01DA202D01DBBDE8F8839C
:106D30000549CDF8008051F824003B4632462946EB
:106D4000F2F752FA00BFF1E77C00002070B504466C
:106D50002C4D2D48844204D0844202D0844200D07D
:106D600000E0284D00BF00BF00BF59202749086040
:106D700016208905C1F800018820C1F80001C0066D
:106D8000D0F800010028F0D000BF2048F43000689F
:106D9000C0B2012801D11E4908604AF6EE204FF02A
:106DA000804188651B48006820F0F0004FF04021CA
:106DB000C1F840010804D0F8000240F001000904C5
:106DC000C1F800020120F2F76BFF4FF40070104988
:106DD00038390860801E091D08600F484FF0804157
:106DE000C1F870022846F2F723FE11208107C1F88E
:106DF0003402F4F763F800BF00200449086000BFC4
:106E000070BD00000090D00300366E01000100400C
:106E1000B0020040404100403030030010B5F3F7AD
:106E2000D9FF0548006820F0080003490860F2F720
:106E300095FFF3F7C9FF10BD00C000402DE9F047F2
:106E400006460F4600240025A046A146F3F7C2FFE0
:106E5000344619E0002500BF2046F2F789FF00F014
:106E6000FF08681CC5B200F0C5FF032D02DAB8F1B7
:106E7000000FF1D1032D02DAB8F1000F02D04FF06C
:106E8000010906E004F58054BC4202D2B4F5002F9B
:106E9000E0D300BFF3F798FF4846BDE8F087000055
:106EA00010B5F3F797FFF2F7E7FF0448006840F0EA
:106EB000080002490860F3F787FF10BD00C00040DA
:106EC0002DE9F04107460D46904600260024F3F7D1
:106ED00081FF00BF10E0E019F2F7D8FF06462E55FB
:106EE000C6F30721601C2954C6F30741A01C29548E
:106EF000310EE01C2954241D4445ECD3F3F764FF04
:106F0000BDE8F0812DE9F05F04460F46904600256C
:106F1000A946AA460026AB46F3F75CFF26461DE0CD
:106F2000002500BF57F80AB059463046F2F7DAFF9D
:106F300000F0FF09681CC5B2032D02DAB9F1000F99
:106F4000F0D1032D07DBB9F1000F04D0F3F73CFFBC
:106F50000120BDE8F09F0AF1040A361D08EB040089
:106F6000B042DDD8F3F730FF0020F2E770B50346FA
:106F7000002011E0012484400C4001258540AC42F2
:106F800009D11C6846000325B540AC43450002FA10
:106F900005F52C431C60401C1028EBD370BD024645
:106FA0009068084008B1012070470020FCE70246C5
:106FB0001069084008B1012070470020FCE7826892
:106FC0008A438260704782680A43826070478268A1
:106FD0000A401AB182688A43826002E082680A43EA
:106FE0008260704710B50448006820B1034A1068F9
:106FF000014A1168884710BDF03D0020003E002086
:1070000010B50448406820B1034A5068014A5168ED
:10701000884710BDF03D0020003E002010B5044818
:10702000806820B1034A9068014A9168884710BD82
:10703000F03D0020003E002010B50448C06820B19B
:10704000034AD068014AD168884710BDF03D00204E
:10705000003E00202DE9F04104460D461646042C62
:1070600000DA15B90020BDE8F081224A02EB0412D3
:107070005168204A02EB041290680C22F2F768FD76
:107080001C4901EB04118868F2F718FB4FF47A7081
:10709000B0FBF5F7174901EB04113A4608684FF0C9
:1070A0000061F3F7CFFF134901EB04110868016891
:1070B00041F00051016000BF0E4901EB041191F94C
:1070C0000C0000F01F02012191404209920002F1E0
:1070D000E022C2F8001100BF064901EB0411086864
:1070E000F3F7D1FF044840F82450044840F82460E6
:1070F0000120B8E78C000020003E0020F03D002079
:1071000010B50446022C00DB10BD0B4A02EB041242
:10711000D168094A02EB04129068FFF754FF064A4F
:1071200002EB04125168044A02EB04121068FFF7E4
:107130004AFF00BFE8E70000F87A030070B5054693
:107140000C460026284600F0C3F844F0010128460A
:1071500000F090F9284600F029F80646284600F08D
:10716000FFF8304670BD000010B50446022C00DB6D
:1071700010BD0D4A02EB041251680B4A02EB0412D7
:1071800010680122FFF7F2FE074A02EB0412D168F1
:10719000054A02EB041290680122FFF7E7FE204641
:1071A000FFF7AEFF00BFE3E7F87A030070B50446CF
:1071B00001260025022C01DB002070BD1E4A02EBD7
:1071C0000412D1681C4A02EB041290680022FFF7F7
:1071D000CDFE042009F044FE174A02EB0412516868
:1071E000154A02EB04121068FFF7EDFE042009F0C7
:1071F00037FE08E0681C85B2FF2D04DD204600F054
:10720000AFF80020D9E70C4A02EB0412D1680A4A11
:1072100002EB04129068FFF7CAFE0028EAD1064A82
:1072200002EB04125168044A02EB04121068FFF7E3
:10723000C6FE3046C1E70000F87A030070B5044688
:1072400000260025022C01DB002070BD1F4A02EB46
:107250000412D1681D4A02EB041290680022FFF765
:1072600085FE00262DE0194A02EB04125168174AE8
:1072700002EB04121068FFF7A2FE042009F0F0FDF3
:10728000124A02EB04125168104A02EB0412106811
:10729000FFF799FE042009F0E3FD6806050E0B4A8E
:1072A00002EB0412D168094A02EB04129068FFF75E
:1072B0007EFE08B145F00105042009F0D1FD701CE7
:1072C000C6B2082ECFDB2846BFE70000F87A0300DD
:1072D00010B50446022C00DB10BD204A02EB04125C
:1072E000D1681E4A02EB041290680122FFF73EFEAD
:1072F0001A4A02EB04125168184A02EB0412106891
:10730000FFF761FE042009F0ABFD144A02EB041202
:10731000D168124A02EB04129068FFF754FE08206D
:1073200009F09EFD0D4A02EB0412D1680B4A02EBF4
:1073300004129068FFF743FE042009F091FD074A0C
:1073400002EB04125168054A02EB04121068FFF7C1
:1073500036FE042009F084FD00BFBDE7F87A030083
:1073600010B50446022C00DB10BD204A02EB0412CB
:10737000D1681E4A02EB041290680122FFF7F6FD65
:107380001A4A02EB04125168184A02EB0412106800
:10739000FFF715FE042009F063FD144A02EB041206
:1073A000D168124A02EB04129068FFF708FE04202D
:1073B00009F056FD0D4A02EB041251680B4A02EB2C
:1073C00004121068FFF7FFFD042009F049FD074A89
:1073D00002EB0412D168054A02EB04129068FFF731
:1073E000F2FD042009F03CFD00BFBDE7F87A030080
:1073F00010B504461E4A02EB041251681C4A02EB07
:1074000004121068FFF7DBFD194A02EB0412D16881
:10741000174A02EB041290680122FFF7A7FD144AF5
:1074200002EB0412D168124A02EB04129068FFF7D3
:10743000C6FD042009F014FD0D4A02EB0412516848
:107440000B4A02EB04121068FFF7BDFD042009F09F
:1074500007FD074A02EB04125168054A02EB0412C9
:107460001068FFF7ACFD042009F0FAFC10BD000025
:10747000F87A030070B504460D460026022C00DBA6
:1074800070BD254A02EB0412D168234A02EB0412B4
:1074900090680122FFF76AFD002638E0042009F019
:1074A000DFFC05F0800050B11B4A02EB0412D168EA
:1074B000194A02EB04129068FFF785FD09E0164AAD
:1074C00002EB0412D168144A02EB04129068FFF731
:1074D00076FD042009F0C4FC0F4A02EB0412516847
:1074E0000D4A02EB04121068FFF76DFD042009F04D
:1074F000B7FC094A02EB04125168074A02EB041276
:107500001068FFF75CFD6806050E701CC6B2082EF9
:10751000C4DB00BFB4E70000F87A030010B50446EE
:107520001E4A02EB041251681C4A02EB0412106856
:10753000FFF745FD194A02EB0412D168174A02EB26
:10754000041290680122FFF711FD144A02EB0412A5
:10755000D168124A02EB04129068FFF734FD042050
:1075600009F07EFC0D4A02EB041251680B4A02EB53
:1075700004121068FFF727FD042009F071FC074A88
:1075800002EB04125168054A02EB04121068FFF77F
:1075900016FD042009F064FC10BD0000F87A030019
:1075A00010B51548FFF7D2FB012000F03BFCF4F7C3
:1075B000D3F9002201211148FFF7D8FC0022042151
:1075C0000E48FFF7D3FC012280214FF04020FFF747
:1075D000CDFC80214FF04020FFF7F5FCF2F7D4FFFF
:1075E000F7F73CFCF4F79EF9022000F0DBF8FFF718
:1075F00089F9F4F7B1F910BD0090D0034040004084
:1076000010B5F3F70FFC0120F2F70CFBF2F7EEF9DF
:1076100000BF00200149086000BF10BD000100400C
:1076200005460C46F3F7FEFB3F48006840F00200B9
:107630004FF08041C1F808020846D0F81C0220F43F
:107640008070394914310860384839490860084663
:107650000068012806D03548086000BF344800683B
:107660000128FBD100BF334A1168002003E0401C11
:10767000884200D906E02E4A526802F08072B2F1C8
:10768000807FF4D000BF284A143A126802F0010249
:107690001AB94AF66512264B5A6003E0401C88422C
:1076A00000D905E0224A526802F48032002AF5D05F
:1076B00000BF00BF02201E49C8622846F2F7B2FA96
:1076C000002201211C48F2F7F7FC01204FF0402175
:1076D0000867000419490860002204211648F2F7DF
:1076E000EBFC00224FF480511348F2F7E5FC002236
:1076F00040211248B038F2F7DFFC2046F1F788FF4E
:107700004FF08040D0F8900240F0080006498831E0
:1077100008600B480B4908604FF00D30091D0860E8
:10772000F2F764F900BFFEE7080200405713EBA52B
:10773000001004400000002040400040F0410040A4
:107740000D0D0809041104402DE9F04106460C46D0
:107750001746002526B1012E03D0022E1DD101E0CF
:107760001CE01BE004F0010008B145F0006504F0E6
:107770000200022801D145F0804504F004000428ED
:1077800001D145F4003504F01000102801D145F076
:10779000407529460620FFF743FF00BF00BFBDE844
:1077A000F081000038B50446022C41D100BF00BF73
:1077B00000BF59201F49086016208905C1F8000143
:1077C0008820C1F80001C006D0F800010028F0D0E0
:1077D00000BF0022C9141848F2F7BAF91648F1F7A9
:1077E0006DFF4FF08040406B1449084389034863A4
:1077F0004FF04020406A40F400504FF04021486272
:1078000001224FF470414FF04020F2F784FC0C4805
:1078100008230C22002100900A48F3F771F9094867
:10782000F3F769F900BF00200249086000BF00BFFC
:1078300038BD0000000100400F00A0660000555553
:1078400040420F00003006402DE9F04107460D464A
:10785000164600241548806820F00C0040F0010016
:107860001249886000BF09E010484069C0F34040F9
:1078700010B9285D0D490862601C84B2B442F3DB84
:1078800000BF0A48406900F001000028F9D107480C
:10789000806820F0080040F0050004498860084630
:1078A000F3F724F90120BDE8F08100000030064024
:1078B00070B505460C4600211548806820F00C0084
:1078C00040F00100124EB06000BF0DE0605C104E51
:1078D000306200BF0E48406900F001000028F9D175
:1078E0000B48006B5054491C9942EFD300BF084825
:1078F000406900F001000028F9D10548806820F0B7
:10790000080040F00500024EB060012070BD00008C
:107910000030064010B504460448406820B10348D2
:10792000214642680020904710BD0000CC00002096
:1079300010B504460448C06820B103482146C26817
:107940000120904710BD0000CC00002010B5044677
:107950000448406920B1034821464269022090470B
:1079600010BD0000CC00002010B504460448C069DA
:1079700020B103482146C2690320904710BD000092
:10798000CC00002010B504460448406A20B10348EA
:107990002146426A0420904710BD0000CC00002020
:1079A00010B504460448C06A20B103482146C26AA3
:1079B0000520904710BD0000CC00002010B5044603
:1079C0000448406B20B103482146426B0620904793
:1079D00010BD0000CC00002010B504460448C06B68
:1079E00020B103482146C26B0720904710BD00001C
:1079F000CC00002070B504460D4600BF00BF00BF9C
:107A00005920AE49086016208905C1F80001882078
:107A1000C1F80001C006D0F800010028F0D000BF76
:107A2000082C7DD2DFE804F0042E58847CAED8FE0A
:107A3000A348F1F743FEA348006800F4003040B9C2
:107A4000A0486038006820F040704FF08041C1F8D5
:107A500014024FF08040006B20F0FF004FF0804197
:107A600008630846006B40F0770008632420F2F7B3
:107A7000C8FF11219448F3F7F3FB29469248F3F726
:107A8000F3FB14E19148F1F719FE8E48006800F409
:107A9000003040B98B486038006820F040604FF0FB
:107AA0008041C1F814024FF08040C06C20F47F4048
:107AB0004FF08041C8640846C06C40F44C50C86424
:107AC0002520F2F79EFF11218148F3F7C9FB2946D3
:107AD0007F48F3F7C9FBEAE07E48F1F7EFFD79480C
:107AE000006800F4003040B976486038006820F043
:107AF00040704FF08041C1F814024FF08040406D5B
:107B000020F0FF004FF0804148650846406D40F08E
:107B1000770048653020F2F774FF11216E4800E0CD
:107B2000C4E0F3F79DFB29466B48F3F79DFBBEE0ED
:107B30006A48F1F7C3FD6348006800F4003040B9BB
:107B400060486038006820F040604FF08041C1F824
:107B500014024FF08040406D20F47F404FF0804190
:107B600048650846406D40F4EE4048653120F2F724
:107B700048FF11215A48F3F773FB29465848F3F799
:107B800073FB94E05748F1F799FD4E48006800F404
:107B9000003040B94B486038006820F040404FF05A
:107BA0008041C1F814024FF08040006B20F47F0048
:107BB0004FF0804108630846006B40F408000863FA
:107BC0004B20F2F71EFF11214748F3F749FB2946E6
:107BD0004548F3F749FB6AE04448F1F76FFD39483F
:107BE000006800F4003040B936486038006820F47E
:107BF00040104FF08041C1F814024FF08040406CBB
:107C000020F47F204FF0804148640846406C40F4E7
:107C1000AA2048646620F2F7F4FE11213448F3F7F5
:107C20001FFB00E00EE029463148F3F71DFB01225F
:107C300091023048FFF79AF94FF480612D48FFF721
:107C4000BEF934E02C48F1F739FD1E48006800F415
:107C5000003040B91B485838006820F440004FF00D
:107C60008041C1F81C024FF08040406B20F0FF00C3
:107C70004FF0804148630846406B40F088004863FD
:107C80006720F2F7BEFE11211C48F3F7E9FA2946F6
:107C90001A48F3F7E9FA012251021648FFF766F98C
:107CA0004FF400711348FFF78AF900E000BF00BFEE
:107CB00000BF00200149086000BF70BD0001004006
:107CC000103D80577402004000000740913DA057CE
:107CD00000100740123C8C7700200740933CAC77A3
:107CE00000300740953DEC7700500740163E4C773A
:107CF0000060074080400040973E6C77007007406E
:107D00002DE9F04104460E4617460025082C01DBFC
:107D1000BDE8F081082C1DD2DFE804F00405060759
:107D200008090A1317E016E015E014E013E012E06A
:107D30004FF480612748FFF746F902201CF0CEFF80
:107D400009E04FF400712348FFF73DF902201CF0D1
:107D5000C5FF00E000BF00BF1F4951F834003A469C
:107D60003146F3F74FFB002507E0681C85B2012080
:107D70001CF0B4FF142D00DB07E0174850F8340066
:107D80008069C0F300700028EFD000BF082C1DD21E
:107D9000DFE804F00405060708090A1317E016E0F7
:107DA00015E014E013E012E002201CF097FF4FF4FE
:107DB00080610848FFF703F909E002201CF08EFFFC
:107DC0004FF400710348FFF7FAF800E000BF00BF6E
:107DD00000BF9DE780400040CC000020082800DB69
:107DE0007047034A02EBC002516000BFF8E7000091
:107DF000CC00002010B5F3F701F845F6A5200649A0
:107E0000886000BF00200549086000BFC91304480E
:107E1000FFF7DDF810BD0000000004400001004045
:107E20000041004010B50446F2F7E8FF0122D103FB
:107E30002E48FFF79BF84FF08040406800F00400A8
:107E4000D0B12B48006840F000404FF08041C1F8AD
:107E500094020620F1F7E6FE2548001F00684FF067
:107E60008041C1F890020846D0F8900240F480703A
:107E7000C1F89002F1F7BAFD00BF00201D4908606B
:107E800000BF4FF0AC40F1F719FC002203214FF086
:107E9000AC40F1F75DFE08200121814042099200CB
:107EA00002F1E022C2F8001100BFF2F7A7FF3CB9CF
:107EB00001231A4600214FF4A060F3F727FB06E0E8
:107EC00001231A4600214FF4C060F3F71FFB00BFE7
:107ED0000948006840F040000749086000BF00BF43
:107EE00000200449086000BF10BD000000410040B0
:107EF00094020040000100400000044010B500243E
:107F000053201DF01FFA08B144F0080403200EF0BE
:107F100035F808B144F0100402200EF02FF808B133
:107F200044F0200401200EF029F808B144F0400488
:107F300000200EF023F808B144F08004204610BD64
:107F400070B5B2B004460D461646642119A8F0F784
:107F500056FA2146684600F027F86422694619A8B7
:107F6000F0F734FAADF86C50ADF86E60094807C808
:107F700012F04EFC60B958221CA96846F0F726FAA8
:107F8000044819A90EC912F010FC012032B070BDCE
:107F90000020FBE7E850002010B5002000F0A0F919
:107FA00000F0B2F910BD00002DE9F0412DED048B79
:107FB0009CB007460D46642103A8F0F720FA002480
:107FC000002600200190029001A8F2F787FC5220C1
:107FD0001DF0B8F9C0B28DF80C00BDF80A00A0F58C
:107FE000FA60C0B28DF80D009DF809008DF80E0002
:107FF0009DF808008DF80F009DF806008DF8100020
:108000009DF805008DF811009DF804008DF8120010
:108010008DF8135006201DF095F9ADF818000820D2
:108020001DF090F9ADF81A0031201DF08BF9804653
:10803000F0F799FB41EC190B9FED6D0B53EC102BF6
:10804000F0F79FFA41EC180BF0F7B9FBC0B28DF8CE
:108050001C0040F209100FF0FBFEC6B2642E00DDDA
:1080600064268DF81D6030201DF06CF9C0B28DF8CB
:108070001E001420F2F71EFB30B99DF81E0020F000
:10808000080008308DF81E001120F2F713FB18B11C
:108090001C20F2F70FFB30B99DF81E0020F02000E5
:1080A00020308DF81E000A20F2F704FB30B99DF84D
:1080B0001E0020F0800080308DF81E000B20F2F7AB
:1080C000F9FA30B99DF81E0020F0400040308DF8DC
:1080D0001E0035201DF036F9C0B28DF81F00FCF7E8
:1080E00065FB0890FCF768FB099040F205100FF063
:1080F000AFFEADF828004FF482700FF0A9FEADF886
:108100002A0032201DF01EF9ADF82C0042201DF08F
:1081100019F9804641201DF015F908EB0040CDF813
:10812000360044201DF00EF9804643201DF00AF968
:1081300008EB0040CDF832000A201DF003F900B230
:10814000ADF82E0009201DF0FDF800B2ADF83000AA
:108150003F200FF07DFEC0B28DF83A009DF83A0046
:10816000102802DB10208DF83A0000240AE004F108
:108170000C001DF0E7F80DF13B0101EB4401088014
:10818000601CC4B29DF83A00A042F0DC16F0BCFDC1
:108190008DF85B00002417E004F11C001DF0D2F8FC
:1081A0008046F0F7E0FA41EC190B9FED130B53EC0E
:1081B000102BF0F7E6F941EC180BF0F700FBC1B219
:1081C00017A80155601CC4B29DF85B00A042E3DC17
:1081D0004FF484700FF03CFEADF86400642203A9F4
:1081E0003846F0F7F3F81CB0BDEC048BBDE8F08125
:1081F0007B14AE47E17A843F9A9999999999B93F4E
:108200000548B0F801004FF4FA7190FBF1F201FB60
:10821000120080B270470000F45000200648B0F809
:108220000100B0F5FA7F02DD4FF4FA7070470248A2
:10823000B0F80100FAE70000F450002010B5044A3D
:108240000A21044812F0D2FA00F02CF810BD000008
:10825000004D0020E8500020F0B599B004460D46CE
:10826000002700BF64216846F0F7C9F814B940F24E
:10827000F31000E0601E84B204EBC40000EB0410B5
:1082800040F6424101EB8006642269463046F2F72F
:10829000DBFA642269462846F0F798F8384619B0A8
:1082A000F0BD000010B500240A220C494FF44360D1
:1082B000F2F7CAFA0446012C0CD1084800785A2873
:1082C00003D10648407AA52804D0002000F008F821
:1082D00000F01AF80148B0F8010010BDF450002079
:1082E0005A21084A11701146A1F80100C143A2F8B1
:1082F00003101146A1F80500C143A2F80710A521FB
:1083000051727047F450002010B500240A2204492D
:108310004FF44360F2F7B6FA0446204610BD000061
:10832000F450002070B59AB000240025642101A803
:10833000F0F765F80026244807C812F05EFAE0BBA3
:1083400001A9214812F06CFA2048B0F801004FF45E
:10835000FA7190FBF1F201FB120084B204EBC4004D
:1083600000EB041040F6424101EB8005642201A9B4
:108370002846F2F787FA06461448B0F80100401C78
:108380001249A1F801000846B0F80100B0F5FA7FE3
:108390000DDB0846B0F801004FF4FA7190FBF1F2E2
:1083A00001FB120000F5FA700849A1F80100074925
:1083B000B1F80100FFF794FF00E001E0FFF7A4FF30
:1083C00030461AB070BD0000E8500020F450002084
:1083D0002DE9F0472DED0A8B04460D464FF00009BC
:1083E00000260027B046B246E08850B9E068058014
:1083F0000020A0800120E0802846BDEC0A8BBDE86B
:10840000F087E088401EE16831F81060B54202DB79
:10841000A5EB060901E0A6EB05092089484508DA25
:10842000E06805800020A0800120E08020702846C0
:10843000E3E700202070A088401CA080A08861880D
:10844000884201DB0020A080A188E06820F811505C
:10845000E088401CE080E0886188884201DD608817
:1084600000E0E088E080002705E0E06830F81700D1
:108470008044781C87B2E088B842F6DCE088F0F7E8
:1084800072F941EC1A0B4046F0F76DF941EC1C0B08
:108490009FED0D0B53EC102BF0F773F841EC1B0B19
:1084A00053EC1A2BF0F7DFF841EC190B9FED080B9A
:1084B00053EC102BEFF7BEFF41EC180BF0F77FF9F0
:1084C0001FFA80FA504698E7000000000000F03FD5
:1084D000000000000000E03F2DE9F0472DED0A8B81
:1084E00004460E464FF00009CA4600250027A8465C
:1084F000E08850B9E06806800020A0800120E0807C
:108500003046BDEC0A8BBDE8F087E088401EE1688C
:1085100031F810A000202070A088401CA080A08806
:108520006188884201DB0020A080A188E06820F8F3
:108530001160E088401CE080E0886188884201DDAD
:10854000608800E0E088E080E08806282FDA0025D7
:1085500005E0E06830F815000744681C85B2E08843
:10856000A842F6DCE088F0F7FEF841EC1A0B38463A
:10857000F0F7F9F841EC1C0B9FED260B53EC102B98
:10858000EFF7FFFF41EC1B0B53EC1A2BF0F76BF8E6
:1085900041EC190B9FED210B53EC102BEFF74AFF29
:1085A00041EC180BF0F70BF91FFA80F830E00325C7
:1085B00005E0E06830F815000744681C85B2E088E3
:1085C000C01EA842F5DCE188881FF0F7BBF841EC3B
:1085D0001A0B3846F0F7C7F841EC1C0B9FED0D0B5A
:1085E00053EC102BEFF7CDFF41EC1B0B53EC1A2B88
:1085F000F0F739F841EC190B9FED080B53EC102BF9
:10860000EFF718FF41EC180BF0F7D9F81FFA80F8D4
:10861000404676E7000000000000F03F0000000048
:108620000000E03F10B5C1604280038100248480D7
:10863000C48010BD37B503460021002202980068AF
:10864000984207D3BDF80400401E029C54F8200055
:10865000984201D924483EBD00213EE0029850F8DE
:108660002100984237D3481C029C54F820009842BD
:1086700031D8029850F821400546481C55F8200092
:10868000201A00EE100AF8EE400A481C029C54F82A
:10869000200000EE100AB8EE401A00EE103AB8EED4
:1086A000400A30EE410AB2EE041A20EE010A80EED2
:1086B000201A481C00EB8000400000EE100AB8EEC3
:1086C000C00A30EE410ABDEEC00A10EE102AA2F533
:1086D000C87000B2BFE7481C81B2BDF80400401E5C
:1086E0008842BBDC0048B6E766FEFFFF70B5044673
:1086F0000D462046F2F7AAFB204670BD00207047C9
:10870000002070470020704700207047002070470D
:1087100010B500240220FCF755F898B90020FCF7AA
:1087200051F878B90420FCF74DF858B90820FCF747
:1087300049F838B90A20FCF745F818B90520FCF7C4
:1087400041F808B144F001040320FCF73BF8B8B944
:108750000120FCF737F898B90620FCF733F878B910
:108760000A20FCF72FF858B90B20FCF72BF838B982
:108770000720FCF727F818B91220FCF723F808B1F6
:1087800044F002040F20FCF71DF898B91320FCF701
:1087900019F878B91420FCF715F858B90D20FCF732
:1087A00011F838B90D20FCF70DF818B90C20FCF7BA
:1087B00009F808B144F004040820FCF703F818B9DC
:1087C0000920FBF7FFFF08B144F008040A20FBF77B
:1087D000F9FF18B90B20FBF7F5FF08B144F01004BE
:1087E00002200DF0CBFB08B144F4805402200DF0C0
:1087F000C5FB08B144F4005401200DF0BFFB08B9DB
:1088000044F4804400200DF0B9FB08B944F400445E
:10881000204610BD10B500240520FBF7B9FF08B1B4
:1088200044F001040420FBF7B3FF08B144F0020454
:108830000620FBF7C7FF18B90720FBF7C3FF08B1F5
:1088400044F0F1040420FBF7BDFF08B144F0F2044A
:10885000204610BD10B500240720FBF799FF08B192
:1088600044F001040620FBF793FF08B144F0020432
:108870001420FBF7A7FF08B144F0F0040920FBF730
:10888000A1FF18B90B20FBF79DFF08B144F0F104DC
:108890000820FBF797FF18B90A20FBF793FF08B1F0
:1088A00044F0F204204610BD08B500200090424874
:1088B00090F84E00C0F3801028B93F4890F84E0061
:1088C000C0F3C01028B1BDF8000020F00100401C2A
:1088D00000903948D0F84E00C0F3804028B1BDF870
:1088E000000020F00200801C00903348B0F84E00D9
:1088F000C0F3802028B1BDF8000020F01000103037
:1089000000902D48B0F84E00C0F3002028B1BDF80B
:10891000000020F02000203000902748B0F84E00E2
:10892000C0F3C02028B1BDF8000020F04000403066
:1089300000902148B0F84E00C0F3402028B1BDF8A7
:10894000000020F08000803000901B4890F84E001E
:10895000C0F3001030B1BDF8000020F4006000F555
:10896000006000901448B0F84E00C0F3003030B101
:10897000BDF8000020F4805000F5805000900E48B3
:10898000B0F84E00C0F3403030B1BDF8000020F424
:10899000005000F5005000900748B0F84E00C0F3BA
:1089A000803030B1BDF8000020F4804000F58040F8
:1089B0000090BDF8000008BD0CD2002010B50024C6
:1089C0000C20FBF7E5FE08B144F001040B20FBF797
:1089D000DFFE08B144F002040E20FBF7F3FE08B1FD
:1089E00044F0F1040D20FBF7EDFE08B144F0F20471
:1089F000204610BD00202449D1F84E10C1F340514B
:108A000009B140F001002049D1F84E10C1F3805166
:108A100009B140F002001C49D1F84E10C1F30051D9
:108A200009B140F004001849D1F84E10C1F3C0411B
:108A300009B140F010001449D1F84E10C1F3806123
:108A400009B140F020001049D1F82A10002902DDB8
:108A500040F4807006E00C49D1F82A10002901DAB0
:108A600040F40070084991F85E1001F0020109B16C
:108A700040F48060044991F85E1001F0010109B1F1
:108A800040F40060704700000CD200200020244910
:108A9000D1F84E10C1F3405109B140F00100204916
:108AA000D1F84E10C1F3805109B140F002001C49C9
:108AB000D1F84E10C1F3005109B140F0040018493B
:108AC000D1F84E10C1F3C04109B140F01000144973
:108AD000D1F84E10C1F3806109B140F02000104977
:108AE000D1F82A10002902DD40F4807006E00C491C
:108AF000D1F82A10002901DA40F40070084991F8F1
:108B00005E1001F0020109B140F48060044991F85F
:108B10005E1001F0010109B140F4006070470000EF
:108B20000CD2002000201449D1F84E10C1F340515E
:108B300009B140F001001049D1F84E10C1F3805145
:108B400009B140F002000C49D1F84E10C1F30051B8
:108B500009B140F004000849D1F84E10C1F3C041FA
:108B600009B140F010000449D1F84E10C1F3806102
:108B700009B140F0200070470CD2002000201449B9
:108B8000D1F84E10C1F3405109B140F00100104935
:108B9000D1F84E10C1F3805109B140F002000C49E8
:108BA000D1F84E10C1F3005109B140F0040008495A
:108BB000D1F84E10C1F3C04109B140F01000044992
:108BC000D1F84E10C1F3806109B140F02000704728
:108BD0000CD2002001460020012900D128E0022902
:108BE00001D1012024E0032901D1042020E007293C
:108BF00001D109201CE00B2901D10E2018E00A291F
:108C000001D1032014E0082901D1022010E0052938
:108C100001D106200CE0142901D10C2008E006291E
:108C200001D10D2004E00E2901D10B2000E000202D
:108C3000704770B505460024FD200FF009F9C4B255
:108C4000012D01D100240CE0022C01D1012408E007
:108C5000032C01D1022404E00D2C01D1062400E0F4
:108C60000124204670BD08B50020009008BD00001A
:108C700008B500200090304890F84E000009BDF87B
:108C8000001060F3082100912B4890F84E00C0F3CB
:108C90008010294991F84E10C1F3C011084328B142
:108CA000BDF8000020F08000803000902248B0F82D
:108CB0004E00C0F300202049B1F84E10C1F38021CE
:108CC000084328B1BDF8000020F0080008300090EB
:108CD0001948B0F84E00C0F3402028B1BDF800009C
:108CE00020F01000103000901348B0F84E00C0F390
:108CF000C02028B1BDF8000020F0200020300090F6
:108D00000D48D0F84E00C0F3C04058B90A48D0F81A
:108D10004E00C0F3005028B90748D0F84E00C0F309
:108D2000405030B1BDF8000020F4006000F5006054
:108D30000090BDF8000008BD0CD2002000201049B2
:108D400091F85E1001F0010109B140F001000C49F9
:108D500091F85E1001F0020109B140F002000849EB
:108D6000D1F82A10002902DD40F0040006E0044991
:108D7000D1F82A10002901DA40F0080070470000FD
:108D80000CD2002010B5002430201CF0DBFA00F0DB
:108D9000010008B144F0010430201CF0D3FA00F0C7
:108DA000020008B144F00204204610BD10B50024B2
:108DB0000A20FBF7EDFC08B144F002040C20FBF79D
:108DC00001FD08B144F0F204204610BD10B50024A6
:108DD0000120FBF7DDFC18B90320FBF7D9FC08B133
:108DE00044F001040020FBF7D3FC18B90320FBF783
:108DF000CFFC08B144F002040120FBF7E3FC18B9F2
:108E00000320FBF7DFFC08B144F0F1040020FBF77E
:108E1000D9FC18B90320FBF7D5FC08B144F0F204E3
:108E2000204610BD70B500250024FB200FF010F87F
:108E3000C4B20CB9012528E0012C01D1022524E09F
:108E4000042C01D1032520E0092C01D107251CE0C9
:108E50000E2C01D10B2518E0032C01D10A2514E0BA
:108E6000022C01D1082510E0062C01D105250CE0CB
:108E70000C2C01D1142508E00D2C01D1062504E0AD
:108E80000B2C01D10E2500E00125284670BD70B5E0
:108E900000250024FD200EF0DBFFC4B20CB9012533
:108EA0000CE0012C01D1022508E0022C01D10325A0
:108EB00004E0062C01D10D2500E00125284670BDF7
:108EC0000020194991F84E10C1F3801129B91649B3
:108ED00091F84E10C1F3C01109B140F4005012498D
:108EE000B1F84E10C1F3002129B90F49B1F84E1065
:108EF000C1F3802109B140F008000B49B1F84E10D0
:108F0000C1F3402129B90849B1F84E10C1F3C0217D
:108F100009B140F004000449B1F84E10C1F300312A
:108F200009B140F0020070470CD2002000201B491C
:108F3000D1F84E10C1F3804109B140F0100017493B
:108F400091F84E10C1F3001129B9144991F84E104F
:108F5000C1F3801109B140F020001049B1F84E1062
:108F6000C1F3002109B140F040000C49B1F84E10A6
:108F7000C1F3402109B140F080000849B1F84E101A
:108F8000C1F3802109B140F480700449B1F84E105A
:108F9000C1F3C02109B140F4007070470CD2002029
:108FA0000020194991F84E10C1F3801129B91649D2
:108FB00091F84E10C1F3C01109B140F400501249AC
:108FC000B1F84E10C1F3002129B90F49B1F84E1084
:108FD000C1F3802109B140F008000B49B1F84E10EF
:108FE000C1F3402129B90849B1F84E10C1F3C0219D
:108FF00009B140F004000449B1F84E10C1F300314A
:1090000009B140F0020070470CD200200021214835
:1090100090F84E00C0F3801028B91E4890F84E001A
:10902000C0F3C01008B141F400511A4890F84E0046
:10903000C0F3001028B9174890F84E00C0F3001094
:1090400008B141F480411348B0F84E00C0F300204D
:1090500028B91048B0F84E00C0F3802008B141F0A4
:1090600008010C48B0F84E00C0F3402028B9094868
:10907000B0F84E00C0F3C02008B141F0040105482B
:10908000B0F84E00C0F3003008B141F002010020FA
:10909000704700000CD2002000203B49B1F84E1070
:1090A000C1F30021B9B93849B1F84E10C1F300211C
:1090B00089B93549B1F84E10C1F3802159B9324907
:1090C000B1F84E10C1F3003129B92F49B1F84E1053
:1090D000C1F3403109B140F008002B49B1F84E10FE
:1090E000C1F3402159B92849B1F84E10C1F3C0214C
:1090F00029B92549B1F84E10C1F3803109B140F0CA
:109100001000214991F84E10C1F380111E4A92F8C7
:109110004E20C2F3C012114309B140F080001A4939
:1091200091F84E10C1F30011174A92F84E20C2F385
:109130004012114309B140F480701349D1F84E1028
:10914000C1F38041E9B91049D1F84E10C1F3405143
:10915000B9B90D49D1F84E10C1F3805189B90A4906
:10916000D1F84E10C1F3806159B90749D1F84E10BA
:10917000C1F3C04129B90449D1F84E10C1F30051DF
:1091800009B140F4006070470CD2002000202E4945
:1091900091F84E10C1F3001129B92B4991F84E10E6
:1091A000C1F3401109B140F01000274991F84E1069
:1091B000C1F3801129B9244991F84E10C1F3C011AF
:1091C00009B140F020002049D1F84E10C1F3804190
:1091D00009B140F040001C49B1F84E10C1F3002124
:1091E00009B140F480701849B1F84E10C1F38021E4
:1091F00009B140F400701449B1F84E10C1F3402198
:1092000009B140F480601049B1F84E10C1F3C0219B
:1092100009B140F400600C49B1F84E10C1F30031BF
:1092200009B140F480500849B1F84E10C1F3403103
:1092300009B140F400500449B1F84E10C1F3803137
:1092400009B140F4804070470CD2002000202E4924
:1092500091F84E10C1F3001129B92B4991F84E1025
:10926000C1F3401109B140F01000274991F84E10A8
:10927000C1F3801129B9244991F84E10C1F3C011EE
:1092800009B140F020002049D1F84E10C1F38041CF
:1092900009B140F040001C49B1F84E10C1F3002163
:1092A00009B140F480701849B1F84E10C1F3802123
:1092B00009B140F400701449B1F84E10C1F34021D7
:1092C00009B140F480601049B1F84E10C1F3C021DB
:1092D00009B140F400600C49B1F84E10C1F30031FF
:1092E00009B140F480500849B1F84E10C1F3403143
:1092F00009B140F400500449B1F84E10C1F3803177
:1093000009B140F4804070470CD2002000202E4963
:1093100091F84E10C1F3001129B92B4991F84E1064
:10932000C1F3401109B140F01000274991F84E10E7
:10933000C1F3801129B9244991F84E10C1F3C0112D
:1093400009B140F020002049D1F84E10C1F380410E
:1093500009B140F040001C49B1F84E10C1F30021A2
:1093600009B140F480701849B1F84E10C1F3802162
:1093700009B140F400701449B1F84E10C1F3402116
:1093800009B140F480601049B1F84E10C1F3C0211A
:1093900009B140F400600C49B1F84E10C1F300313E
:1093A00009B140F480400849B1F84E10C1F3403192
:1093B00009B140F480500449B1F84E10C1F3803136
:1093C00009B140F4005070470CD2002000202C4915
:1093D00091F84E10C1F3001129B9294991F84E10A6
:1093E000C1F3401109B140F02000254991F84E1019
:1093F000C1F3801129B9224991F84E10C1F3C0116F
:1094000009B140F001001E49B1F84E10C1F300212E
:1094100029B91B49B1F84E10C1F3802109B140F0C0
:1094200004001749B1F84E10C1F3402129B914497D
:10943000B1F84E10C1F3C02109B140F0020010494B
:10944000D1F84E10C1F3C041B9B90D49D1F84E1051
:10945000C1F3005189B90A49D1F84E10C1F38061B6
:1094600059B90749D1F84E10C1F3405129B90449FF
:10947000D1F84E10C1F3805109B140F0400070475F
:109480000CD2002008B50246002100200090C2EB5B
:109490000213474800EBC300B0F8401001F0010090
:1094A00020B1009820F00100401C009001F0020063
:1094B00020B1009820F00200801C009001F0040010
:1094C00020B1009820F020002030009001F008002A
:1094D00020B1009820F010001030009001F0100032
:1094E00020B1009820F00400001D009001F0200041
:1094F00020B1009820F008000830009001F04000F2
:1095000020B1009820F040004030009001F0800031
:1095100020B1009820F080008030009001F480702D
:1095200028B1009820F4807000F58070009001F45C
:10953000007028B1009820F4007000F500700090D1
:1095400001F4806028B1009820F4806000F580600C
:10955000009001F4006028B1009820F4004000F56C
:109560000040009001F4805028B1009820F4006081
:1095700000F50060009001F4005028B1009820F43C
:10958000805000F58050009001F4804028B1009890
:1095900020F4005000F50050009001F4004028B184
:1095A000009820F4802000F580200090009808BDED
:1095B00075D2002008B5014600200090C1EB0112D1
:1095C0007A4800EBC20090F83A00009A60F300027B
:1095D0000092C1EB0112754800EBC20090F83A000E
:1095E0004208009862F341000090C1EB01126F48FD
:1095F00000EBC20090F83A008209009862F3820002
:109600000090C1EB0112694800EBC20090F83A00EB
:10961000C209009862F3C3000090C1EB01126348D5
:1096200000EBC20090F83A000209009862F30410BF
:109630000090C1EB01125D4800EBC20090F83A00C7
:109640008208009862F386100090C1EB011257481F
:1096500000EBC20090F83A00C208009862F3C7100D
:109660000090C1EB0112514800EBC20090F83A00A3
:109670004209009862F392400090C1EB01124B48FE
:1096800000EBC200408F020A009862F3D3400090C2
:10969000C1EB0112454800EBC200408F420A00981E
:1096A00062F39A600090C1EB0112404800EBC200E7
:1096B000408F820A009862F3CF300090C1EB011214
:1096C0003A4800EBC20090F83C004208009862F370
:1096D00008200090C1EB0112344800EBC20090F862
:1096E0003C00C208009862F38A200090C1EB01128E
:1096F0002E4800EBC20090F83C00009A60F349222B
:109700000092C1EB0112294800EBC20090F83C0026
:109710008208009862F3CB200090C1EB011223482D
:1097200000EBC20090F83C000209009862F30C3094
:109730000090C1EB01121D4800EBC20090F83C0004
:109740008209009862F38E300090C1EB0112174835
:1097500000EBC20090F83C004209009862F34D30E3
:109760000090C1EB0112114800EBC20090F83C00E0
:10977000C209009862F355500090C1EB01120B48EA
:1097800000EBC200808F020A009862F396500090AE
:10979000C1EB0112054800EBC200808F420A00981D
:1097A00062F314500090009808BD000075D20020AC
:1097B00070B50024002530201BF0C4FDC5B205F0B3
:1097C000020008B144F0010405F0010008B144F0C2
:1097D000020435201BF0B6FDC5B2022D02D144F0C3
:1097E000080403E0012D01D144F004041120F0F736
:1097F00061FF08B944F010040A20F0F75BFF08B9D4
:1098000044F020040B20F0F755FF08B944F0400461
:10981000204670BD01460020C1EB0113294A02EB2E
:10982000C30292F83E2002F001020AB140F00100AA
:10983000C1EB0113234A02EBC30292F83E2002F06F
:1098400002020AB140F00200C1EB01131D4A02EB13
:10985000C30292F83E2002F008020AB140F0040070
:10986000C1EB0113174A02EBC30292F83E2002F04B
:1098700004020AB140F00800C1EB0113114A02EBE7
:10988000C30292F83E2002F010020AB140F010002C
:10989000C1EB01130B4A02EBC30292F83E2002F027
:1098A00020020AB140F02000C1EB0113054A02EB8F
:1098B000C30292F83E2002F040020AB140F040009C
:1098C0007047000075D2002008B500200090304895
:1098D000D0F82A00002806DDBDF8000020F00300C3
:1098E000801C009011E02A48D0F82A00002806DAEF
:1098F000BDF8000020F00300C01C009005E0BDF89A
:10990000000020F00300401C0090BDF8000020F093
:1099100004000090BDF8000020F008000090BDF8A1
:10992000000020F01000009000200CF027FBBDF894
:10993000001060F38611009101200CF01FFBBDF8B0
:10994000001060F345110091BDF8000020F0800088
:1099500000900F484088012807DDBDF8000020F482
:10996000407000F58070009004E0BDF8000020F425
:109970004070009003200CF001FB30B1BDF80000F6
:1099800020F4805000F580500090BDF8000008BD24
:109990000CD2002070B50024002530201BF0D2FC32
:1099A000054605F0020008B144F0010405F001008D
:1099B00008B144F002041620F0F77CFE08B944F028
:1099C00004041420F0F776FE08B944F008041320CC
:1099D000F0F770FE08B944F010040B20F0F76AFEAF
:1099E00008B944F020040A20F0F764FE08B944F0F6
:1099F00040041120F0F75EFE08B944F080042046D0
:109A000070BD000001460020C1EB01132E4A02EB9D
:109A1000C30292F83E2002F001020AB140F00100B8
:109A2000C1EB0113284A02EBC30292F83E2002F078
:109A300002020AB140F00200C1EB0113224A02EB1C
:109A4000C30292F83E2002F010020AB140F08000FA
:109A5000C1EB01131C4A02EBC30292F83E2002F054
:109A600020020AB140F04000C1EB0113164A02EB9C
:109A7000C30292F83E2002F040020AB140F02000FA
:109A8000C1EB0113104A02EBC30292F83E2002F030
:109A900080020AB140F01000C1EB01130A4A02EB48
:109AA000C302D28F02F480720AB140F00800C1EB09
:109AB0000113054A02EBC302D28F02F400720AB10D
:109AC00040F004007047000075D2002010B500245B
:109AD0000020F0F7CBFD08B944F001040120F0F7B5
:109AE000C5FD08B944F002040A20F0F7BFFD08B92B
:109AF00044F00404204610BD01460020C1EB0113D0
:109B00000F4A02EBC302D28F02F480620AB140F026
:109B10000100C1EB01130A4A02EBC302D28F02F427
:109B200000620AB140F00200C1EB0113044A02EBEB
:109B3000C302D28F02F480520AB140F00400704791
:109B400075D2002010B50024D1201BF0FBFB0028AB
:109B500001DD44F00104D2201BF0F4FB002801DDFC
:109B600044F0020402200CF009FA012801D144F06B
:109B7000040403200CF002FA012801D144F0080487
:109B80001920FAF71FFE08B144F01004204610BD5A
:109B90002DE9F04105460E460024002700BF2DE0C8
:109BA00004EB4400184901EB80008088284404EB52
:109BB0004401154A02EB8101888004EB4400114600
:109BC00001EB8000808804EB440102EB81014988AD
:109BD000884211DB002004EB440102EB8101888004
:109BE0003A467B1CDFB206EB021004EB4402064B44
:109BF00003EB820291688847601CC4B2092CCFD362
